:100000000C944C0B0C947D0B0C947D0B0C947D0B81
:100010000C947D0B0C947D0B0C947D0B0C947D0B40
:100020000C947D0B0C947D0B0C947D0B0C947D0B30
:100030000C947D0B0C947D0B0C947D0B0C947D0B20
:100040000C947D0B0C947D0B0C947D0B0C947D0B10
:100050000C947D0B0C947D0B0C947D0B0C94F48A0A
:100060000C947D0B0C94D76D0C94AD6D0C947D0BA2
:100070000C947D0B0C947D0B0C947D0B0C947D0BE0
:100080000C947D0B0C947D0B0C947D0B0C947D0BD0
:100090000C94836D0C94596D0C947D0B0C94BD21C4
:1000A0000C947D0B0C947D0B0C947D0B0C947D0BB0
:1000B0000C947D0B0C947D0B0C947D0B0C947D0BA0
:1000C0000C947D0B0C947D0B0C947D0B0C942F6D7C
:1000D0000C94056D0C947D0B0C947D0B0C947D0B96
:1000E0000C947D0B07634236B79BD8A71A39685624
:1000F00018AEBAAB558C1D3CB7CC5763BD6DEDFD4A
:10010000753EF6177231BF000000803F0800000006
:10011000BE922449123EABAAAA2ABECDCCCC4C3EFC
:1001200000000080BEABAAAAAA3E00000000BF00EB
:100130000000803F0000000000084178D3BB4387E7
:10014000D1133D190E3CC3BD4282AD2B3E68EC82FB
:1001500076BED98FE1A93E4C80EFFFBE01C4FF7F80
:100160003F00000000000C948F650C94F9280C945B
:10017000751A0C94130D0C947C130C94080F0C94AA
:10018000CC3E0C94F20C0C94322A0C9469630C94BF
:1001900027830C9403640C94BD200C944E840C941F
:1001A00035830C9407120C9414610C94E6830C9420
:1001B000F60C0C941F130C9411150C94CC6F0C942A
:1001C000DC190C9427620C946D610C942E0D0C9428
:1001D000FE640C9462840C941E510C945B110C947C
:1001E0001E620C942D9D0C949E3C0C94C64C0C9459
:1001F00025130C94D3100C948A100C9421620C9447
:1002000057630C9485290C9430520C9483280C94D9
:10021000F6100C94E90C0C9413830C94EE830C945C
:100220002D630C94122A0C9439830C940D990C9420
:10023000C30E0C9456150C94C23C0C947C2C0C945C
:100240008C2C0C9413150C948E280C94210D0C946A
:10025000AF0B0C94990B0C94F3180C940F1A0C948C
:100260000C0D0C9421830C940F150C9419130C9401
:10027000199D0C94D2290C9424320C94FD610C9499
:1002800052200C94F5120C94A95C0C94D8A90C94EF
:1002900097510C9476840C94C1280C9419830C9477
:1002A000A63F0C94B40E0C94034D0C947E510C9408
:1002B0007A9D0C94E5590C94950B0C94FD830C9449
:1002C000463F0C9440830C9402280C9405510C94E6
:1002D00005700C94E9270C94A0190C94ED0C0C9467
:1002E0004D1C0C942B830C9411840C94D9500C94B9
:1002F000DB560C9409830C940C4D0C9449290C94F6
:100300008D500C940D150C9424210C94CD300C942C
:1003100013100C94352E0C946C840C94EA0C0C94F1
:100320001B970C94CF270C943E6F0C94C6170C941B
:1003300070630C94BB0F0C94A6500C94095A0C9447
:10034000D41F0C941B640C944F210C94BA6F0C9422
:10035000D0190C942B840C94F4200C94C4190C9494
:1003600058840C94920F0C9405280C94A0560C946D
:100370005B290C94E3630C94FB660C94FA3F0C9499
:1003800038400C9433180C9435190C94F90E0C94D5
:10039000209D0C943B2E0C9401830C944D9D0C9449
:1003A00000610C94460D0C94260D0C94ED100C94E9
:1003B000EC110C9402630C9441830C9407840C940C
:1003C000170D0C940C690C946A4C0C945E3C0C94C4
:1003D00097620C94064D0C94803C0C9470290C94FC
:1003E00033520C94322E0C941E630C944D0D0C94CD
:1003F000CE110C9440490C94FB0C0C94CD280C9419
:10040000E84C0C94F81A0C948C200C9435840C94C1
:10041000F30C0C94F94C0C94E4140C9442250C94B9
:10042000FE120C94230D0C9461100C9410290C9462
:10043000C9130C94EA0E0C9430290C94AA600C9405
:10044000D1280C943F840C94F1600C9423500C94AC
:100450009C0E0C945F9D0C945D510C940F0D0C94AC
:10046000DC1A0C94A50E0C94FF100C94194D0C94EE
:10047000360D0C948F0F0C94C72D0C941D830C9487
:10048000586F0C9467640C94151B0C9421840C9485
:10049000F3830C9454100C946F6F0C9439520C9499
:1004A00033120C9458500C94FF510C94A29C0C9451
:1004B000CC230C94774C0C94611E0C94A4280C94BF
:1004C000E0120C940F830C9469290C9432400C9424
:1004D000BA0B0C94AFA90C94324D0C94320D0C94C1
:1004E00014970C94B0620C94DB0C0C94E3590C94AC
:1004F00070100C948C1A0C94331C0C941F290C94BF
:10050000E30E0C943D830C9405830C94D5290C9434
:10051000F00E0C94DF0F0C94815D0C949C980C945D
:1005200098290C9475290C9448710C947F0B0C94A9
:1005300023940C94A8950C94D8160C9436520C94D1
:1005400019840C944F6F0C94D5260C9455120C946E
:10055000A9100C94FE0C0C94B35C0C942F830C9497
:100560007F3A0C94B4610C9480840C9464620C9473
:1005700022610C94A40F0C94BC0E0C940F4D0C949F
:10058000FB820C94D74C0C94CF170C9417620C94EC
:10059000AB600C94D8186364696E6F70737578588B
:1005A0005B00556E6B6E6F776E207375666669784B
:1005B0002000556E6B6E6F776E20636D6420006354
:1005C0006C724374723A20005365656B3A002F00D9
:1005D000496E3A20002D3E002000230050656E64D5
:1005E00065642073746174652072657472696576E0
:1005F00065643A003D004C454741435920494E3A15
:10060000003D00494E3A000000200023002600294A
:10061000002C002F00320000010000030106010938
:10062000017261770076616C0074656D70007361B2
:1006300074006875650066616E0052474200485359
:1006400056006D6F646500536574436D643A0053E2
:100650006574466C61673A00436C72466C61673A38
:100660000053746F726564204558543A0073756680
:10067000666978436F64653A0054787432436D64F8
:100680003A004452590046414E5F4F4E4C59005873
:100690004F4E0048414C54002054533A0020543AE5
:1006A000003D0050696E3A004472697665722052CE
:1006B00065733A00416C72656164792048616C74BD
:1006C00065640A00416C726561647920496E6163FA
:1006D000746976650A00416C7265616479204163D2
:1006E000746976650A005475726E696E6720584F9A
:1006F0004E0A00584F464620736B69707065642E31
:10070000205072657620636D643A005475726E6590
:1007100064206F66662066726F6D3A00526573746E
:100720006F7265642066726F6D3A004E6F2073744D
:100730006F7265642076616C756573202D20646529
:100740006661756C743A200049676E6F7265642C3F
:10075000206368616E6E656C20636D643D00446962
:100760007361726D656400206D73203A0041726D93
:10077000656420666F7220004F75744F664D656D1D
:100780006F7279210A0020436D643A00205375622C
:100790003D00204974656D3D0052414D3D0020698A
:1007A0006E616374697665200020616374697665A3
:1007B00020002076616C7565206973200020756EBD
:1007C0006B6E6F776E0A00204772703A0020696E78
:1007D00076616C696400206F6B003A002066616985
:1007E0006C6564003A005265747279696E67206DB9
:1007F0006F6462757320434D440A00207365632063
:1008000072656D61696E696E6700537461747573AA
:100810002064656666657265640A002D3E00507549
:10082000623A2000636D6400434F4F4C00484541DD
:1008300054004155544F002D3E005075623A20003F
:100840007365740064656C002D3E005075623A203B
:10085000002D3E005075623A2000556E6B6E6F772A
:100860006E20636D64200A004F4646004F4E002004
:10087000002D3E00436F6E76657274696E672000CE
:100880002D3E0057726F6E672041737369676E6DFE
:10089000656E742000524742783A200020764C65FD
:1008A00076656C3A0020436F6E76563A0020436FAF
:1008B0006E76533A0020486F743A00436F6C643A86
:1008C0000020436F6E76657274656420563A00436B
:1008D0006F6E76657274656420533A002D3E005742
:1008E000726F6E672041737369676E6D656E7420F9
:1008F000002D3E0057726F6E672041737369676EFB
:100900006D656E7420004C6F6164656420466C6F89
:1009100061743A004C6F6164656420496E743A00FA
:100920004C6F61646564203A000000000000000024
:1009300000004F4E000000000000004F464600003F
:1009400000000000524553540000000000544F477F
:10095000474C4500000048414C540000000000583E
:100960004F4E000000000000584F464600000000B7
:1009700000494E4352454153450044454352454189
:10098000534500484541540000000000434F4F4C80
:1009900000000000004155544F0000000000464197
:1009A0004E5F4F4E4C590044525900000000000069
:1009B00053544F50000000000048494748000000D1
:1009C00000004D454449554D0000004C4F57000074
:1009D0000000000054525545000000000046414C04
:1009E000534500000000454E41424C454400004440
:1009F000495341424C454400524742000000000028
:100A00000048535600000000000020537566663A07
:100A1000002041543A00536B697070696E672E2E46
:100A2000004F75744F664D656D6F727921005D20C2
:100A3000000A5B003A004D41433A005544502053B0
:100A400079736C6F6720696E697469616C697A6526
:100A5000642E0A005379736C6F6720706172616D48
:100A6000733A0043757272656E74204C414E206378
:100A70006F6E6669672869702C646E732C67772CBB
:100A80007375626E6574293A000A5573652074683F
:100A900065736520636F6D6D616E64733A202768BE
:100AA000656C7027202D20746869732074657874D4
:100AB0000A276D61632064653A61643A62653A654C
:100AC000663A66653A3030272073657420616E643B
:100AD0002073746F7265204D41432D6164647265AB
:100AE000737320696E20454550524F4D0A27697037
:100AF000205B69705B2C646E735B2C67775B2C7377
:100B000075626E65745D5D5D5D27202D2073657473
:100B1000207374617469632049500A277361766594
:100B200027202D207361766520636F6E66696720CC
:100B3000696E204E5652414D0A2767657427205B27
:100B4000636F6E66696720616464725D27202D2083
:100B500067657420636F6E6669672066726F6D20CB
:100B60007072652D636F6E66696775726564205576
:100B7000524C20616E642073746F726520616464EE
:100B8000720A276C6F616427202D206C6F616420CE
:100B9000636F6E6669672066726F6D204E565241B4
:100BA0004D0A2770776427202D20646566696E657D
:100BB000204D5154542070617373776F72640A270B
:100BC0006B696C6C27202D207465737420776174B9
:100BD0006368646F670A27636C65617227202D2044
:100BE000636C65617220454550524F4D0A2772650E
:100BF000626F6F7427202D207265626F6F7420639F
:100C00006F6E74726F6C6C657200536F66742072D5
:100C100065626F6F74696E672E2E2E0052414D3DD6
:100C2000000A6D71747420000A696E707574732007
:100C3000000A6974656D7320000A436F6E66696708
:100C4000757265643A003B003D0050696E3A003BA6
:100C5000003D4C4F5700546865726D6F3A004C6F01
:100C600061646564006C6F6164206661696C6564D1
:100C7000004E6F2073746F72656420636F6E6669D7
:100C800067004C6F6164696E6720436F6E666967C9
:100C90002066726F6D20454550524F4D005361766E
:100CA000656420746F20454550524F4D0053617666
:100CB000696E6720636F6E66696720746F204545B3
:100CC00050524F4D2E2E0053617665640A005365D5
:100CD000742064796E616D69632049500A0045454E
:100CE00050524F4D20636C65617265640A0050611B
:100CF0007373776F726420757064617465640A0041
:100D0000636F756C64206E6F742070617273653AE6
:100D10002000557064617465640A002B002D004842
:100D20005454502F312E31202569002048545450FE
:100D30002F312E310D0A486F73743A2025730D0A36
:100D40004163636570743A202A2F2A0D0A436F6E3F
:100D50006E656374696F6E3A20636C6F73650D0A1C
:100D60000025730020000D0A0047455400666169A4
:100D70006C656420746F20636F6E6E6563740A0027
:100D80004552524F523A2053657276657220726511
:100D90007475726E65642000446F6E652E0A0041A2
:100DA00070706C79696E672E0A00436F6E666967B2
:100DB0002070617273696E67206661696C65640A90
:100DC00000676F7420436F6E6669670A007265740E
:100DD000636F6465200068636C69656E7400667299
:100DE00065652000436F6E666967205552493A2059
:100DF000687474703A2F2F002044656661756C74B6
:100E000020636F6E66696720736572766572207500
:100E10007365643A20006C617A79686F6D652E7233
:100E20007500205361766564000A282B294D444ED5
:100E300053000A282D2955415254425249444745EE
:100E4000000A282B295359534C4F47000A282D29B3
:100E5000504944000A282D294D4350323330313750
:100E6000000A282D294152544E4554000A282B29A6
:100E70004F5441000A282D29535049204C45440025
:100E80000A282D294D4F544F5220435452000A280E
:100E90002D294143204841494552000A282D294324
:100EA0004353383131202620484443313038300014
:100EB0000A282D29524553544152545F4C414E5FEC
:100EC0004F4E5F4D5154545F4552524F5253000A9A
:100ED000282D294841524452455345542C207573BE
:100EE000696E6720736F6674000A282D29434F5579
:100EF0004E544552000A282D29444854000A282DF2
:100F0000294F57495245000A282D294D4F44425533
:100F100053000A282D29444D58000A282B295769C7
:100F20007A6E657435783030000A282B29445332A4
:100F30003438322D313030000A282B29467265654D
:100F400052616D207072696E74696E670064653AF3
:100F500030313A32333A30303A30303A3031000AB8
:100F60004669726D77617265204D4143204164642A
:100F70007265737320006C617A79686F6D652E728B
:100F800075000A436F6E66696720736572766572D5
:100F90003A000A282B295741544348444F4700320E
:100FA00030313130334C0020432B2B207665727367
:100FB000696F6E3A00333265616361655F3230326A
:100FC000312D30362D3139000A4C617A79686F6DD8
:100FD000652E7275204C6967687448756220636F6E
:100FE0006E74726F6C6C65722000204F4646002054
:100FF0004F4E00757074696D650066726565686551
:10100000617000204C6F636B733A002000204C6FBE
:10101000636B733A000A52414D3D00204578706978
:101020007265640A00202D746172676574207A6F9E
:101030006E652D0020416C61726D2045787069727B
:1010400065640A0020636D643A00204375723A00BB
:10105000205365743A00206973200044656C657400
:10106000696E6720636F6E662E2052414D20776156
:10107000733A0053746F707065640053746F7070CE
:10108000696E67206368616E6E656C73202E2E2E0C
:10109000004E6F7420756E6C6F636B656420696EB3
:1010A00020313073202D20636F6E74696E7565205A
:1010B0002E2E2E00556E6C6F636B696E6720636F0A
:1010C0006E666967202E2E2E0044656661756C740D
:1010D0002073657269616C206D6F6465204E3831D4
:1010E000207573656400384531002600384E3100A4
:1010F0000600384532002E00384E32000E00384FC0
:1011000031003600384F32003E00374531002400B0
:10111000374532002C00374F31003400374F320052
:101120003C00374E31000400374E32000C00203DA9
:101130003E002C002C002C002C00456C6576617460
:101140006F723A20636F6E666967206661696C65CD
:10115000643A00456C657661746F7220636F6E66E9
:101160006967206572726F7200456C657661746F95
:101170007220636F6E666967206C6F6164656420BE
:1011800000456C657661746F723A204F7574206FFC
:1011900066206D656D6F7279003C003E00556E6B88
:1011A0006E6F776E207375666669782000556E6B7A
:1011B0006E6F776E20636D642000536574206E6FD0
:1011C0007420696D706C656D656E74656400466F42
:1011D0007263656420657865637574696F6E004D30
:1011E000756C746956656E7420636F6E66696720EE
:1011F0006661696C6564004D756C746956656E74E2
:1012000020696E6974004D756C746976656E742022
:1012100044652D496E697400204F75743A00206D45
:1012200033002066726F6D2000204D61782072655A
:1012300071756573743A002066616E253A0020610D
:10124000637469766520563A00546F74616C205659
:101250003A0050574D2D4F757420496E69740050F7
:10126000574D2D4F75742073746F70005247422094
:1012700050574D002050574D00524742572050576D
:101280004D003D0050696E3A005B305D3A20002011
:101290002D202D202D20EFBBBF003E003E31202D04
:1012A00020002C20002E00696E00735F6F757400A3
:1012B0006D79686F6D6500202D3E2000202D3E2049
:1012C00000202D3E20003E3E2000496E76616C6974
:1012D0006420636F6D6D616E64003E3E3E004E6F34
:1012E000204D414320636F6E666967757265643A8D
:1012F00020736574206669726D776172652773204B
:101300004D41430A00476F74204950206164647264
:101310006573733A00276970205B69705B2C646E9B
:10132000735B2C67775B2C7375626E65745D5D5DB6
:101330005D27202D207365742073746174696320A8
:1013400049500A004661696C656420746F20636FC0
:101350006E6669677572652045746865726E65743E
:10136000207573696E6720444843502E20596F756D
:101370002063616E20736574206970206D616E75E5
:10138000616C6C7921000A75736573204448435081
:101390000A00204D41534B3A002047573A00204461
:1013A0004E533A004C6F616465642066726F6D2025
:1013B000666C6173682049503A00537461727469B5
:1013C0006E67206C616E004F544120696E697469CC
:1013D000616C697A65640A00757074696D652C6664
:1013E000726565686561700024737461747300339D
:1013F0003265616361655F323032312D30362D31B7
:1014000039004C696768744875622000246E616D0C
:10141000650072656164790020747279206167618A
:10142000696E20696E2035207365636F6E6473008A
:101430006661696C65642C2072633D004177616967
:1014400074696E6720666F722072657461696E657B
:101450006420746F7069637300636F6E6E6563748C
:1014600065642061732000202E2E2E002075736588
:10147000723A003A000A417474656D7074696E675F
:10148000204D51545420636F6E6E656374696F6EA6
:1014900020746F2000247374617465006469736341
:1014A0006F6E6E6563746564005573696E67204D79
:1014B0005154542070617373776F72642066726F39
:1014C0006D20636F6E6669670044657669636520A9
:1014D0004E616D653A00526562696E642073756392
:1014E000636573732E204950206164647265737361
:1014F0003A004572726F723A20726562696E6420BA
:101500006661696C0052656E65776564207375630A
:10151000636573732E204950206164647265737330
:101520003A004572726F723A2072656E6577656433
:10153000206661696C000A4E6F206C696E6B004119
:101540006363657074696E6720636F6D6D616E644F
:10155000732E2E2E0A0000002100240027002A00EE
:101560002D003000330001010000040107010A01D1
:1015700000002200250028002B002E00310034003E
:1015800002010000050108010B010505050507051D
:1015900008080808020202020A0A080804040404EF
:1015A000010101010101010103030303030303031B
:1015B000040707070C0C0C0C0C0C0C0C02020202AA
:1015C00006060606060606060B0B0B0B0B0B0B0B93
:1015D000050505080807070404040A0A0A0A0A0A96
:1015E0000102102020080810204010204080020135
:1015F000020108040201010204081020408080401A
:101600002010080402018004020180402010080418
:1016100002010804020101020408102040800102B6
:1016200004081020408004408004800810102040EE
:1016300004081020408000000B0C030A0D0E0F0957
:101640000804050200000000000000000000000087
:10165000000000000000000000000000000000008A
:101660000000131211000000000000000000000044
:10167000000000000000000000000000000000006A
:1016800000000000000000000000000053617665CB
:10169000643A0000D8A9AFA911241FBECFEFD1E250
:1016A000DEBFCDBF00E00CBF18E0A0E0B2E0EAE38F
:1016B000FEE701E00BBF02C007900D92A031B10719
:1016C000D9F72FE0A0E1B8E001C01D92AB31B2071D
:1016D000E1F71BE0CBE4DBE000E006C02197010965
:1016E000802FFE010E94DBB9CA34D10780E00807D1
:1016F000A9F70E94BC920C940BBF0C940000CF93EE
:10170000DF931F92CDB7DEB76983DC01ED91FC91C9
:101710000280F381E02D41E050E0BE016F5F7F4F1A
:1017200019950F90DF91CF910895FC01818D928DD5
:101730000895CF93DF931F92CDB7DEB76983DC01A5
:10174000ED91FC910280F381E02D41E050E0BE017B
:101750006F5F7F4F19950F90DF91CF910895FC0136
:101760009485FB018485981303C081E0983008F0CC
:1017700080E00895CF93DF931F92CDB7DEB76983E2
:10178000DC01ED91FC910280F381E02D41E050E01D
:10179000BE016F5F7F4F19950F90DF91CF91089534
:1017A00085ED8093BC008091BC0084FDFCCF10923D
:1017B0005409089520913009260F3327331F213211
:1017C0003105ECF420915409FC0190E080E02430D4
:1017D00069F082E00895A09130092191AC01405F49
:1017E000564FA40FB52FB11D2C930196861798F371
:1017F00080913009680F6093300980E0089581E09E
:1018000008958FEF9FEF08958FEF9FEF08958091D8
:101810000F0990E09195819591090895CF93DF93F9
:10182000CB01EA01642F0E94DA0BCE01DF91CF9148
:101830000895CF93DF931F92CDB7DEB7698361E040
:10184000CE0101960E94DA0B81E090E00F90DF91CB
:10185000CF9108958F929F92AF92BF92CF92DF92D5
:10186000EF92FF920F931F93CF93DF9300D000D09E
:1018700000D01F921F92CDB7DEB77C018E010F5FA3
:101880001F4F68018AE0882E912CA12CB12CC60133
:10189000801B910B411551056105710581F0CB014C
:1018A000BA01A50194010E9450B9942F852F605D63
:1018B000F60161936F01A901692F782FE8CFF80134
:1018C000E80FF91FD7010150110922912D93E0175C
:1018D000F107D9F7E80EF91EF70110822B960FB623
:1018E000F894DEBF0FBECDBFDF91CF911F910F9156
:1018F000FF90EF90DF90CF90BF90AF909F908F9030
:101900000895FC01DC018D918111FDCF30E020E0D4
:1019100050E040E08AE09191992301F14430510573
:101920005CF59E3271F42F3F310509F02CF5DB0197
:10193000A40FB51F12962C934F5F5F4F30E020E04D
:10194000EACF829FD001839FB00D1124292F990FD8
:10195000330B205331092A0F3B1FDDCF2F3F3105B9
:1019600009F054F4443051053CF4640F751FFB0139
:10197000228381E090E0089590E080E00895CF9385
:10198000DF931F921F92CDB7DEB780910F0F90911A
:10199000100F009711F48BE19FE0BE016F5F7F4F46
:1019A000681B790B072E000C880B990B0F900F907A
:1019B000DF91CF910895DC0116968D919C9100974F
:1019C00039F0DC01ED91FC910680F781E02D19944E
:1019D0000895089590E080E008958091B70890916F
:1019E000B8080895089583E090E008958091B508BF
:1019F0009091B608089584E090E00895DC01149673
:101A0000ED91FC91309729F08081082E000C990B04
:101A1000089590E080E0089581E090E00895FC0151
:101A2000848195810895FC01768765870895DC019E
:101A3000ED91FC91068CF78DE02D199591E08927A9
:101A40000895862F089581E08627089521E0FC01FE
:101A50008485883008F020E0822F0895FC01848579
:101A600095850895FC018489958908952BE933E0D3
:101A7000FC0131832083FB0140895189628973898C
:101A8000FC0142835383648375830895DC01ED91E7
:101A9000FC91048CF58DE02D199490E080E0089580
:101AA000CF93DF9300D000D01F921F92CDB7DEB747
:101AB000FC01862F8F706281607F682B628388E0D3
:101AC000DE01119601900D928A95E1F729813A8104
:101AD0004B815C816D817E818F81988528960FB6C0
:101AE000F894DEBF0FBECDBFDF91CF910895CF93A5
:101AF000DF9300D000D01F921F92CDB7DEB7FC015C
:101B0000608398E0DE01119601900D929A95E1F7BD
:101B100029813A814B815C816D817E818F8198859D
:101B200028960FB6F894DEBF0FBECDBFDF91CF91E0
:101B30000895CF93DF9300D000D01F921F92CDB7AE
:101B4000DEB7FC016F3F710519F014F06FEF70E024
:101B500077FD60E09281892F82958F70815082306D
:101B6000C8F4648388E0DE01119601900D928A9595
:101B7000E1F729813A814B815C816D817E818F8182
:101B8000988528960FB6F894DEBF0FBECDBFDF91C3
:101B9000CF9108959F7090619283E3CF0F931F932D
:101BA000CF93DF93FC01C62F928192959F70963060
:101BB00009F486C030F49150923040F16FEF7FEF1E
:101BC0001FC0973071F19A509230C0F7848195818F
:101BD000A681B7818F3F9105A105B10529F024F0B9
:101BE0008FEF90E0A0E0B0E0B7FF03C080E090E0AE
:101BF000DC016FEF70E0681B790BC11101C0BC0103
:101C0000CB01DF91CF911F910F910895648170E016
:101C1000CC23B1F38FEF90E09C01261B370BB90169
:101C2000EFCF862F04811581D681C78120E030E077
:101C3000A901B801882331F18D2F9C2F0E9406B88D
:101C400087FD1BC020E030E04FE753E4B8018D2F43
:101C50009C2F0E940EBB181624F400E010E0DFE772
:101C6000C3E498014D2F5C2F60E070E08FE793E4B0
:101C70000E94F9B90E94D8BAC3CF00E010E0D0E0CA
:101C8000C0E0EFCF8D2F9C2F0E9406B887FD13C0B8
:101C900020E030E04FE753E4B8018D2F9C2F0E94E5
:101CA0000EBB181624F400E010E0DFE7C3E4B8012F
:101CB0008D2F9C2FDFCF00E010E0D0E0C0E0F7CF09
:101CC00064817581868197812AE030E040E050E0B0
:101CD0000E9472B92F3F31054105510529F024F0CA
:101CE0002FEF30E040E050E057FF03C020E030E04D
:101CF000A9016FEF70E0621B730BC11181CF8FCF11
:101D0000DC011296EC911297E295EF70E150EB3006
:101D100008F039C0F0E08827EF56F14F8F4F0C9450
:101D2000DBB9B40EB40EC30E9C0E9C0EA50EBC0EF9
:101D3000BC0EBC0E9C0E9C0E14966D917D918D91E7
:101D40009C9117970E940DB8089514966D917D91FE
:101D50008D919C9117972AE030E040E050E00E947E
:101D600072B9CA01B901EECF14966C9170E090E09F
:101D700080E00E940BB8089514966D917D918D912D
:101D80009C911797089560E070E0CB010895DC0105
:101D90001296EC911297E295EF70E150EB3008F05B
:101DA00037C0F0E08827E852F14F8F4F0C94DBB931
:101DB000EA0EEA0E080FE30EE30EF90EF00EF00E37
:101DC000F00EE30EE30E14966D917D918D919C9132
:101DD0001797089514966C9170E090E080E0089554
:101DE00014966D917D918D919C9117970E94D8BA10
:101DF000089514966D917D918D919C9117972AE08D
:101E000030E040E050E00E9472B9CA01B901089583
:101E100060E070E0CB010895FC01A7812A2F2E7F9E
:101E2000D1F0828182958F7081508330A0F4A69585
:101E3000A150BB0B2BE531E00E94F2B924E630E063
:101E400040E050E00E9472B9DA01C90187569F4F05
:101E5000AF4FBF4F08958FEF9FEF0895CF93DF935C
:101E6000EC018A81982F92959F7041F180E0943027
:101E700010F59B01770F440B550B29593109410986
:101E80005109A4E6B0E00E9491B92BE531E040E0B1
:101E900050E00E9472B937FF02C030E020E02536E2
:101EA000310514F024E630E02F5F220F8F8181701E
:101EB000282B2F8381E0DF91CF9108958F7080626E
:101EC0008A83D7CFFC019281892F82958F7021F070
:101ED000823029F080E008959F70906292839B0188
:101EE00077FF02C030E020E02E3681E0380714F0A2
:101EF0002DE631E02683878130FB80F9878381E0FE
:101F00000895DC0119968D919C91009739F0DC01C0
:101F1000ED91FC910280F381E02D199408958AE0FF
:101F200090E00895CF93DF93EC01E881F981048478
:101F3000F585E02D19952E853F852F5F3F4F3F8713
:101F40002E87DF91CF910895FC0122813381232BCD
:101F500049F0868197818130910539F01CF0039713
:101F6000029730F090E080E0089581E090E00895DD
:101F700082E090E00895CF93DF93CDB7DEB760970E
:101F80000FB6F894DEBF0FBECDBF19821A821B8236
:101F90001C821D821E821F8218868B818F708B830C
:101FA0006FEF70E0CE0101960E94990D60960FB61A
:101FB000F894DEBF0FBECDBFDF91CF910895CF92D1
:101FC000DF92EF92FF920F931F93CF93DF93CDB7E2
:101FD000DEB760970FB6F894DEBF0FBECDBF7C01B1
:101FE0006B01BA01A901CE0101960E942A0CD7010A
:101FF000ED91FC910288F389E02D9801AE014F5FCD
:102000005F4FB601C701199560960FB6F894DEBF11
:102010000FBECDBFDF91CF911F910F91FF90EF9039
:10202000DF90CF900895CF92DF92EF92FF920F93BF
:102030001F93CF93DF9300D000D0CDB7DEB78C01D4
:102040006B017A01FC01808D883010F40E94D476F7
:102050008BE993E09A838983F60182819381A4813D
:10206000B5818B839C83AD83BE83B701CE0101967E
:102070000E94F981F801808F8830A0F4F586E4860B
:10208000128E118E81E026960FB6F894DEBF0FBE39
:10209000CDBFDF91CF911F910F91FF90EF90DF9017
:1020A000CF90089580E0EFCFCF93DF93EC01888D40
:1020B000883020F40E94D47688E0888FDF91CF9119
:1020C0000895FC01808D883040F4218D328D232BC2
:1020D00021F00E94A67590E008958FEF9FEF08957C
:1020E000CF93DF93FC012485283028F08FEF9FEFFA
:1020F000DF91CF910895EC010190F081E02D0084F3
:10210000F185E02D1995892B89F38C850E94A675A0
:1021100090E0EECFCF93DF93FC01218D328D21151E
:10212000310529F48FEF9FEFDF91CF910895EC01F6
:10213000808D4217530708F0A9010E94F575181603
:10214000190684F7298D3A8D281B390B3A8F298F70
:10215000EBCF0F931F93CF93DF931F92CDB7DEB7D3
:10216000FC01218D328D232B41F48FEF9FEF0F90D7
:10217000DF91CF911F910F9108958C0141E050E0C4
:10218000BE016F5F7F4FFC01808D0E94F5751816B0
:1021900019065CF7F801818D928D0197928F818FDE
:1021A000898190E0E4CFCF93DF931F92CDB7DEB764
:1021B00041E050E0BE016F5F7F4FFC0184850E94CB
:1021C000F5751816190634F4898190E00F90DF91A7
:1021D000CF9108958FEF9FEFF9CFFC018485883070
:1021E00010F40C94F57590E080E00895FC0184856E
:1021F000883010F40C94CE7590E080E008950F9331
:102200001F93CF93DF9300D000D01F921F92CDB7C2
:10221000DEB78C01D80159964D915C915A974115C2
:10222000510551F0ED91FC91048CF58DE02D70E09D
:1022300060E0C8011995EECFF801808D0E94CE753F
:10224000892BB1F148E050E0BE016F5F7F4FD801AC
:1022500058968C910E94F57518161906F4F4D80159
:10226000509684E0FE01319601900D928A95E1F737
:102270008D8190E0982F88272E81820F911DF80183
:10228000958B848B8F81282F30E0322F22278885F1
:10229000820F932F911D928F818F28960FB6F894FD
:1022A000DEBF0FBECDBFDF91CF911F910F9108957B
:1022B00090E080E0F2CFCF92DF92EF92FF920F9307
:1022C0001F93CF93DF93CDB7DEB7AF970FB6F894D8
:1022D000DEBF0FBECDBF7C016A010BE913E01A839C
:1022E00009831C861B8688EE93E0A0E0B0E08D8712
:1022F0009E87AF87B88B83E393E09A878987188F8F
:102300000F8B198E1A8E1B8E1C8E88E089A31BA73B
:102310000AA71CA61DA61EA61FA68091360C90918A
:10232000370CA091380CB091390C8EA39FA3A8A7AD
:10233000B9A78B839C83AD83BE8318861F82AE01B1
:10234000465D5F4FCE0101960E948F8881309105D6
:10235000B1F4D701ED91FC910488F589E02D1DA31E
:102360000CA38CA59DA5AEA5BFA58EA39FA3A8A7D2
:10237000B9A7A601BE016C5D7F4FC7011995AF9645
:102380000FB6F894DEBF0FBECDBFDF91CF911F9186
:102390000F91FF90EF90DF90CF9008950F931F93D0
:1023A000CF93DF93EC018B01888D883010F40E946D
:1023B000D476B80182E00E941D77888F883050F46F
:1023C0001D870C871A8E198E81E0DF91CF911F91A6
:1023D0000F91089580E0F9CF0F931F93CF93DF9370
:1023E0008C01EA01FC018485883048F40E94447520
:1023F000892B39F481E090E0F80193838283D0E067
:10240000C0E0CE01DF91CF911F910F910895EF921F
:10241000FF920F931F93CF93DF937C018091C20AA9
:10242000D4E0833309F0D8E002EB1AE0C0E0F80111
:10243000219131918F01F701848195812817390706
:1024400029F0CF5FDC13F3CF80E006C08C2F0E9411
:10245000E2768431B1F781E0DF91CF911F910F9146
:10246000FF90EF900895CF93DF93EC018C85883037
:10247000D0F40E94E276843189F0882379F08831A3
:1024800069F021E08C3159F4E881F9810084F1850B
:10249000E02DCE01199521E0892B09F420E0822F4F
:1024A000DF91CF91089580E0FBCFCF92DF92EF9242
:1024B000FF920F931F93CF93DF93CDB7DEB7AF9704
:1024C0000FB6F894DEBF0FBECDBF8C016B017A0151
:1024D0008BE993E09A8389831B821C821D821E8272
:1024E0001C861B8648EE53E060E070E04D875E87F7
:1024F0006F87788B23E333E03A872987988F8F8B18
:10250000198E1A8E1B8E1C8E28E029A39BA78AA7E2
:102510001CA61DA61EA61FA6D8011C968C9188304D
:1025200060F40E94E276882321F0F80184850E94FD
:10253000C67688E0D8011C968C938091360C9091D9
:10254000370CA091380CB091390C8EA39FA3A8A78B
:10255000B9A78B839C83AD83BE8318861F82AE018F
:10256000465D5F4FB601CE0101960E948F880097AD
:10257000C1F0D801ED91FC910684F785E02D8BE93F
:1025800093E09DA38CA38CA59DA5AEA5BFA58EA30E
:102590009FA3A8A7B9A7A701BE016C5D7F4FC80183
:1025A0001995AF960FB6F894DEBF0FBECDBFDF9181
:1025B000CF911F910F91FF90EF90DF90CF900895F2
:1025C000CF93DF93EC018C85883060F40E94E27633
:1025D000873111F08C3131F48C850E94277581157B
:1025E000984088F3DF91CF910895FC01848588306D
:1025F00010F40C94277590E080E0089566E072E195
:102600008FE19DE00E94B0698FE19DE00E94A76884
:102610001092B6081092B50881E090E008956BE141
:102620007DE0811102C06DE17DE08CE69CE00C94C0
:10263000B0696EEE7CE08CE69CE00C94B0696EEDC7
:102640007CE08CE69CE00C94B0690F931F93CF93D1
:10265000DF9300D000D0CDB7DEB78B012BE933E09C
:102660003A8329831B821C821D821E82853091053C
:102670008CF1BE016F5F7F4FF801808591850E94CC
:10268000810CBE016F5F7F4FF801868197810E94A8
:10269000810CBE016F5F7F4FF801848195810E949C
:1026A000810CBE016F5F7F4FF801828193810E9490
:1026B000810C67EC7CE08CE69CE00E94B069269679
:1026C0000FB6F894DEBF0FBECDBFDF91CF911F9143
:1026D0000F91089584309105A1F283309105C9F2DC
:1026E00082309105F1F2019721F76EEC7CE08CE6E7
:1026F0009CE00E94B069DDCF6AE07CE08CE69CE063
:102700000E94B069F0E0E0E0199469EA77E0811195
:1027100002C06EE977E08FE19DE00C94B069EF9222
:10272000FF920F931F93CF93DF93EC01A881B981A0
:10273000109761F18C91882349F108811981F80182
:102740008081882351F08D3241F080538A3028F007
:102750000F5F1F4F19830883F0CFC8010E9458B044
:102760007C016CE270E0C8010E9429BE009751F420
:1027700019821882C701DF91CF911F910F91FF90AD
:10278000EF900895019699838883F4CFF12CE12C82
:10279000F1CF4F925F926F927F92AF92BF92DF9292
:1027A000EF92FF920F931F93CF93DF9300D000D04F
:1027B000CDB7DEB77C01D62E80910B09882309F4B2
:1027C000B5C08091090990910A092AE06213E7C017
:1027D0008754974FDC011C92F70100851185011584
:1027E000110509F49FC0D80119966D917C911A9733
:1027F00061157105A1F415964D905D906D907C90DA
:1028000018978091300C9091310CA091320CB091BE
:10281000330C481659066A067B0609F483C0F80192
:10282000438554854115510509F47CC0D7011496A0
:10283000AD90BC90838990E095012770332702C04A
:10284000959587952A95E2F780FF6CC0C501887F32
:102850009370892B31F481899289887F9370A82A9B
:10286000B92AF80180819181DC01ED91FC9161151B
:10287000710509F47EC00688F789E02D1995019746
:1028800009F050C06CE3F801808191810E94BD681D
:10289000A50170E060E02AE0D8018D919C910E9432
:1028A0005B68F8012281808191816CE972E12223C9
:1028B00011F06AE972E10E94B069D8011D966D912C
:1028C0007C911E978D919C910E944A6960E2F8016B
:1028D000808191810E94BD68D8011F966D917C9185
:1028E00050978D919C910E944A69F80122818081C4
:1028F00091816FE872E1222311F069E872E10E9490
:10290000B06969EB78E0D8018D919C910E944A6989
:10291000F80180819181DC01ED91FC91008CF18DB9
:10292000E02D199510920A0910920909D7011696FF
:102930008D919C91009709F444C0DC01ED91FC91CC
:102940000190F081E02D6D2D199526960FB6F89423
:10295000DEBF0FBECDBFDF91CF911F910F91FF90D2
:10296000EF90DF90BF90AF907F906F905F904F900F
:1029700008950488F589E02D2BE933E03A83298313
:10298000D80115964D905D906D907C9018974B8274
:102990005C826D827E82BE016F5F7F4F6FCF8F340E
:1029A000910524F6BDE06B1709F29C012F5F3F4FA4
:1029B00030930A09209309098754974FFC016083DB
:1029C000B5CF81E090E0C1CFCF93DF93EC01888950
:1029D00099892A893B89680F791F820F931F68178D
:1029E000790708F4CB019F878E8768EC75E08FE14B
:1029F0009DE00E94B0694E855F8570E060E02AE04E
:102A00008FE19DE00E945B688FE19DE00E94A768D6
:102A10008E859F85DF91CF9108950C9428AE0C94FC
:102A200028AE0C9428AECF93DF93DC011296ED9183
:102A3000FC913097C1F1EC018E819F81833091052B
:102A4000B1F0049719F160858FE19DE00E94DB7D74
:102A500064E772E18FE19DE00E94B0698FE19DE043
:102A60000E94A768EA81FB81808590E00CC06CE63B
:102A700072E18FE19DE00E94B0698FE19DE00E94CC
:102A8000A76882E090E0DF91CF91089569E772E155
:102A90008FE19DE00E94B0698FE19DE00E94A768F0
:102AA00081E090E0F0CF90E080E0EDCFCF93C1E007
:102AB00068EE73E080E090E00E94CA846C2F8CE6A0
:102AC0009CE00E94DB7DCF5FC43191F7CF910895E8
:102AD000CF93DF93EC01FB0124813581408151814B
:102AE000628173810E94C468CE01DF91CF91089505
:102AF000EF92FF920F931F93CF93DF93EC018B0123
:102B00001D821C821A821B82E880F980E114F10484
:102B100009F459C08091230890912408892B09F465
:102B200052C0672B09F48701F80180858F708630C9
:102B3000A9F46DEB73E0C8010E94667D009719F05F
:102B4000FC0181858A836FE576E0C8010E94667D7D
:102B5000009709F43FC0FC0181858B836FEB73E024
:102B6000C7010E94667D009759F560ED75E08FE121
:102B70009DE00E94B0696B818FE19DE00E94DB7D4A
:102B80006EEC75E08FE19DE00E94B0696A818FE193
:102B90009DE00E94DB7D8FE19DE00E94A76820E020
:102BA00030E0A9016FEB73E0888199810E949A7EE1
:102BB0006FEB73E0888199810E94667D009719F020
:102BC00009969D838C83DF91CF911F910F91FF9088
:102BD000EF900895F801808191810E9458B0BDCF97
:102BE000CF93DF93009709F484C0FC012081222356
:102BF00009F47FC0EC0160E478E00E94A6B0892B64
:102C000009F456C064E278E0CE010E94A6B0892B98
:102C100009F451C062E476E0CE010E94A6B0892B8F
:102C200009F44CC06EE376E0CE010E94A6B0892B79
:102C300009F447C06AE376E0CE010E94A6B0892B72
:102C400009F442C066E376E0CE010E94A6B0892B6B
:102C5000F1F162E376E0CE010E94A6B0892BD1F1BA
:102C60006EE276E0CE010E94A6B0892BB1F169E256
:102C700076E0CE010E94A6B0892B91F165E276E064
:102C8000CE010E94A6B0892B71F164E478E0CE01F8
:102C90000E94A6B0892B51F161E276E0CE010E943C
:102CA000A6B0892B31F58EE090E0DF91CF910895A9
:102CB00082E090E0FACF81E090E0F7CF88E090E00A
:102CC000F4CF85E090E0F1CF86E090E0EECF87E0B2
:102CD00090E0EBCF89E090E0E8CF8AE090E0E5CFAC
:102CE0008BE090E0E2CF8CE090E0DFCF8DE090E0F1
:102CF000DCCF90E080E0D9CFFC01868197810097FE
:102D000099F0FC0120852F70223029F461857285AD
:102D1000838594850895253039F460E00E94E27D32
:102D2000009711F0FC01F2CF60E070E0CB01089554
:102D30000F931F93CF93DF93FC01C281D381209720
:102D4000F9F088858F70823049F4672BC9F4898542
:102D50009A85DF91CF911F910F910895853081F46D
:102D60008B01CE010E94427E8017110649F044F08B
:102D7000602FCE010E94E27DFC0181859285E9CF22
:102D800090E080E0E6CFFC016115710519F48481C3
:102D90009581089586819781681779072CF0848141
:102DA0009581860F971F0895828193810C949816C0
:102DB000CF93DF93EC016FE572E18FE19DE00E941C
:102DC000B0698FE19DE00E94A768E881F981028CDB
:102DD000F38DE02DCE0119958130910529F00297F0
:102DE00059F060E08C811AC063E070E0CE010E946F
:102DF000C31660E00E94728360E08C810E9472833F
:102E000061E070E0CE010E94C31660E00E94728310
:102E100062E070E0CE010E94C31660E00E947283FF
:102E20001092B8081092B70881E090E0DF91CF913E
:102E300008950F931F93CF93DF93EB0163E0FC01A1
:102E4000808191810E94E27D009731F1AE01409531
:102E500050954F6F70E060E0FC010185128523857D
:102E6000348540235123622373234187528763872C
:102E7000748768E576E08FE19DE00E94B069BE014D
:102E80008FE19DE00E94EF7D8FE19DE0DF91CF918A
:102E90001F910F910C94A768DF91CF911F910F9113
:102EA00008950F931F93CF93DF93EB0163E0FC0131
:102EB000808191810E94E27D009721F18E0100279F
:102EC00030E020E0FC014185528563857485402B0C
:102ED000512B622B732B41875287638774876FE472
:102EE00076E08FE19DE00E94B069BE018FE19DE038
:102EF0000E94EF7D8FE19DE0DF91CF911F910F91B7
:102F00000C94A768DF91CF911F910F910895CF93F3
:102F1000DF93EB0163E0FC01808191810E94E27DFF
:102F2000009741F0FC01818592858C239D23DF91E0
:102F3000CF91089590E080E0FACFCF93C62F63E061
:102F4000FC01808191810E94E27D0097E9F0FC0103
:102F500041855285638574854427662777274C2BE6
:102F6000418752876387748767E476E08FE19DE04D
:102F70000E94B0696C2F8FE19DE00E94DB7D8FE1A4
:102F80009DE0CF910C94A768CF910895FC018281B8
:102F90009381009719F062E00E949D170895CF93E6
:102FA000DF93EC010E94C61762E572E18FE19DE0BC
:102FB0000E94B0698FE19DE00E94A7688A819B8191
:102FC000892B09F44DC08C819D81892B09F048C063
:102FD000E881F981028CF38DE02DCE0119958130C5
:102FE000910529F0029759F061E08C811AC063E0E5
:102FF00070E0CE010E94C31661E00E94728361E01E
:103000008C810E94728361E070E0CE010E94C31641
:1030100061E00E94728362E070E0CE010E94C316FC
:1030200061E00E9472838091A100887F8093A1005B
:1030300080919100887F809391008091A1008260AF
:103040008093A1008091910082608093910081E043
:1030500090E09093B8088093B708DF91CF910895DE
:1030600090E080E0FACFCF93DF93EC010E94C61787
:10307000EC81FD81309709F44FC0C681D78120973C
:10308000C1F1E881F981309781F18081882369F16C
:1030900062EC73E0CE010E94667D892B41F42FEF34
:1030A0003FEFA90162EC73E0CE010E949A7E65E7D2
:1030B00074E0CE010E94667D892B41F42FEF3FEF33
:1030C000A90165E774E0CE010E949A7E66EC73E088
:1030D000CE010E94667D892B41F42FEF3FEFA901BD
:1030E00066EC73E0CE010E949A7E0A80DB81C02DDF
:1030F000C6CF67EF71E18FE19DE00E94B0698FE17B
:103100009DE00E94A76881E090E09093B6088093CC
:10311000B508DF91CF9108956FED71E18FE19DE0EA
:103120000E94B0698FE19DE00E94A76890E080E076
:10313000F0CF63E0FC01808191810E94E27D0097E5
:1031400019F0FC01818508958FEF08950F931F9367
:10315000CF93DF93C92FD62F082F192F17FF03C046
:1031600011950195110961E0802F0E9472836C2FE7
:10317000DD23A9F06095661F6627661F802F0E94D9
:1031800044836FEE7FE08FE19DE00E94B0698FE1A4
:103190009DE0DF91CF911F910F910C94A768661F5E
:1031A0006627661F802F0E9444836AEE7FE0EBCF84
:1031B0001F93CF93DF93162FFC01C685D7859E0101
:1031C0002F5F3F4F37872687CE010E942AB91817F5
:1031D00021F0612FCE010E9432B981E090E0DF91B1
:1031E000CF911F910895CF93DF9300D000D01F920D
:1031F0001F92CDB7DEB770E060E086ED9DE00E94E3
:10320000E4141C821B828EEA92E09A83898386ED05
:103210009DE09E838D838FEF9FEF98878F836DEA6C
:103220007CE08CE69CE00E94B0696091230870917C
:103230002408CE0101960E94106F6FEF86ED9DE08D
:103240000E94D8186DE97CE08CE69CE00E94B06991
:103250008CE69CE00E94A76828960FB6F894DEBF23
:103260000FBECDBFDF91CF910895FC018685978574
:103270000E942AB990E008952F923F924F925F9258
:103280006F927F928F929F92AF92BF92CF92DF9276
:10329000EF92FF920F93CF93DF9300D01F92CDB7A1
:1032A000DEB77C017A8369835C834B83DB011C92EC
:1032B000FC016081662309F4C2C130FFC0C1F9E09E
:1032C0006F9FB0011124675D764FCD010E94DDB084
:1032D0004B815C816FEC76E089819A810E9444BECB
:1032E000E981FA8101900020E9F7319789819A817B
:1032F000E81BF90B1C012E0E3F1EAB81BC81AE1BDF
:10330000BF0B1197BC83AB83D7011296EC91E2956A
:10331000EF70E150EC3008F0B3C0F0E08827EC56D5
:10332000F64E8F4F0C94DBB9A0190F1A751ADC1AE0
:10333000F81ADC198C1A8C1A8C1AD019C419151B9E
:10334000F7018481282F30E050E040E0002359F05D
:1033500030E0A4E6B0E00E94A4B92FEF30E040E0F6
:1033600050E00E9472B95F934F933F932F938AEC82
:1033700093E09F938F93FC81FF938B818F933F9278
:103380002F920E947CBE77C0F70187818F93868140
:103390008F9385818F9384818F938DEC93E0E9CF18
:1033A000F70187818F9386818F9385818F938481A5
:1033B0008F9381ED93E0DDCFF701C480D580E68067
:1033C000F780C701B6012AE030E040E050E00E94FB
:1033D00072B997FF07C090958095709561957F4F62
:1033E0008F4F9F4F9F938F937F936F93C701B6012A
:1033F0002AE030E040E050E00E9472B95F934F93C2
:103400003F932F9385ED93E09F938F93FC81FF93E0
:103410008B818F933F922F920E947CBE2CC0C7015C
:103420000E940C0FBC01F701C680D780D0FADD24C2
:10343000D0F89481F580EB80BC80292F30E050E0FB
:1034400040E077FD35C0011135C07F936F931F9227
:103450001F921F929F931F92FF92DF92CF928CED4B
:1034600093E09F938F939C819F93AB81AF933F9207
:103470002F920E947CBE0FB6F894DEBF0FBECDBF68
:1034800089819A810F900F900F900F90DF91CF91CB
:103490000F91FF90EF90DF90CF90BF90AF909F90F3
:1034A0008F907F906F905F904F903F902F900895F6
:1034B000002361F0292F30E0A4E6B0E00E94A4B917
:1034C0002FEF30E040E050E00E9472B95F934F93DD
:1034D0003F932F931F92FF92DF92CF928FED93E055
:1034E0009F938F93BF92EF9295CFD70115968C91B2
:1034F00015971F928F9316969C91169717968C91FD
:1035000081708F939F9382EE93E09F938F93BC8102
:10351000BF93EB81EF9333CFD70114968D909D909D
:10352000AD90BC90179720E030E0A901C501B4012F
:103530000E9406B82401350187FF04C077FA709411
:1035400077F87094C301B2010E94D8BA6B01072EBC
:10355000000C880B990B0E940DB89B01AC01C301B4
:10356000B2010E94F9B920E030E048EC52E40E9438
:103570006CB80E9463BB0E94D8BA062F772E20E059
:1035800030E0A901C501B4010E9406B887FF07C059
:103590007F920F93DF92CF9288EE93E0B6CF7F9227
:1035A0000F93DF92CF9289EE93E09F938F939C814C
:1035B0009F93AB81AF93E3CED70114968C91149770
:1035C0001F928F9315968C9115971F928F93169635
:1035D0008C911F928F938FED93E09F938F93BC817B
:1035E000BF93EB81EF933F922F920E947CBE43CF1B
:1035F000D70117968C9117971F928F9314968C91E1
:1036000014971F928F9315968C9115971F928F93F5
:1036100016968C911F928F938CED93E09F938F93CE
:10362000BC81BF93EB81EF93F5CED70114966D91DA
:103630007C914B815C81C1010E9462BE21CF2980B7
:103640003A8062CEDF92EF92FF920F931F93CF9357
:10365000DF93EC01888199810E94427E082F10E05F
:1036600004301105ACF40E941571FC01892B41F066
:103670008085807F826080871186128613861486FB
:10368000BF01888199810E947E7E0F5F1F4FE8CF26
:10369000E880F98060E0C7010E94E27DDC011996B4
:1036A000DC90D88661E0C7010E94E27D8C019B839B
:1036B0008A8362E0C7010E94E27D9D838C8364E07F
:1036C000C7010E94E27D7C019F838E83B0E1DB16FF
:1036D00009F46AC0E2E1DE1609F44BC0F3E0DF1240
:1036E00031C08AE090E00E948CAD7C01DC01139631
:1036F000DC93CE93129787E392E08D939C9370E0D6
:1037000060E0CE010E94981697FD24C0F7019583D2
:1037100084830115110551F1F80180858F70823085
:1037200011F1853019F5C8010E94427E90E0D70161
:1037300017969C938E9316978BE592E08D939C93AE
:10374000FA86E986DF91CF911F910F91FF90EF905C
:10375000DF900895919581959109D70115969C93D5
:103760008E931497D6CF81E090E0E1CF90E080E097
:10377000DECF86E090E00E948CADFC01D383C28353
:103780008FE792E0918380831582148201151105E1
:1037900041F0D80118968C918F70863011F4158302
:1037A0000483FA87E987CECF86E090E00E948CAD53
:1037B000FC01D383C28385E192E091838083E1148D
:1037C000F10469F0D70118968C9118978F708230A8
:1037D00031F416968D919C9195838483E2CF90E08D
:1037E00080E0FACFEF92FF920F931F93CF93DF9376
:1037F000EC017B018E819F81892B01F58881998164
:103800000E94427E082F10E005301105BCF40E9492
:103810001571FC01892B41F08085807F8260808753
:103820001186128613861486FF83EE83BF0188817A
:1038300099810E947E7E0F5F1F4FE6CFEE81FF8150
:10384000309771F080858F70823051F4F782E68274
:10385000C701DF91CF911F910F91FF90EF900895D5
:10386000F12CE12CF5CFCF93DF93EC0161EF73E006
:1038700082E89CE00E94AB688C819D810E9428AE0A
:1038800070E060E08A819B810E94F21B1D821C8295
:1038900081E090E0DF91CF910895CF92DF92EF9297
:1038A000FF920F931F93CF93DF93EC010E94C617F3
:1038B0008C819D81892B61F40A811B8185E090E0D8
:1038C0000E948CADBC01C8010E94F21B9D838C83B9
:1038D000EC80FD80E114F104A9F461E871E187E76F
:1038E0009CE00E94B06987E79CE00E94A76890E096
:1038F00080E0DF91CF911F910F91FF90EF90DF90CB
:10390000CF9008951092B0081092AF081092AA08B4
:103910001092A9081092B1081092B2081092B30840
:103920001092B4081092AB081092AC081092AD0837
:103930001092AE081092270810926908EA81FB8164
:10394000309759F082819381009739F0DC01189605
:103950002C912F70263009F468C06AE371E187E783
:103960009CE00E94B06961E070E08C819D81892BB0
:1039700011F470E060E087E79CE00E94EF7D68E36F
:1039800071E187E79CE00E94B06961E070E08A81A4
:103990009B81892B11F470E060E087E79CE00E9436
:1039A000EF7D66E371E187E79CE00E94B069EA8100
:1039B000FB8161E070E082819381892B11F470E0DA
:1039C00060E087E79CE00E94EF7D64E371E187E7B8
:1039D0009CE00E94B069EA81FB810280F381E02DC6
:1039E00080858F7061E070E0863011F470E060E0F7
:1039F00087E79CE00E94EF7D62E371E187E79CE04E
:103A00000E94B06987E79CE00E94A76863E571E1C6
:103A100087E79CE00E94B06987E79CE00E94A76866
:103A2000EC81FD8182E0808362CF62E074E00E94DD
:103A3000667D009709F4A8C0FC0120852F70243012
:103A400009F0A2C0C184D284B6018FE19DE00E943A
:103A50004A696EE271E18FE19DE00E94B06910E079
:103A600000E0C114D10409F486C0B8016A517F4E48
:103A7000C6010E94A6B0892B09F077C0F801E65173
:103A8000FF4E25913491922F832FD70113969C934B
:103A9000139714968C93EA81FB8169E074E082812C
:103AA00093810E94667DEC81FD81009709F472C0CC
:103AB000DC0118962C9118972F70223009F06AC0FB
:103AC00019964D915D916D917C911C974115510511
:103AD0006105710509F45EC05283418341815281C1
:103AE000052E000C660B770B238182E79BE00E947A
:103AF000016EEC81FD8141815281052E000C660B27
:103B0000770B238185ED9AE00E94016EEA81FB81AB
:103B10006FE174E0828193810E94667D009739F0A5
:103B2000FC0181859285909368088093670869E617
:103B300071E18CE69CE00E94B069EA81FB81019012
:103B4000F081E02D608171818CE69CE00E944A69E1
:103B50008CE69CE00E94A768EC81FD8181E0808377
:103B60008093000281E090E0C4CE0A5F1F4F0834CA
:103B7000110509F076CF69EC70E18FE19DE00E94BC
:103B8000B06996E080E081CF86E090E0F701948311
:103B9000838381CF80E09BE4928381839FCFCF9208
:103BA000DF92EF92FF920F931F93CF93DF93EC017D
:103BB0006A017B018E819F81892B01F58881998122
:103BC0000E94427E082F10E005301105BCF40E94CF
:103BD0001571FC01892B41F08085807F8260808790
:103BE0001186128613861486FF83EE83BF018881B7
:103BF00099810E947E7E0F5F1F4FE6CFEE81FF818D
:103C0000309711F180858F708230F1F4C186D286B1
:103C1000E386F48661E676E08FE19DE00E94B0697C
:103C20002AE030E0B701A6018FE19DE00E94C46860
:103C30008FE19DE0DF91CF911F910F91FF90EF9069
:103C4000DF90CF900C94A768DF91CF911F910F91D7
:103C5000FF90EF90DF90CF9008950F931F93CF9335
:103C6000DF938C01FC01C081D1816FE270E0CE0155
:103C70000E9471BE0097D9F0FC011192CF010E9401
:103C8000F015EC016DE676E08FE19DE00E94B069F1
:103C9000BE018FE19DE00E94EF7D8FE19DE00E94DB
:103CA000A768CE01DF91CF911F910F910895CE01AA
:103CB0000E94F015EC01892BA1F3F801118210820A
:103CC000F0CF2F923F924F925F926F927F928F929E
:103CD0009F92AF92BF92CF92DF92EF92FF920F939B
:103CE0001F93CF93DF93CDB7DEB762970FB6F894EB
:103CF000DEBF0FBECDBF5C014B0129013A01CA01F5
:103D0000B9010E94D8BA1B013F926F9385EE93E0F0
:103D10009F938F93CE0101967C019F938F930E9476
:103D2000B9BE0F900F900F900F900F900F9020E062
:103D300030E0A901C301B2010E940EBB181624F0A5
:103D400077FA709477F87094F70101900020E9F702
:103D500031976F01CE18DF088EE28083A2E0B0E0D9
:103D6000AC0FBD1FAC0DBD1DBA8BA98BB10137FEC9
:103D700003C0719561957109072E000C880B990B92
:103D80000E940DB89B01AC01C301B2010E94F9B9B8
:103D900020E030E040E251E40E946CB80E94D8BAC2
:103DA000605DE989FA896083FE01EC0DFD1D1382D7
:103DB000D501ED91FC910288F389E02D9801A701CE
:103DC000B401C501199562960FB6F894DEBF0FBE17
:103DD000CDBFDF91CF911F910F91FF90EF90DF90BA
:103DE000CF90BF90AF909F908F907F906F905F909B
:103DF0004F903F902F900895DA01E0917A09F0E01A
:103E0000FE2FEE27E60FF71F90E0982F8827A901D5
:103E1000BD018E0F9F1F0C949972CF93DF931F9259
:103E2000CDB7DEB720917A0930E0322F2227260F56
:103E3000371F90E0982F8827498341E050E0BE016A
:103E40006F5F7F4F820F931F0E9499720F90DF91D7
:103E5000CF910895CF93DF931F92CDB7DEB741E0A6
:103E600050E0BE016F5F7F4F0E940E7289810F90FC
:103E7000DF91CF91089520917A0930E0322F2227E7
:103E8000620F731F90E0982F8827860F971F0C945E
:103E90002A1F63E070E00C943B1F9F92AF92BF9289
:103EA000CF92DF92EF92FF920F931F93CF93DF9306
:103EB000EC017B018091C20A811121C01B821A8210
:103EC00088EE93E0A0E0B0E08C839D83AE83BF8357
:103ED0008DE693E09983888388E08C8788EE93E071
:103EE0009E878D87CE01DF91CF911F910F91FF901B
:103EF000EF90DF90CF90BF90AF909F90089534E007
:103F0000932E833311F028E0922E82EBC82E8AE0A4
:103F1000D82E10E098E0B92EA12CD6012D913D911C
:103F20006D01F701848195812817390791F4812F5C
:103F30000E94E276082F873111F08C3139F5812FFC
:103F40000E94CE75892B59F50C3119F4812F0E94EE
:103F5000C6761F5F9112E1CFA11008C0D701ED9185
:103F6000FC910084F185E02DC70119951B821A820E
:103F700088EE93E0A0E0B0E08C839D83AE83BF83A6
:103F80008DE693E099838883BC86A8CF843149F07D
:103F90008111DFCFF601329711821082DACFB12E74
:103FA000D8CFAA24A394D5CF8F929F92AF92BF92DD
:103FB000CF92DF92EF92FF920F931F93CF93DF93F5
:103FC000CDB7DEB72F970FB6F894DEBF0FBECDBFCB
:103FD0005C014B017A018091C20A8823C9F104E097
:103FE000833309F008E0B501CE0101960E944D1F10
:103FF00082EBC82E8AE0D82E10E0F6012191319193
:104000006F01F501848195812817390751F4812FBB
:104010000E94E276873129F4A701B401812F0E9422
:1040200044751F5F0113E9CFC7012F960FB6F894AF
:10403000DEBF0FBECDBFDF91CF911F910F91FF90DB
:10404000EF90DF90CF90BF90AF909F908F900895AA
:10405000F12CE12CE9CFDA01E0917A09F0E0FE2FB2
:10406000EE27E60FF71F90E0982F8827A901BD01E2
:104070008E0F9F1F0C940E7244E050E0BC018FE045
:1040800090E00C94997244E050E0BC0185E090E02F
:104090000C94997244E050E0BC0181E090E00C94F3
:1040A000997208959F92AF92BF92CF92DF92EF9252
:1040B000FF920F931F93CF93DF938C015B01942E9C
:1040C000E52EFC01C688D788F08C80E591E00E943F
:1040D00003808F2D0E94EA74C92DDE2D8C179D0759
:1040E00008F4EC019E01A501B6018F2D0E946774B2
:1040F000F801868997898C0F9D1F978B868BCE013F
:10410000DF91CF911F910F91FF90EF90DF90CF90B3
:10411000BF90AF909F900895CF93FC01C08D80E534
:1041200091E00E94038060E270E08C2F0E94FE719B
:1041300062E070E08C2F0E943B1F84FD16C062E09D
:1041400070E08C2F0E943B1F83FF0AC048E162E0B1
:1041500070E08C2F0E940D1F80E090E0CF910895B9
:1041600080E591E00E940380E3CF40E162E070E0EF
:104170008C2F0E940D1F81E0F0CFFF920F931F93B1
:10418000CF93DF93EB01FC01178A168A2A81211154
:1041900009C02B81211106C02C81211103C02D8162
:1041A000222301F141155105E9F08A01FC01F08C4F
:1041B00080E591E00E940380AE014E5F5F4F24E0F6
:1041C00030E06CE070E08F2D0E94FC1EB8018F2D56
:1041D0000E94F17681E090E0DF91CF911F910F91E5
:1041E000FF90089580E0F7CF0F931F93CF938C013A
:1041F000FC016481758181E20E941D77C82F88309F
:10420000F8F480E591E00E9403808C2F0E94491F02
:10421000833131F08C2FCF911F910F910C94C67682
:1042200062E070E08C2F0E94FE71F801848195811C
:10423000EC2FF0E0EE0FFF1FEE54F54F91838083DB
:10424000CF911F910F9108950F931F93CF93DF93F9
:104250001F921F92CDB7DEB7FC0124852830E0F411
:104260008C0180E591E00E94038022E030E0AE0105
:104270004F5F5F4F60E170E0F80184850E942B2062
:1042800089819A819827892798270F900F90DF912D
:10429000CF911F910F91089590E080E0F6CF0F939A
:1042A0001F93CF93DF931F921F92CDB7DEB7FC0110
:1042B00024852830E0F48C0180E591E00E940380A1
:1042C00022E030E0AE014F5F5F4F64E070E0F80144
:1042D00084850E942B2089819A8198278927982795
:1042E0000F900F90DF91CF911F910F91089590E063
:1042F00080E0F6CFCF93DF93EC018BE993E09983D5
:1043000088831A821B821C821D8280E591E00E94B4
:104310000380BE016E5F7F4F44E050E08FE090E08D
:104320000E940E72CE01DF91CF9108950E945A73C0
:10433000882331F08091C20A843329F0873381F0D9
:1043400090E080E0089580E591E00E94038085E39D
:1043500090E00E942A1F85FD0DC082E090E0089544
:1043600080E591E00E9403808EE290E00E942A1F87
:1043700080FFF3CF81E090E008951F920F920FB677
:104380000F9211240BB60F922F933F934F935F938D
:104390006F937F938F939F93AF93BF93EF93FF930D
:1043A0008091B900887F803609F44DC008F040C084
:1043B000883209F4A7C028F5803109F49BC0C8F4FD
:1043C000882309F4F7C0883009F494C0FF91EF9175
:1043D000BF91AF919F918F917F916F915F914F911D
:1043E0003F912F910F900BBE0F900FBE0F901F901B
:1043F0001895883109F486C0803241F780935309BB
:1044000014C0803409F49BC040F48033B9F388337E
:10441000E9F68093530985ECAEC0803509F483C07A
:10442000883509F494C0883489F60E94D00BCECF29
:10443000883909F48AC038F5883729F050F488366D
:1044400011F0803719F683E08093540910925209D5
:1044500055C0883809F479C0803919F0803809F0DE
:10446000B5CF80915209803208F06FC0E0915209B7
:1044700081E08E0F809352098091BB00F0E0EE5CEA
:10448000F64F80833BC0803B39F0D0F4803A09F48A
:1044900077C0883A09F09ACF84E08093540910924B
:1044A000310910923009F0E0E0E01995809130096F
:1044B00081110FC081E0809330091092100909C06A
:1044C000803C09F4A8CF883C09F4A5CF883B09F0CB
:1044D0007DCFE091310981E08E0F80933109F0E0CA
:1044E000E05FF64F80818093BB009091310980910D
:1044F000300929C0809179098093BB0085EC8093B5
:10450000BC0064CF9091780980917709981758F58D
:10451000E091780981E08E0F80937809F0E0E95A04
:10452000F64F8081E9CFE091780981E08E0F80938A
:1045300078098091BB00F0E0E95AF64F80839091B2
:104540007809809177099817C8F285E8D8CFE0916B
:10455000780981E08E0F809378098091BB00F0E0AC
:10456000E95AF64F80838091560981115ECF81E030
:104570008093550984EA8093BC001092540926CF99
:1045800085EC8093BC0010925409809152098032CE
:1045900030F4E0915209F0E0EE5CF64F1082609149
:1045A000520970E082E399E0F0E0E0E019951092A2
:1045B00052090CCF1092530938CF4F925F926F92ED
:1045C0007F92AF92BF92CF92DF92EF92FF920F93C2
:1045D0001F93CF93DF9300D01F92CDB7DEB72B018F
:1045E0003C0129833A834B835C83A60195016E0DC0
:1045F0007F1D801F911F0E9450B929813A814B81F4
:104600005C81621773078407950708F52415350543
:1046100046055705A8F421E0822F0F900F900F90C8
:104620000F90DF91CF911F910F91FF90EF90DF904E
:10463000CF90BF90AF907F906F905F904F90089514
:1046400021E0461657066806790630F30FC0461675
:1046500057066806790650F421E089819A81AB817A
:10466000BC8184159505A605B705B0F220E0D4CF2E
:104670008F929F92AF92BF92CF92DF92EF92FF9272
:104680000F931F93CF93DF937C014A015901C0918F
:104690000C09D0910D09062F660F110B209709F414
:1046A0005CC088858F70863009F055C06EE074E07C
:1046B000CE010E94667D6C0182E08816910449F06B
:1046C00066EC73E0E3E08E16910429F0D0E0C0E0E0
:1046D00006C063E174E0CE010E94667DEC01C11466
:1046E000D104D9F1F60180858F708430B1F56185F0
:1046F0007285A801C7010E9462BEA80168E174E04A
:10470000C7010E9444BE209779F188858F7084305C
:1047100059F569857A85A801C7010E9444BEA801A0
:1047200068E174E0C7010E9444BEA114B10429F0FD
:10473000A801B501C7010E9444BEC701DF91CF9116
:104740001F910F91FF90EF90DF90CF90BF90AF90AF
:104750009F908F900895D0E0C0E0A80160EB72E1D7
:10476000C7010E94DDB0C9CFF2E08F16910481F03D
:1047700083E08816910429F060917B0970917C098F
:10478000CACFA8016AEA72E1C7010E94BFB0C7CFD1
:10479000A80167EA72E1F8CFCF92DF92EF92FF9221
:1047A0000F931F93CF93DF93CDB7DEB7C054D109DA
:1047B0000FB6F894DEBF0FBECDBF809182099091F5
:1047C0008309059709F449C06115710509F445C0CD
:1047D00069017A018B0140E450E0CE0101960E940C
:1047E00062BE6FE270E0CE0101960E9429BE892B65
:1047F00041F4980143E050E060E4CE0101960E944C
:10480000382340E450E0B601CE0101960E9444BE38
:104810000E94817D882309F180918209909183090A
:104820000697D9F480910E09811117C0B701CE0106
:1048300001960E94058681E090E0C05CDF4F0FB6D4
:10484000F894DEBF0FBECDBFDF91CF911F910F91C6
:10485000FF90EF90DF90CF90089590E080E0EDCF53
:10486000AF92BF92CF92DF92EF92FF921F93CF93BE
:10487000DF9300D000D0CDB7DEB76C017C0110E033
:104880008AE0A82EB12C133061F1F701828190E00B
:10489000B0E0A0E089839A83AB83BC83BE82AD8203
:1048A000BE016F5F7F4F8FE19DE00E94681565EA52
:1048B00072E10E94B0691F5FFFEFEF1AFF0A143028
:1048C00011F726960FB6F894DEBF0FBECDBFDF916D
:1048D000CF911F91FF90EF90DF90CF90BF90AF905E
:1048E0000895F601858190E0B0E0A0E089839A8385
:1048F000AB83BC83BE82AD82BE016F5F7F4F8FE111
:104900009DE00E94681562EA72E1D3CF68EC7FE017
:104910008CE69CE00E94B06965EB7FE08CE69CE051
:104920000E94B06967EA7FE08CE69CE00E94B06973
:104930006FE97FE08CE69CE00E94B0698CE69CE029
:104940000E94A76862E97FE08CE69CE00E94B06963
:1049500062E87FE08CE69CE00E94B06966E77FE059
:104960008CE69CE00E94B0696FE57FE08CE69CE0FD
:104970000E94B0696DE47FE08CE69CE00E94B06923
:1049800068E37FE08CE69CE00E94B06969E27FE02A
:104990008CE69CE00E94B0696AE17FE08CE69CE0D6
:1049A0000E94B06962E17FE08CE69CE00E94B06901
:1049B00067E07FE08CE69CE00E94B0696DEF7EE0EE
:1049C0008CE69CE00E94B06965EF7EE08CE69CE09E
:1049D0000E94B06969EE7EE08CE69CE00E94B069BE
:1049E0006FEC7EE08CE69CE00E94B06960EB7EE0BC
:1049F0008CE69CE00E94B0696BE97EE08CE69CE06E
:104A00000E94B0696EE87EE08CE69CE00E94B0698E
:104A100060E87EE08CE69CE00E94B06964E77EE09E
:104A20008CE69CE00E94B0696CE67EE08CE69CE03F
:104A30000E94B06961E67EE08CE69CE00E94B0696D
:104A400064E57EE08CE69CE00E94B0696CE47EE068
:104A50008CE69CE00E94B06961E47EE08CE69CE01C
:104A60000E94B06962E37EE08CE69CE00E94B0693F
:104A700069E27EE08CE69CE00E94B0698CE69CE0F6
:104A80000C94A7680F931F93CF93DF9300D000D0AF
:104A9000CDB7DEB70E94862463E67AE08CE69CE020
:104AA0000E94B069CE0101960E947A21CE01019642
:104AB0000E9430240BE913E01A8309831B821C82B5
:104AC0001D821E8280E591E00E94038044E050E058
:104AD000BE016D5F7F4F81E090E00E940E72CE01BB
:104AE00001960E9430241A8309831B821C821D8236
:104AF0001E8280E591E00E94038044E050E0BE0108
:104B00006D5F7F4F85E090E00E940E72CE010196AE
:104B10000E94302469E87AE08CE69CE00E94B0694B
:104B200026960FB6F894DEBF0FBECDBFDF91CF91B2
:104B30001F910F910895009789F0FC0120852F7037
:104B4000253061F40E94E27D009741F0FC01208550
:104B50002F70243019F481859285089590E080E0CB
:104B60000895CF92DF92EF92FF920F931F93CF930E
:104B7000DF9300D000D0CDB7DEB780910B09811153
:104B80009CC0809182099091830902970CF495C092
:104B900000912308109124080115110509F48DC016
:104BA00062E072E08EE39DE00E94CE116CE174E061
:104BB000C8010E94667D8C01009709F47EC00E94A6
:104BC000427EE82EF12CE114F10409F476C070E085
:104BD00060E0C8010E949B256C01EA94EF2809F46B
:104BE0007BC061E0C8010E94E27DFC010185128565
:104BF000CE0101960E947A21CE0101960E94068084
:104C000064E57AE08CE69CE00E94B069B6018CE62F
:104C10009CE00E944A696DE076E08CE69CE00E9490
:104C20004A69B8018CE69CE00E94EF7D6DE076E079
:104C30008CE69CE00E944A6963EC7AE08CE69CE09A
:104C40000E944A698CE69CE00E94A768D092340DCD
:104C5000C092330D1093360D0093350D83EC9AE01E
:104C6000892BE9F58AE194E09093380D8093370D14
:104C700080917D0990917E09009741F070E060E09D
:104C80000E949B2590937C0980937B0980917B09EE
:104C900090917C09009721F090933A0D8093390D03
:104CA00010923C0D10923B0D81E080930B096BE359
:104CB0007AE08CE69CE00E94B06926960FB6F894E4
:104CC000DEBF0FBECDBFDF91CF911F910F91FF903F
:104CD000EF90DF90CF90089502E012E089CF83EC4F
:104CE0009AE0C2CFCF92DF92EF92FF921F93CF93C1
:104CF000DF9300D000D0CDB7DEB766E37AE08CE674
:104D00009CE00E94B06980EDE82E8DE0F82E10E066
:104D100090E1C92ED12CF70181917F01803130F4CF
:104D200063E274E08CE69CE00E944A69153041F130
:104D3000F7013197808190E0B0E0A0E089839A8309
:104D4000AB83BC83DE82CD82BE016F5F7F4F8CE67A
:104D50009CE00E94681564E37AE00E94B0691F5FDE
:104D60001630C9F626960FB6F894DEBF0FBECDBF3B
:104D7000DF91CF911F91FF90EF90DF90CF9008953A
:104D80008091D50D90E0B0E0A0E089839A83AB8359
:104D9000BC83DE82CD82BE016F5F7F4F8CE69CE0DC
:104DA0000E9468150E94A768DACF0F931F93CF93D4
:104DB000DF9300D000D01F92CDB7DEB78B01CE01BC
:104DC00007969F938F9301979F938F9301979F933C
:104DD0008F9301979F938F9301979F938F93019741
:104DE0009F938F9301979F938F9385E294E09F9376
:104DF0008F93FB0183818F9382818F930E94E9BE01
:104E00000FB6F894DEBF0FBECDBF0697C4F460E0C6
:104E10007DE087E79CE00E94B069F80162817381C0
:104E200087E79CE00E944A6927960FB6F894DEBF98
:104E30000FBECDBFDF91CF911F910F9108950E94BA
:104E4000722662E17DE08CE69CE00E94B069ECCFC6
:104E5000EF92FF920F93CF93DF93CDB7DEB7A0977A
:104E60000FB6F894DEBF0FBECDBF7C0100E020E09E
:104E700033E040E250E0BE016F5F7F4F0E943C197B
:104E8000BE016F5F7F4F8FE19DE00E944A6961E143
:104E90007AE08FE19DE00E94B069F701628162953E
:104EA0006F708FE19DE00E94DB7D6AE07AE08FE128
:104EB0009DE00E94B069F70162816F708FE19DE013
:104EC0000E94DB7D8FE19DE00E94A768A0960FB64F
:104ED000F894DEBF0FBECDBFDF91CF910F91FF9051
:104EE000EF9008952F923F924F925F926F927F9230
:104EF0008F929F92AF92BF92CF92DF92EF92FF92EA
:104F00000F931F93CF93DF93CDB7DEB768970FB69C
:104F1000F894DEBF0FBECDBF1C0109871A872B870F
:104F20003C874D875E876F87788B2DE0E216F10412
:104F300008F033C0F701E356FD4F3081398BCE01C5
:104F400009960E940C0F97FD04C0BC01C1010E948C
:104F50002E0F9B85892F8F70D1011296EC9112979D
:104F6000E07FE82B1296EC931297E295EF70EC300D
:104F700008F061C0F0E08827EF53F84D8F4F0C9494
:104F8000DBB91029E927E9271F29CF27D2291029C2
:104F900030293029302910291029198AD0CFB12C75
:104FA00092959F70EFEFE90FEB3008F0A5C4F0E0A9
:104FB0008827E252F84D8F4F0C94DBB9122A322A1F
:104FC000122AD529D529122A122A7C2C7C2C122AA5
:104FD000122A92959F70EFEFE90FEB3008F009C1AC
:104FE000F0E08827E950F84D8F4F0C94DBB9CD28BD
:104FF000C128832805280228A428D128F928F928BF
:105000008E288E288889F10187838F85D101169695
:105010008C9316978E8515968C9315978D8514967F
:105020008C9314979295907F12968C9112978F7013
:10503000982B12969C93B989BB2309F4CAC1F1013C
:10504000828182958F702B2F30E08217130609F42E
:10505000C0C164E778E08FE19DE00E94B069D101B2
:1050600012966C9162956F708FE19DE00E94DB7DDE
:1050700061E778E08FE19DE00E94B06969898FE186
:105080009DE00E94DB7D6FE678E08FE19DE00E946D
:10509000B069F101008119821A821B821C821D8273
:1050A0001E821F82188689898295807F9B819F70CE
:1050B000892B8B830983EE24EA94FE2C11812281B3
:1050C00033814481558166817781CE0101960E94AA
:1050D0007227D1012C9311963C93119712964C9301
:1050E000129713965C93139714966C9314971596D6
:1050F0007C93159716968C93169717969C93C101DF
:105100000E94282766C18F859889F101868387814F
:1051100090FB80F987838E8585838DCF8D859E85D5
:10512000AF85B8898F3F9105A105B10529F024F01D
:105130008FEF90E0A0E0B0E0B7FF03C080E090E028
:10514000DC01F101848377CF6D857E858F85988919
:105150002AE030E040E050E00E9472B92F3F310574
:105160004105510529F024F02FEF30E040E050E0F8
:1051700057FF03C020E030E0A901D10114962C9321
:105180005ACF8F859889F1018683878190FB80F9BA
:1051900087838E8585838D85D5CF8D8514968C9359
:1051A0004ACFCD84DE84EF84F88820E030E0A90186
:1051B000C701B6010E9406B887FD17C020E030E0A5
:1051C0004FE753E4C701B6010E940EBB181634F432
:1051D000C12CD12CAFE7EA2EA3E4FA2EC701B60109
:1051E0000E94DFBAF101648326CFC12CD12C760155
:1051F000F5CF64EF78E08FE19DE00E94B0696B85A8
:1052000062956F708FE19DE00E94DB7D61EF78E039
:105210008FE19DE00E94B069D10112966C91B7C0F8
:105220004D855E856F857889F1014483558366835A
:105230007783907F82818F70982B9283FCCE60E081
:10524000CE0109960E94CE0DD10114968C9314972D
:1052500012968C9112978F70806212968C93EBCE7F
:1052600092959F70EFEFE90FEB3008F07BC0F0E014
:105270008827E25CF64D8F4F0C94DBB95B298529BA
:105280009829852985294929752975297529692923
:1052900070296D857E858F8598890E940DB820E0E4
:1052A00030E040E251E40E9466BAF1016483758304
:1052B00086839783C0CE6D8570E090E080E00E9489
:1052C0000BB8D10114966D937D938D939C93179792
:1052D000B2CE6D857E858F8598890E940DB8E5CF09
:1052E0006D857E858F859889EACF9295907FF101B3
:1052F00082818F70982B92838D859E85AF85B8892A
:1053000084839583A683B78396CE9295907F1296D9
:105310008C9112978F70982B12969C938D859E85F9
:10532000AF85B889F10184839583A683B78383CE43
:1053300060E0C1010E94CE0DD10114968C931497A8
:105340008F85988916968C93169717968C91179738
:1053500090FB80F917968C9317978E8515968C93F2
:10536000159776CF6FED78E08FE19DE00E94B069F0
:105370006B8562956F708FE19DE00E94DB7D6CED27
:1053800078E08FE19DE00E94B069F1016281629551
:105390006F708FE19DE00E94DB7D8FE19DE00E94B8
:1053A000A76849CEBB24B394FBCD4D855E856F8540
:1053B0007889D10114964D935D936D937C931797E3
:1053C0009295907F12968C9112978F70982B1296CF
:1053D0009C9388E0F101DE01119601900D928A956F
:1053E000E1F729813A814B815C816D817E818F81DA
:1053F000988568960FB6F894DEBF0FBECDBFDF91DB
:10540000CF911F910F91FF90EF90DF90CF90BF90C1
:10541000AF909F908F907F906F905F904F903F9054
:105420002F900895963009F43AC148F46D85913073
:1054300071F06FEF70E0933051F060E008C097308A
:1054400009F439C19A506D857E859230B0F784E6B3
:105450008F8788898E7F888B1E868B858F70806270
:105460008B876D872E8530E0AFEFB0E00E94A4B946
:1054700024E630E040E050E00E9472B969017A0110
:10548000BFEFCB16D104E104F10429F024F0C12CC4
:10549000D12C7601CA948601ED85EA8B6E2E712C93
:1054A000BB2009F471C088898695282F2150330BC1
:1054B00029013FEF4316530609F01EC100381105BC
:1054C0000CF000C18FE790E08C199D09869DD001FA
:1054D000879DB00D969DB00D11242FEF30E00E94F6
:1054E000F2B921E83EE740E050E00E9472B9D101F4
:1054F00017962C93ABE9B0E0A70196010E9491B9F1
:10550000EFE78E2E912CA12CB12CA50194010E94C5
:1055100072B989019A010C591F4F2F4F3F4FAEEFBF
:10552000B1E0A70196010E9491B9A50194010E94E2
:1055300072B9D3010E9491B92FEF30E040E050E002
:105540000E9472B939012F3F310521F01CF0662409
:105550006A94712C6FEC78E08FE19DE00E94B06955
:10556000B8018FE19DE00E94EF7D61EC78E08FE172
:105570009DE00E94B069B3018FE19DE00E94EF7D44
:105580008FE19DE00E94A768EAE8F5E1E491F0E090
:10559000EE0FFF1FE059FA4E85919491E0EEF5E190
:1055A000E4912F8538893170AFEFBFEF0E94A4B925
:1055B0002DE631E040E050E00E9472B944275527C3
:1055C000AAEFB5E00E9491B9DC01CB019058AF4F32
:1055D000BF4FCD01BB2797FDB095AB2F8E3FE1E0CC
:1055E0009E0708F062C1382F8F3F910508F47FC1F4
:1055F0004EEF481B50E03FEFF301319678012FEF5B
:10560000E21AF20A009510E03E9DC0013F9D900D08
:105610001124292F3327200F311FDF010E94F2B9F7
:105620004B015C018824AA24BB245E9D90015F9DF0
:10563000300D1124232F3327200F311F0E94F2B980
:10564000BB27A92F982F872F882A992AAA2A4E9DEF
:1056500090014F9D300D1124232F3327200F311F30
:10566000DF010E94F2B9B82FA72F962F882788272D
:105670009927BB2788299929AA29F101A68395830F
:10568000848365E978E08FE19DE00E94B069C10103
:105690000E94282760E080E00E947283CCCC6D8558
:1056A0007E858F8598892AE030E040E050E00E94B6
:1056B00072B9B901CCCE6D857E858F8598890E949F
:1056C000D8BAC5CEA7019601205831094109510920
:1056D000ABE9B0E00E9491B92FE730E040E050E044
:1056E0000E9472B989019A010C591F4F2F4F3F4FE9
:1056F000D10117961C922ECF9201AAEBBFEF0E9408
:10570000EAB944E6842E912CA12CB12CA501940178
:105710000E9472B9DA01C9018C599F4FAF4FBF4F38
:105720008B8B9C8BAD8BBE8B26E430E0D2010E942C
:10573000F2B9A50194010E9472B949015A019EE192
:10574000890E911CA11CB11C003811050CF093C0EE
:105750008FE790E08C199D09869DD001879DB00D43
:10576000969DB00D1124A50194010E949CB99B0146
:10577000AC01AFEFB0E00E9491B924E63AE640E018
:1057800050E00E9472B9D10117962C932B893C8965
:105790004D895E892C0D3D1D4E1D5F1DAEEFB1E0A4
:1057A0000E9491B923EE30E040E050E00E9472B9CF
:1057B00029013A01388F2F8BAFEFB0E0A701960196
:1057C0000E9491B92FE730E040E050E00E9472B9AA
:1057D0008901EA89AE2FB0E0A30192010E9491B93C
:1057E0002FEF30E040E050E00E9472B939012F3FC6
:1057F000310521F01CF066246A94712C6BEB78E083
:105800008FE19DE00E94B0692AE030E04B895C891D
:105810006D897E898FE19DE00E94C46865EB78E028
:105820008FE19DE00E94B0692AE030E0B501A4015B
:105830008FE19DE00E94C4686DEA78E08FE19DE011
:105840000E94B069B8018FE19DE00E94EF7D65EA9A
:1058500078E08FE19DE00E94B069B3018FE19DE0A7
:105860000E94EF7D6CE978E08FE19DE00E94B069D5
:105870006F89788D81CEA7019601205831094109A1
:105880005109ABE9B0E00E9491B92FE730E040E068
:1058900050E00E9472B989019A010C591F4F2F4F95
:1058A0003F4FD10117961C92A9CF8C3FF3E09F0781
:1058B00068F48D3F22E0920728F452E0580F3FEF42
:1058C00040E09ACE3CEF381B5FEFFACF8A3F35E0DD
:1058D000930781F08B3FE4E09E0728F444E0480FF3
:1058E0005FEF30E089CE5AEF581B30E001C050E046
:1058F0004FEF82CE50E0F9CF63E878E08FE19DE092
:105900000E94B0696B8562956F708FE19DE00E9487
:10591000DB7D60E878E07CCCAF92BF92CF92DF92E3
:10592000EF92FF920F931F93CF93DF93CDB7DEB724
:1059300068970FB6F894DEBF0FBECDBFFC01098B90
:105940001A8B2B8B3C8B4D8B5E8B6F8B788F828170
:105950009381009709F49FC024813581232B09F49A
:105960009AC0CC2009F497C06F0170E060E00E94FB
:105970009816192FD601ED91FC91028CF38DE02D34
:10598000C60119955C018230910509F478C003972E
:1059900009F447C095E0F1E0AF16B10409F091E0D9
:1059A00019861A861B861C861D861E861F86188AE7
:1059B0009295907F8B858F70892B8B87EE24EA944C
:1059C000FE2C09891A892B893C894D895E896F894A
:1059D000788DCE0109960E947227F1E0AF16B104CE
:1059E00009F44FC082E0A816B10409F045C06F85E4
:1059F00070E0D60114968C910E94AE8361E070E055
:105A0000C6010E94C3166E8570E00E94AE8362E0FC
:105A100070E0C6010E94C3166D8570E00E94AE83DF
:105A20002BC0612F661F6627661FCE0141960E941C
:105A3000CE0D5C01BC01D60114968C910E94AE8300
:105A400064E872E18FE19DE00E94B069F601648133
:105A500075818FE19DE00E94EF7D62E872E18FE148
:105A60009DE00E94B069B5018FE19DE00E94EF7D4D
:105A70008FE19DE00E94A76881E090E00EC094E075
:105A80008FCF63E070E0C6010E94C316688970E0A2
:105A90000E94AE83ACCF90E080E068960FB6F89499
:105AA000DEBF0FBECDBFDF91CF911F910F91FF9051
:105AB000EF90DF90CF90BF90AF900895AF92BF92DC
:105AC000CF92DF92EF92FF920F931F93CF93DF93CA
:105AD000CDB7DEB7CC55D1090FB6F894DEBF0FBEF7
:105AE000CDBF5C0166960FAF669767961FAF67974D
:105AF00068962FAF689769963FAF69976A964FAFE0
:105B00006A976B965FAF6B976C966FAF6C976D965D
:105B10007FAF6D971AAA19AAFE01F39682E1DF0101
:105B20001D928A95E9F77A961192119286E0DF012B
:105B30001D928A95E9F7CE018B5A9F4F0E94282724
:105B4000F0FE2CC06696EFAD6697E83108F08DC088
:105B5000F0E08827E155F24D8F4F0C94DBB93B2ED6
:105B6000C72D322E352E352E322EC72D352E352E01
:105B7000352EC72DC72DC72D352E352E352E352E5A
:105B8000352E352E352E352E352E352E3B2E6CE608
:105B900078E0CE01835B9F4F0E94AFB068968FADD7
:105BA000689782958F70813008F48DC0833018F02B
:105BB000883009F088C00E94817D882309F41DC1C6
:105BC00080910E09811119C1C114D10409F015C1C8
:105BD00030E020E043E050E060E3CE0101960E9417
:105BE0003823D501ED91FC91608171814FE250E045
:105BF000CE0101960E9444BE01E020E032E044E183
:105C000050E0BE016F5C7F4FCE018B5A9F4F0E94C8
:105C10003C19F1FE07C066968FAD6697823011F091
:105C2000853061F5F0FE4FC0BE01635B7F4FCE0152
:105C300001960E9405866BE478E08FE19DE00E946A
:105C4000B069BE016F5F7F4F8FE19DE00E944A699E
:105C500068E478E08FE19DE00E94B069BE01635B7B
:105C60007F4F29C068E678E094CF6AE578E08FE15D
:105C70009DE00E94B069E894F0F890CFBE016F5C9F
:105C80007F4FCE0101960E94058664E578E08FE1A2
:105C90009DE00E94B069BE016F5F7F4F8FE19DE084
:105CA0000E944A6961E578E08FE19DE00E94B06959
:105CB000BE016F5C7F4F8FE19DE00E944A698FE1DA
:105CC0009DE00E94A768C70188279271892B09F47B
:105CD000C0C030E020E043E050E060E3CE01019638
:105CE0000E943823D501ED91FC91608171814FE2D2
:105CF00050E0CE0101960E9444BEC114D10469F067
:105D000068E174E0CE0101960E941EBE4FE250E0B1
:105D1000B601CE0101960E9444BE87010027107192
:105D200068E174E0CE0101960E941EBE4FE250E091
:105D300064E478E00115110511F460E478E0CE0127
:105D400001960E94BFB068968FAD689782958F705C
:105D50008450823008F069C067E1CE018B5A9F4FB2
:105D60000E94770D26962FAF269727963FAF27974D
:105D700028964FAF289729965FAF29972A966FAF3D
:105D80002A972B967FAF2B972C968FAF2C972D961B
:105D90009FAF2D9700E020E033E044E150E0BE01EA
:105DA0006F5C7F4FCE018B5A9F4F0E943C196AE374
:105DB00078E08FE19DE00E94B069BE016F5F7F4F88
:105DC0008FE19DE00E944A6967E378E08FE19DE002
:105DD0000E94B069BE016F5C7F4F8FE19DE00E9421
:105DE0004A698FE19DE00E94A7680E94817D882317
:105DF00021F080910E09882301F1B701C5010E94AD
:105E0000511790E080E0C45ADF4F0FB6F894DEBF20
:105E10000FBECDBFDF91CF911F910F91FF90EF90FB
:105E2000DF90CF90BF90AF90089520E032E0012B3B
:105E300011F020E033E000E0B0CFBE016F5C7F4F97
:105E4000CE0101960E94058660E072E0C5010E94C5
:105E50001917F0FE73C066968FAD66978A3009F405
:105E600078C008F06EC0813009F47EC0863009F435
:105E70007BC030E020E043E050E060E3CE010196DB
:105E80000E943823D501ED91FC91608171814FE230
:105E900050E0CE0101960E9444BEC114D10469F0C5
:105EA00068E174E0CE0101960E941EBE4FE250E010
:105EB000B601CE0101960E9444BE68E174E0CE01B5
:105EC00001960E941EBE40E350E064E278E0CE01FD
:105ED00001960E94BFB06EE178E08FE19DE00E94E4
:105EE000B069BE016F5F7F4F8FE19DE00E944A69FC
:105EF0006BE178E08FE19DE00E94B069BE01635BD9
:105F00007F4F8FE19DE00E944A698FE19DE00E94F2
:105F1000A7680E94817D882309F46FCF80910E09C4
:105F200081116BCFBE01635B7F4FCE0101960E9452
:105F3000058660E071E0C5010E94191781E090E0DC
:105F400062CF8B3071F08C3009F093CF62E378E050
:105F500002C06DE278E0CE01835B9F4F0E94AFB03C
:105F600088CF68E278E0F7CFF5018085853009F0C9
:105F700080CFECCFDC01ED91FC91309729F090853A
:105F80009F7081E0953009F080E00895AF92BF9254
:105F9000CF92DF92EF92FF920F931F93CF93DF93F5
:105FA0006115710559F1A42E6B01EC01CB010E9422
:105FB000BA2FB82E882309F456C0F601E480F58084
:105FC000F7011085E114F10469F0812F8F709EEFC5
:105FD000980F9230A8F4012F059505950595059524
:105FE00009F04DC01295107F1595159515951595CD
:105FF000123009F44AC0133009F457C0B12C33C031
:10600000853081F760E0C7010E94E27D009751F37F
:10601000FC010085059505950595059519F360E04A
:10602000C7010E94E27D009761F1FC0181859285A4
:10603000A385B4858C839D83AE83BF830295007F47
:106040008A818F70082B0A83AA2021F0C6010E9442
:106050009918888360E279E08FE19DE00E94B06941
:10606000CE010E9428278B2DDF91CF911F910F9198
:10607000FF90EF90DF90CF90BF90AF900895823067
:10608000A9F280E090E0DC01D5CFF701418552858F
:10609000638574858A818F70806A8A834C835D836F
:1060A0006E837F8364E179E0D7CFF70161857285E4
:1060B000838594850E940DB82A812F7020672A83DA
:1060C0006C837D838E839F8366E079E0C5CFAF923A
:1060D000BF92CF92DF92EF92FF920F931F93CF93D5
:1060E000DF9300D000D01F921F92CDB7DEB75C01C6
:1060F0007B0173FD0DC00E94BF0C663971058105DF
:10610000910530F080918209909183090597F9F407
:10611000B70166277370C5010E9451176AE078E0E5
:106120008FE19DE00E94B0698FEF9FEF28960FB638
:10613000F894DEBF0FBECDBFDF91CF911F910F91BD
:10614000FF90EF90DF90CF90BF90AF9008951982AD
:106150001A821B821C821D821E821F8218868B81DE
:106160008F708B8341E0B501CE0101960E94C62F4E
:1061700060E073E0C5010E948717E82AF92AD12C54
:10618000C12C09811A812B813C814D815E816F81F7
:106190007885C5010E945E2DC9CF4F925F926F92A4
:1061A0007F92AF92BF92CF92EF92FF920F931F9385
:1061B000CF93DF9300D000D01F921F92CDB7DEB7F0
:1061C0005C0109831A832B833C834D835E836F8339
:1061D00078876FEB75E08FE19DE00E94B069CE019A
:1061E00001960E9428276981611134C00B810F70CC
:1061F000013081F160F1023021F010E0053009F04A
:1062000045C0D501ED91FC91068CF78DE02D0981FB
:106210001A812B813C814D815E816F817885C5011A
:10622000199581E090E028960FB6F894DEBF0FBE76
:10623000CDBFDF91CF911F910F91FF90EF90CF9045
:10624000BF90AF907F906F905F904F900895CC2457
:10625000C394D7CFF501828193810E949D178981D4
:10626000813051F1823009F4DDC062EB75E08FE1DD
:106270009DE00E94B06969818FE19DE00E94DB7D15
:106280008FE19DE00E94A76801E010E062EA75E0FE
:106290008FE19DE00E94B069B8018FE19DE00E940E
:1062A000EF7D8FE19DE00E94A768CE0101960E94DC
:1062B000282790E080E0B7CF1B8112951F70163021
:1062C00009F477C0E8F48FEF810F8230F0F11630D7
:1062D00009F4A3C008F086C01150123008F491C030
:1062E000D50112966D917C91CE0101960E94F77DA9
:1062F00060E07AE0F501828193810E9467301CC0E2
:10630000173081F186EF810F823008F78D819E81F1
:10631000AF81B88585369105A105B10524F084E6E5
:1063200090E0A0E0B0E0B7FF03C080E090E0DC01C7
:106330009C01293131055CF2D501ED91FC91068C6F
:10634000F78DE02DCC24C39462CF2D8130E0A4E6FC
:10635000B0E00E94A4B92FEF30E040E050E00E948E
:1063600072B9E7CF4D805E806F80788420E030E0A6
:10637000A901C301B2010E9406B887FD11C020E047
:1063800030E048EC52E4C301B2010E940EBB181683
:1063900054F4412C512C88EC682E82E4782E03C0F2
:1063A000412C512C3201C301B2010E94D8BA9B0189
:1063B000C0CF6D817E818F8198852AE030E040E0FA
:1063C00050E00E9472B9253631054105510524F08F
:1063D00024E630E040E050E057FFABCF20E030E073
:1063E000A901A7CF173081F01A5086E690E0A0E00F
:1063F000B0E0123008F074CF8D839E83AF83B887EE
:106400006FCF86E68D836CCF80E090E0ACECB2E499
:106410008D839E83AF83B88763CF8CEF93E0A0E03A
:10642000B0E0EACF1D821E821F821886D501ED9151
:10643000FC91068CF78DE02DCC24C39402E01A81E8
:106440002B813C8140E0E8CE0F931F93CF93DF93E5
:1064500000D000D01F921F92CDB7DEB719821A82EA
:106460001B821C821D821E821F8218862B812F7028
:106470002B83FC0102811381C8010E94991882308C
:10648000C1F08530B1F040E0B801CE0101960E9424
:10649000C62F60E0CE0101960E94CE0D28960FB661
:1064A000F894DEBF0FBECDBFDF91CF911F910F914A
:1064B000089590E080E0F2CF8F929F92AF92BF92CA
:1064C000CF92DF92EF92FF920F931F93CF93DF93C0
:1064D000CDB7DEB767970FB6F894DEBF0FBECDBF5E
:1064E0008C017B014C018BE0880E911C9F8A8E8A67
:1064F000F801128611861386168A158A672B09F40D
:1065000063C0A0908409B0908509A114B10409F476
:106510005BC06FE270E0C7010E9429BE6C01892B4D
:1065200009F44AC0F701DE01119690E080E0BD0158
:106530002191222341F02F3231F08431910519F05D
:106540002D930196F5CF860F971FFC011082C50190
:106550000E94667DF80191838083B6016F5F7F4F53
:106560004AE050E0C4010E9462BECE0146960E94FD
:106570002D1EF801968B858B8E899F89892B09F4B6
:106580001386C8010E94BA2F882319F0C8010E94FF
:10659000221B67960FB6F894DEBF0FBECDBFDF910A
:1065A000CF911F910F91FF90EF90DF90CF90BF9010
:1065B000AF909F908F900895B701C5010E94667DAE
:1065C000F80191838083DDCFF80111821082D9CF49
:1065D000CF93DF93EC01798368831A8619861B8633
:1065E0001E8A1D8A0E94BA2F882329F0CE01DF91CE
:1065F000CF910C94221BDF91CF9108954F925F921F
:106600006F927F928F929F92AF92BF92CF92EF92B2
:10661000FF920F931F93CF93DF93CDB7DEB76797AA
:106620000FB6F894DEBF0FBECDBF009709F4A4C02B
:10663000FC0120852F70253009F09EC02A015B01E6
:1066400086809780809180098F5F80938009811474
:10665000910409F48CC0F40180858F70843009F0B6
:1066600082C06185728580918409909185090E941C
:10667000667D3C01009709F476C0FC0180858F702F
:10668000853009F070C0B301CE0101960E94E83256
:10669000A114B104A9F0CE0101960E94BA2F88235B
:1066A00079F0C12C7201F5010081118122813381C1
:1066B0004481558166817781CE0101960E94E7363B
:1066C00060E0C3010E94E27D0097D1F1FC012085CA
:1066D0002F702230A9F581859285A385B48507970F
:1066E000A105B10569F561E0C3010E94E27DA20147
:1066F000B5010E94FE32A114B10489F5882379F115
:1067000080918009815080938009CE0101960E947A
:10671000810F81E067960FB6F894DEBF0FBECDBF44
:10672000DF91CF911F910F91FF90EF90CF90BF908D
:10673000AF909F908F907F906F905F904F90089553
:10674000A114B10461F4CE0101960E94BA2F8823EE
:1067500031F0CE0101960E94BE33892B89F6CE011D
:1067600001960E94810FF4018280938070CF809106
:10677000800981508093800980E0CCCF0F931F93D4
:10678000CF93DF9300D000D01F921F92CDB7DEB71A
:106790008C0119821A821B821C821D821E821F821A
:1067A00018868B818F708B83D801ED91FC9160816D
:1067B00071818FE19DE00E944A69C8010E94BA2F51
:1067C000811118C06DEC77E08FE19DE00E94B06907
:1067D0008FE19DE00E94A7680FEF1FEFC801289688
:1067E0000FB6F894DEBF0FBECDBFDF91CF911F91E2
:1067F0000F910895C8010E949918F801908597306B
:1068000039F0853049F1D0F48130E9F0823021F15E
:10681000D80119968D919C91009721F1DC01ED91A1
:10682000FC910688F789E02D199501E0892B09F480
:1068300000E0802F0E94851310E0D0CF863019F041
:106840008A50833028F769EA77E08FE19DE00E9463
:10685000B06901E010E0C2CF80E00E94851310E033
:1068600000E0BCCF40E0B801CE0101960E94C62FE7
:10687000F8018085873071F160F4833009F445C0F8
:10688000843059F06DEB77E08FE19DE00E94B069B4
:10689000E6CF8830D1F18930A9F760E0CE010196CA
:1068A0000E94CE0D8C0162EB77E08FE19DE00E94AB
:1068B000B069B8018FE19DE00E94EF7D8FE19DE01E
:1068C0000E94A76891E080E0012B09F490E0092F75
:1068D000182F84CF0280F381E02D80858F70853062
:1068E000D1F467EC77E08FE19DE00E94B06950E061
:1068F00040E070E060E0F801828193810E94FE3206
:10690000082F10E00E94851369CFCE0101960E94E6
:10691000C70E8B01C8CF10E000E0C5CF2F923F9289
:106920004F925F926F927F928F929F92AF92BF929F
:10693000CF92DF92EF92FF920F931F93CF93DF934B
:10694000CDB7DEB7CB55D1090FB6F894DEBF0FBE79
:10695000CDBF0E9437859B01AC0160911D087091ED
:106960001E0880911F0890912008AA24AA94BA2C8E
:10697000650110E3E12E15E7F12E00E010E00E9422
:10698000DD22882309F4F7C1E0918409F09185099B
:10699000309709F4F0C1809180098F5F809380095E
:1069A0002680378010E02114310409F442C1F1013E
:1069B00080858F708530F9F460E0C1010E94E27D2E
:1069C000FC0181859285A385B4850597A105B10554
:1069D00091F4B101CE0101960E94E832CE010196F8
:1069E0000E94BA2F6A968FAF6A97811108C0CE01B4
:1069F00001960E94810FF10122803380D4CF259629
:106A00001CAE1DAE1EAE1FAE259729961CAE1DAE48
:106A10001EAE1FAE299740E0BE016F5F7F4FCE01D3
:106A20008F5B9F4F0E94C62FCE0101960E947C165D
:106A300065966CAF7DAF8EAF9FAF659770E060E0FD
:106A4000CE0101960E9498164C01CE018F5B9F4F9C
:106A50000E94800E69966CAF7DAF8EAF9FAF699735
:106A6000CE0101960E949918182F63962EAD3FAD66
:106A70006397B901330F880B990B0E940DB820E082
:106A800030E048EC52E40E9466BA2B013C01CE0192
:106A900001960E94BE336C969FAF8EAF6C9760E5F7
:106AA00070E18FE19DE00E94B06969966CAD7DADAB
:106AB0008EAD9FAD69970E94D97E6AE470E18FE147
:106AC0009DE00E94B069C301B2010E94D97E64E4D6
:106AD00070E18FE19DE00E94B069612F70E08FE16D
:106AE0009DE00E94EF7D65960EAD1FAD6597011587
:106AF000110509F497C00E943785BB27A92F982F4D
:106B0000872F0097A105B10521F481E090E0A0E076
:106B1000B0E09C01AD0144275527B80190E080E02A
:106B2000AA24AA94BA2CC12CD12C17E2E12E19E088
:106B3000F12E00E010E00E94DD22882321F1F10116
:106B40006081718187E79CE00E944A6964E370E19B
:106B500087E79CE00E94B069F1016081718189E35F
:106B600094E00E94208665961FAE1EAE65976596DE
:106B70004CAD5DAD6EAD7FAD6597CE0101960E94C7
:106B8000CF1D60E02CC020E030E048E152E4C301BA
:106B9000B2010E940EBB18163CF4F10160817181B4
:106BA00085E494E00E9420866C962EAD3FAD6C97F4
:106BB000232B39F320E030E040E85FE369966CADC9
:106BC0007DAD8EAD9FAD69970E94F9B99B01AC0177
:106BD000C301B2010E9406B887FF0CC061E0C40186
:106BE0000E94A618CE0101960E94810F6A961FADE1
:106BF0006A9701CFA301920169966CAD7DAD8EAD10
:106C00009FAD69970E9406B818160CF0BACF65E2DE
:106C100070E18FE19DE00E94B0698FE19DE00E94EC
:106C2000A768E0CF6BE170E18FE19DE00E94B06961
:106C3000D9CF809180098150809380090E94378547
:106C400060931D0870931E0880931F08909320087E
:106C50000E94BF0C4B015C010E9437852B013C0157
:106C60000E94817D882309F466C080910E098111FC
:106C700062C030E020E041E050E060E4CE010196E7
:106C80000E94382340E450E068EE73E1CE010196A3
:106C90000E94BFB068E174E0CE0101960E941EBE62
:106CA00040E450E06AEF7FE0CE0101960E94BFB061
:106CB000B501A401CE018F5B9F4F0E942A0CBE013B
:106CC0006F5B7F4FCE0101960E94058630E020E089
:106CD00041E050E060E4CE0101960E94382340E498
:106CE00050E068EE73E1CE0101960E94BFB068E10A
:106CF00074E0CE0101960E941EBE40E450E063EFB6
:106D00007FE0CE0101960E94BFB0C301B20128EE20
:106D100033E040E050E00E9450B9BA01A901CE0131
:106D20008F5B9F4F0E942A0CBE016F5B7F4FCE018D
:106D300001960E9405861123C1F165E170E18FE1A2
:106D40009DE00E94B0690E94BF0CAB01BC012AE02B
:106D50008FE19DE00E945B686DE070E18FE19DE056
:106D60000E94B06960918009062E000C770B8FE1BC
:106D70009DE00E94EF7DC55ADF4F0FB6F894DEBF4D
:106D80000FBECDBFDF91CF911F910F91FF90EF907C
:106D9000DF90CF90BF90AF909F908F907F906F903B
:106DA0005F904F903F902F9008956BE070E18FE1DE
:106DB0009DE00E94B0690E94BF0CAB01BC012AE0BB
:106DC0008FE19DE00E945B6863E070E1C7CF2F9286
:106DD0003F924F925F926F927F928F929F92AF926B
:106DE000BF92CF92DF92EF92FF920F931F93CF93B8
:106DF000DF93CDB7DEB7CE5BD1090FB6F894DEBF17
:106E00000FBECDBF5C01CF54DF4F0883C15BD040C4
:106E1000CE54DF4F1883C25BD040822FCD54DF4F5A
:106E20002883C35BD040CC54DF4F3883C45BD04051
:106E3000CB54DF4F4883C55BD040CA54DF4F5883E3
:106E4000C65BD040C954DF4F6883C75BD040C8548D
:106E5000DF4F7883C85BD040C754DF4FF982E882A8
:106E6000C95BD0402C2C8F70682E712C4090820909
:106E700050908309EE2DFF2D309721F080818111F4
:106E80000C94DB41D5011B968C91882341F0C50100
:106E90000B96C754DF4F99838883C95BD040611438
:106EA000710411F00C94ED41C754DF4FE881F98172
:106EB000C95BD040309711F00C94DE41F501658834
:106EC00076886114710411F40C94ED41CD54DF4FB8
:106ED0008881C35BD0408F7011F00C94ED41662D1A
:106EE000CE018F549F4F0E94500DCF55DF4F288306
:106EF000C15AD040CE55DF4F3883C25AD040CD550D
:106F0000DF4F4883C35AD040CC55DF4F5883C45A13
:106F1000D040CB55DF4F6883C55AD040CA55DF4FAC
:106F20007883C65AD040C955DF4F8883C75AD040AE
:106F3000C855DF4F9883C85AD0400C94ED41CE011C
:106F40008F549F4F0E942827F501808191810097DF
:106F500011F40C943042FDE06F16710409F0B1C0D9
:106F60000E94427E082F10E006301105B4F40E9402
:106F70001571FC01892B41F08085807F82608087BC
:106F80001186128613861486BF01D5018D919C91BE
:106F90000E947E7E0F5F1F4FE7CF65E0F501808185
:106FA00091810E94E27D8C01892BE9F410E000E0E0
:106FB000C801C254DF4F0FB6F894DEBF0FBECDBF7D
:106FC000DF91CF911F910F91FF90EF90DF90CF90C5
:106FD000BF90AF909F908F907F906F905F904F90F9
:106FE0003F902F900895CF54DF4F8881C15BD040F0
:106FF0008031E0F6CE018F549F4F0E94C70E1616C7
:107000001706180619060CF04EC00E9437856B0152
:107010007C01CE018F549F4F0E94C70EC60ED71E13
:10702000E81EF91ED8011996CD92DD92ED92FC92E0
:107030001C97CF54DF4F8881C15BD040982F929529
:10704000907F18968C9118978F70892B18968C9337
:107050006DE677E08FE19DE00E94B069CE018F542C
:107060009F4F0E94C70EAB01BC012AE030E08FE1C8
:107070009DE00E94C46867E677E08FE19DE00E9492
:10708000B069F80141855285638574852AE030E056
:107090008FE19DE00E94C4688FE19DE00E94A76897
:1070A00001E010E085CFD80118968C9118978F7069
:1070B00018968C936EE577E08FE19DE00E94B069B1
:1070C000EBCFC5010E94BE334C01CC24C3941816EB
:1070D00019060CF0C12C8FE19DE00E94A768F50114
:1070E0003084F7E03F1609F492C0C754DF4F08819F
:1070F0001981C95BD0400115110509F449C06CE63E
:1071000078E0C8010E94A6B0892B09F444C068E663
:1071100078E0C8010E94A6B0892B09F45DC063E93C
:1071200076E0C8010E94A6B0892B09F458C06FE828
:1071300076E0C8010E94A6B0892B09F453C06DE225
:1071400078E0C8010E94A6B0892B09F44EC068E21D
:1071500078E0C8010E94A6B0892B09F449C062E317
:1071600078E0C8010E94A6B0892B09F444C066E803
:1071700076E0C8010E94A6B0892B09F43FC062E8FE
:1071800076E0C8010E94A6B00EE010E0892B29F03D
:1071900010E000E002C001E010E0C5010E94991873
:1071A000E82EF12CE114F10411F4EC2CF12C011572
:1071B000110569F1E016F10621F168E477E08FE14D
:1071C0009DE00E94B069B7018FE19DE00E94EF7DD4
:1071D0008FE19DE00C942E4202E010E0DECF05E04E
:1071E00010E0DBCF06E010E0D8CF0AE010E0D5CF0A
:1071F0000BE010E0D2CF0CE010E0CFCF0DE010E0BC
:10720000CCCFC754DF4F19821882C95BD040C75416
:10721000DF4F48815981C95BD0404115510509F4C0
:1072200053C027E0321218C0222009F439CFD5010B
:107230001296ED91FC9190859F70953009F030CFBA
:10724000B5E04B16510409F42BCFBE016F547F4FAC
:10725000CF010E94FE3224CFF501818592850097EF
:1072600009F4A4CEDC01ED91FC910488F589E02DB0
:107270007A01CF54DF4F0881C15BD040CE54DF4F3D
:107280001881C25BD040CD54DF4F2881C35BD04012
:10729000CC54DF4F3881C45BD040CB54DF4F4881A2
:1072A000C55BD040CA54DF4F5881C65BD040C9543B
:1072B000DF4F6881C75BD040C854DF4F7881C85B1F
:1072C000D04019958C0174CEC755DF4F18821982B2
:1072D0001A821B82C95AD040C355DF4F18821982C7
:1072E0001A821B82CD5AD040C555DF4F8881CB5AB8
:1072F000D0408F70C555DF4F8883CB5AD04040E0D7
:10730000B501CE0187559F4F0E94C62F811164C0E1
:107310006BE277E08FE19DE00E94B069F501818525
:107320009285009779F1DC01ED91FC91028CF38D4F
:10733000E02D19958D30910540F583569D4FDC0168
:107340008C918F70282F2295207FC555DF4F988113
:10735000CB5AD0409F70922BC555DF4F9883CB5AA4
:10736000D0408430A0F4823008F062C0813009F44B
:1073700075C0C355DF4F188219821A821B82CD5AFD
:10738000D0401AC0808590E0D5CF80E0DACF883039
:1073900039F0893071F780E090E0A6E9B2E404C0EA
:1073A00080E090E0A0EAB1E4C355DF4F8883998381
:1073B000AA83BB83CD5AD040B501CE0187559F4FDC
:1073C0000E94F77DCE0187559F4F0E94282760E0DD
:1073D0007AE0C5010E946730CF54DF4F6881C15BFE
:1073E000D040643009F4ABC008F03FC0662309F414
:1073F00041C3633009F439C1CE0187559F4F0E94C4
:10740000770D29A73AA74BA75CA76DA77EA78FA7E3
:1074100098AB662DCE0187559F4F0E94500D29A332
:107420003AA34BA35CA36DA37EA38FA398A7EBC045
:1074300084E6C155DF4F8883CF5AD040C055DF4F17
:107440008881C05BD0408E7FC055DF4F8883C05B92
:10745000D040C255DF4F1882CE5AD0408FEFC3556F
:10746000DF4F8883CD5AD040A7CF673009F46FC172
:1074700018F26A3008F660E0CE0187559F4F0E94EF
:10748000770DAA962FAFAA97AB963FAFAB97AC9666
:107490004FAFAC97AD965FAFAD97AE966FAFAE976F
:1074A000AF967FAFAF97E0968FAFE097E1969FAF33
:1074B000E197CD54DF4F8881C35BD040807F09F4D2
:1074C00093C1CE018F549F4F0E94C70E8B01672B33
:1074D00009F48AC1CF54DF4F8881C15BD040893025
:1074E00019F4119501951109F2E06F16710409F470
:1074F000C8C10CF07CC16114710409F4C0C1F5016C
:10750000A185B285109709F40DC6CF54DF4F68816D
:10751000C15BD0406A3008F0ABC5E62FF0E08827A9
:10752000EB56F54C8F4F0C94DBB9FA3F3240A63F37
:1075300038403840463FCC3E3840FA3FFA3F1814B6
:1075400019040CF063C062E0CE0187559F4F0E9482
:10755000770DC756DF4F2883C959D040C656DF4F35
:107560003883CA59D040C556DF4F4883CB59D040E5
:10757000C456DF4F5883CC59D040C356DF4F688381
:10758000CD59D040C256DF4F7883CE59D040C15636
:10759000DF4F8883CF59D040C056DF4F9883C05A01
:1075A000D040C755DF4F6881C95AD040CE018F54B3
:1075B0009F4F0E94770DC757DF4F2883C958D0408F
:1075C000C657DF4F3883CA58D040C557DF4F48836E
:1075D000CB58D040C457DF4F5883CC58D040C35706
:1075E000DF4F6883CD58D040C257DF4F7883CE58E5
:1075F000D040C157DF4F8883CF58D040C057DF4FAE
:107600009883C059D040CC24C39479CF61E0CE0197
:1076100087559F4F0E94770DCF56DF4F2883C15962
:10762000D040CE56DF4F3883C259D040CD56DF4FC1
:107630004883C359D040CC56DF4F5883C459D040FB
:10764000CB56DF4F6883C559D040CA56DF4F788389
:10765000C659D040C956DF4F8883C759D040C85655
:10766000DF4F9883C859D0409CCFF5018085873083
:1076700009F445CFC5010E949918853009F0B1C0C1
:107680006CE177E08FE19DE00E94B06965E070E019
:107690008FE19DE00E94EF7D8FE19DE00E94A76851
:1076A000D50118968C91853079F56CE0CE0187551F
:1076B0009F4F0E94770DCF57DF4F2883C158D0408E
:1076C000CE57DF4F3883C258D040CD57DF4F488365
:1076D000C358D040CC57DF4F5883C458D040CB5705
:1076E000DF4F6883C558D040CA57DF4F7883C658EC
:1076F000D040C957DF4F8883C758D040C857DF4FA5
:107700009883C858D0407FCF61E0CE0187559F4F06
:107710000E94770DEA962FAFEA97EB963FAFEB9773
:10772000EC964FAFEC97ED965FAFED97EE966FAF9F
:10773000EE97EF967FAFEF97C158DF4F8883CF5713
:10774000D040C058DF4F9883C058D0405CCFF5017F
:107750008085873009F4D3CEC5010E949918182F6F
:10776000863079F56BE077E08FE19DE00E94B069AB
:1077700066E070E08FE19DE00E94EF7D8FE19DE08B
:107780000E94A76862E0CE0187559F4F0E94770D47
:10779000E2962FAFE297E3963FAFE397E4964FAFC1
:1077A000E497E5965FAFE597E6966FAFE697E796C5
:1077B0007FAFE797E8968FAFE897E9969FAFE99795
:1077C00022CF63EF76E08FE19DE00E94B069612FE8
:1077D00070E08FE19DE00E94EF7D8FE19DE00E94CF
:1077E000A7680DEF1FEFE4CB05E010E073CE89E052
:1077F0006816710409F4EBC0AAE06A16710409F076
:107800007ECEC555DF4F8881CB5AD04082958F7090
:10781000823009F074CEC255DF4F6881CE5AD04015
:10782000060F111D17FF02C010E000E0053611051C
:1078300014F004E610E0C255DF4F0883CE5AD04062
:1078400062E0CE0187559F4F0E94500D6A962FAF80
:107850006A976B963FAF6B976C964FAF6C976D9630
:107860005FAF6D976E966FAF6E976F967FAF6F97A6
:10787000A0968FAFA097A1969FAFA19735C0CC24BB
:10788000C394C555DF4FE881CB5AD040E295EF70E5
:10789000E150EB3008F033CEF0E08827ED5AF34C9E
:1078A0008F4F0C94DBB95E3C5E3C7F3A7F3A7F3A67
:1078B000C23C9E3C9E3C9E3C803C803CC355DF4F7E
:1078C0006881CD5AD040060F111D17FF02C010E08D
:1078D00000E00F3F110519F014F00FEF10E0C35551
:1078E000DF4F0883CD5AD040B501CE0187559F4F59
:1078F0000E94F77D60E07AE0C5010E946730FFCD0D
:10790000C355DF4F68817981CD5AD040060F171FCC
:1079100017FF02C010E000E00536110514F004E680
:1079200010E0012E000C220B330BC355DF4F0883F0
:1079300019832A833B83CD5AD040D6CFC355DF4F1E
:10794000688179818A819B81CD5AD0400E94D8BAC2
:10795000600F711F77FF02C070E060E0653671054F
:1079600014F064E670E0072E000C880B990B0E945F
:107970000DB8C355DF4F688379838A839B83CD5AC3
:10798000D040B2CFC355DF4F28813981CD5AD04086
:107990004AE0409FC001419F900D1124820F931F28
:1079A00097FF02C090E080E0893EB3E09B0714F0AF
:1079B00088EE93E0092E000CAA0BBB0BC355DF4FDA
:1079C00088839983AA83BB83CD5AD0408DCFC55578
:1079D000DF4F8881CB5AD04082958F70823009F07A
:1079E0008ECDC155DF4F6881CF5AD040C055DF4F93
:1079F0008881C05BD040782F7170060F171F0E363C
:107A0000E1E01E072CF417FF05C00DE611E002C0EF
:107A100010E000E0C155DF4F0883CF5AD040C05579
:107A2000DF4F8881C05BD04010FB80F9C055DF4F2D
:107A30008883C05BD04062E0CE0187559F4F0E9493
:107A4000500DA2962FAFA297A3963FAFA397A496EF
:107A50004FAFA497A5965FAFA597A6966FAFA697D1
:107A6000A7967FAFA797A8968FAFA897A9969FAF25
:107A7000A9973ACFCD54DF4F8881C35BD040807F38
:107A800009F43DCDF9E06F16710409F457C10CF00B
:107A9000C4C06114710409F4D8C0312C82E06816A6
:107AA000710409F02CCDC555DF4F8881CB5AD040E9
:107AB000982F92959F70945F9F70923080F4CD5470
:107AC000DF4F9881C35BD04092959F70923039F41C
:107AD0008F708062C555DF4F8883CB5AD040D50167
:107AE00018969C919730B1F4CD54DF4F8881C35BD9
:107AF000D040807E803211F0803461F4C555DF4F74
:107B00008881CB5AD0408F708062C555DF4F888303
:107B1000CB5AD040F501A185B285892F90E010970E
:107B200041F0ED91FC911197028CF38DE02DCD0188
:107B300019957C01CF54DF4F0881C15BD040CE54F2
:107B4000DF4F1881C25BD040CD54DF4F2881C35B2B
:107B5000D040CC54DF4F3881C45BD040CB54DF4F92
:107B60004881C55BD040CA54DF4F5881C65BD040C6
:107B7000C954DF4F6881C75BD040C854DF4F78815C
:107B8000C85BD040CE0187559F4F0E947227229636
:107B90002FAF229723963FAF239724964FAF24977A
:107BA00025965FAF259726966FAF269727967FAFCE
:107BB000279728968FAF289729969FAF299733202C
:107BC00009F492CEC555DF4F8881CB5AD0408295BB
:107BD0008F708150823008F087CEC355DF4F2881E7
:107BE000CD5AD04030E0AFEFB0E00E94A4B924E617
:107BF00030E040E050E00E9472B92F3F310541056E
:107C0000510529F024F02FEF30E040E050E0C3555B
:107C1000DF4F2883CD5AD04067CEABE06A1671049F
:107C200009F4AEC00CF454C0ECE06E16710409F017
:107C300066CC88E0FE01EF54FF4FDE01A755BF4F31
:107C400001900D928A95E1F75ACCCE018F549F4F47
:107C50000E94C70E181419040CF089C3672B682BF7
:107C6000692BF1F462E0CE0187559F4F0E94770D9A
:107C700062962FAF629763963FAF639764964FAF5C
:107C8000649765965FAF659766966FAF66976796E0
:107C90007FAF679768968FAF689769969FAF699730
:107CA000C755DF4F6881C95AD040C5010E949D1752
:107CB000B501CE0187559F4F0E94F77D60E079E0C6
:107CC000C5010E94673033243394CC24C394EBCE97
:107CD000CA54DF4F9881C65BD040C555DF4F8881BD
:107CE000CB5AD040282F22952F7001F1223009F075
:107CF00006CC892F90E08536910514F084E690E05B
:107D0000C255DF4F8883CE5AD04062E0CE018755FE
:107D10009F4F0E94500D29AF3AAF4BAF5CAF6DAF94
:107D20007EAF8FAF21969FAF2197DECD8F7080629F
:107D3000C555DF4F8883CB5AD040DBCFC954DF4FC6
:107D40006881C75BD040C854DF4F7881C85BD040A2
:107D50007170CE0187559F4F0E94620F882309F4EE
:107D6000CECB62E0CE0187559F4F0E94500D29ABCC
:107D70003AAB4BAB5CAB6DAB7EAB8FAB98AFB4CDDE
:107D8000CE018F549F4F0E940C0FBC01CE0187552E
:107D90009F4F0E942E0FA8CD181419040CF46FC029
:107DA00066EE76E08FE19DE00E94B06961E0CE0171
:107DB00087559F4F0E94770D298F3A8F4B8F5C8F8D
:107DC0006D8F7E8F8F8F98A3D50119968D919C9181
:107DD000C754DF4FE880F980C95BD040DC01ED91EA
:107DE000FC910488F589E02DCC24C394C755DF4F5E
:107DF0000881C95AD040C655DF4F1881CA5AD040B1
:107E0000C555DF4F2881CB5AD040C455DF4F38814C
:107E1000CC5AD040C355DF4F4881CD5AD040C255CF
:107E2000DF4F5881CE5AD040C155DF4F6881CF5ABD
:107E3000D040C055DF4F7881C05BD04019958C0190
:107E400066E0C5010E949D17B501CE0187559F4F81
:107E50000E94F77D60E071E0C5010E94673068EA2A
:107E600076E08FE19DE00E94B069B8018FE19DE06E
:107E70000E94EF7D8FE19DE00E94A76899C866EDA2
:107E800076E08FE19DE00E94B069ABCC1814190434
:107E90000CF059C062E0CE0187559F4F0E94770DCC
:107EA000298B3A8B4B8B5C8B6D8B7E8B8F8B988F5A
:107EB000F50181859285C754DF4FE880F980C95B61
:107EC000D040DC01ED91FC910488F589E02DCC24B3
:107ED000C394C755DF4F0881C95AD040C655DF4FFC
:107EE0001881CA5AD040C555DF4F2881CB5AD0409F
:107EF000C455DF4F3881CC5AD040C355DF4F48813D
:107F0000CD5AD040C255DF4F5881CE5AD040C155CE
:107F1000DF4F6881CF5AD040C055DF4F7881C05BBA
:107F2000D04019958C0165E0C5010E949D17B501EF
:107F3000CE0187559F4F0E94F77D60E071E0C5013B
:107F40000E94673035C864EC76E09BCFC5010E9483
:107F50009918853009F44BC062E0CE0187559F4FD8
:107F60000E94770D29873A874B875C876D877E87CC
:107F70008F87988BF50181859285C754DF4FE88004
:107F8000F980C95BD040DC01ED91FC910488F58952
:107F9000E02DCC24C394C755DF4F0881C95AD04087
:107FA000C655DF4F1881CA5AD040C555DF4F2881CA
:107FB000CB5AD040C455DF4F3881CC5AD040C3553E
:107FC000DF4F4881CD5AD040C255DF4F5881CE5A3D
:107FD000D040C155DF4F6881CF5AD040C055DF4FE8
:107FE0007881C05BD04019958C0162E02ACF64EBA8
:107FF00076E047CFC754DF4FE880F980C95BD040B7
:10800000ED91FC9111970488F589E02DC755DF4F5C
:108010000881C95AD040C655DF4F1881CA5AD0408E
:10802000C555DF4F2881CB5AD040C455DF4F38812A
:10803000CC5AD040C355DF4F4881CD5AD040C255AD
:10804000DF4F5881CE5AD040C155DF4F6881CF5A9B
:10805000D040C055DF4F7881C05BD040CD0119952D
:108060008C01FDCE0FEF1FEF181419040CF4F7CE9E
:10807000CE0187559F4F0E94770D29833A834B830A
:108080005C836D837E838F839887F50181859285DC
:10809000C754DF4FE880F980C95BD040DC01ED9127
:1080A000FC910488F589E02DCC24C394C755DF4F9B
:1080B0000881C95AD040C655DF4F1881CA5AD040EE
:1080C000C555DF4F2881CB5AD040C455DF4F38818A
:1080D000CC5AD040C355DF4F4881CD5AD040C2550D
:1080E000DF4F5881CE5AD040C155DF4F6881CF5AFB
:1080F000D040C055DF4F7881C05BD04019958C01CE
:10810000B501CE0187559F4F0E94F77DC755DF4FC0
:108110006881C95AD040662309F4A1CEC5010E94E6
:108120009D1798CE8085863009F4B1C0873009F458
:108130006EC0853009F084C0B2E06B16710409F49A
:1081400007C1ECE06E16710409F07AC0C5010E9407
:108150007C16892B49F4D501ED91FC9160817181E8
:1081600082E594E00E942086CE0187559F4F0E94B1
:10817000800E20E030E048EC52E40E946CB80E948F
:10818000D8BAC554DF4F688379838A839B83CB5BDE
:10819000D040C554DF4F48805980CB5BD0400E940F
:1081A0003785C72ED82EE92EFF24C114D104E1044F
:1081B000F10421F4C12CD12C7601C3946DE976E051
:1081C0008FE19DE00E94B069C554DF4F68817981DD
:1081D000CB5BD0408FE19DE00E94EF7D68E976E0C7
:1081E0008FE19DE00E94B069B701A601662777275D
:1081F0002AE08FE19DE00E945B688FE19DE00E9494
:10820000A768B601A201C5010E94CF1D19C0222096
:10821000B9F00280F381E02D90859F70953081F454
:10822000B5E04B16510461F0C754DF4F48815981C6
:10823000C95BD040BE016F547F4FCF010E94FE3218
:10824000C755DF4F6881C95AD040662311F40C949A
:108250005038CF54DF4F8881C15BD040853009F062
:108260007EC01814190414F00C94503865E0C50150
:108270000E949D17B501CE018F549F4F0E94F77D3C
:1082800060E071E0C5010E9467300C94503870E0E6
:1082900060E0C5010E9498168C01009789F2712C4C
:1082A000612C97FF06C0119501951109662463940E
:1082B000712CC80101978635910510F6C755DF4F1F
:1082C000E880C95AD040F12CD02E61E0802F0E9466
:1082D0007283672851F1E1E0EE16F10429F061E0C4
:1082E000F6E0EF16F10409F460E0E62EF12C8D2D96
:1082F0000E94448363EA76E08FE19DE00E94B069CA
:10830000B8018FE19DE00E94EF7D61EA76E08FE1A8
:108310009DE00E94B069B7018FE19DE00E94EF7D72
:108320008FE19DE00E94A7688BCF21E0E216F10467
:1083300059F091E080E0A6E0EA16F10409F090E03F
:10834000E92EF82E6E2DD3CFEE24E394F12CFACF44
:10835000B501CE0187559F4F0E94F77D71CFC501B2
:108360000E949D17B501CE0187559F4F87CF672B80
:10837000682B692B09F494CC61E0CE0187559F4F9F
:108380000E94770D2A962FAF2A972B963FAF2B97F7
:108390002C964FAF2C972D965FAF2D972E966FAFE3
:1083A0002E972F967FAF2F9760968FAF609761962D
:1083B0009FAF619775CC6114710479F48081882333
:1083C00011F40C945E37CE0187549F4F0E942D1EEE
:1083D0003C01892B11F40C945E370E94BF0C6B0199
:1083E0008B0169E977E08FE19DE00E94B069B601F9
:1083F0008FE19DE00E94EF7D62E977E08FE19DE0F3
:108400000E94B069D501ED91FC91608171818FE18D
:108410009DE00E944A696CE877E08FE19DE00E9450
:10842000B069C754DF4F68817981C95BD0408FE163
:108430009DE00E944A6966E877E08FE19DE00E9436
:10844000B069083C110514F00C949F3768E777E099
:1084500087E79CE00E94B06987E79CE00E94A768DC
:108460000FEF1FEF0C94D8372F923F924F925F92ED
:108470006F927F928F929F92AF92BF92CF92DF9234
:10848000EF92FF920F931F93CF93DF93CDB7DEB799
:10849000A5970FB6F894DEBF0FBECDBF5C0179A3E0
:1084A00068A370901008772009F4B7C08091800904
:1084B0008F5F80938009E0918409F091850930975E
:1084C00009F4A3C086809780409084095090850964
:1084D0004114510409F495C08114910409F491C028
:1084E000D40118968C918F70853091F7C4010E9449
:1084F000427E823068F3B401CE0101960E94E832D8
:10850000CE0101960E94BA2F882309F45DC060E075
:1085100074E0CE0101960E948717892B09F454C09C
:10852000188E198E1A8E1B8E1C8E1D8E1E8E1F8EFF
:108530008A8D8F708A8F41E0BE016F5F7F4FCE01C1
:1085400048960E94C62F66EE77E08FE19DE00E947C
:10855000B06960E074E0CE0101960E9419178A8527
:108560009B85009789F1DC01ED91FC910488F589E8
:10857000E02DCC24C394F12CE12C088D198D2A8D8B
:108580003B8D4C8D5D8D6E8D7F8D19958F3F98073E
:10859000D9F0E981FA8160817181892BE9F48FE159
:1085A0009DE00E944A6964EE77E08FE19DE00E94C1
:1085B000B0696CED77E08FE19DE00E94B0698FE1DA
:1085C0009DE00E94A768712CF40182809380CE0107
:1085D00001960E94810F78CF8FE19DE00E944A6949
:1085E0006AED77E08FE19DE00E94B06966ED77E08B
:1085F0008FE19DE00E94B0698FE19DE00E94A76835
:10860000E3CF8FE19DE00E94A768809180098150AF
:108610008093800971101092100865E0D5018D914A
:108620009C910E94E27D1C01009709F48FC0FC011F
:108630008084859485948594859441845284638450
:1086400074840E943785882009F480C0461A570A2E
:10865000680A790A188E198E1A8E1B8E888E8A8D5A
:108660008F70806A982E8A8F4C8E5D8E6E8E7F8E74
:10867000C301B20128EE33E040E050E00E9472B93D
:108680002AA33BA34CA35DA3672B682B692B21F581
:10869000D12CC12CE12C90E1F92E082D198D292D1A
:1086A0003B8D4C8D5D8D6E8D7F8DC5010E945E2D45
:1086B0002AE030E04AA15BA16CA17DA18FE19DE0A1
:1086C0000E94C4686BEF77E08FE19DE00E94B06983
:1086D0008FE19DE00E94A76877FE38C0F2E04F1658
:1086E00051046104F0E87F068CF1D12CC12CE12CFF
:1086F00080E1F82E088D198D2A8D3B8D4C8D5D8D76
:108700006E8D7F8DC5010E945E2D19821A821B829B
:108710001C821D821E821F8218862B812F702B8344
:108720008982CC24C394F12CE12C082D1A813C8140
:1087300040E05E816F817885C5010E94E736D101F6
:1087400018968C9118978F7018968C93E8A1F9A1C0
:108750003197B9F460E073E0C5010E948717009774
:1087600081F020918209309183092630310549F446
:10877000BC01C5010E94673060E073E0C5010E9442
:108780001917D50119968D919C910097D9F490E015
:1087900080E0A5960FB6F894DEBF0FBECDBFDF9187
:1087A000CF911F910F91FF90EF90DF90CF90BF90EE
:1087B000AF909F908F907F906F905F904F903F9081
:1087C0002F900895DC01ED91FC910484F585E02D56
:1087D0001995892BE1F2F50181859285DC01ED91F6
:1087E000FC910480F581E02D68A179A11995D1CF84
:1087F000AF92BF92CF92DF92EF92FF920F931F93AF
:10880000CF93DF93CDB7DEB767970FB6F894DEBF8F
:108810000FBECDBFE0918409F0918509309709F42E
:108820009EC0809180098F5F8093800906811781A7
:10883000E0908409F0908509E114F10431F101150B
:10884000110519F1F80180858F708530A9F7C801ED
:108850000E94427E823080F3B801CE0101960E94D0
:10886000E832CE0101960E94BA2F882331F062E0EF
:1088700070E0CE0101960E943442F801028113811A
:10888000CE0101960E94810FD3CF80918009815043
:10889000809380098091820990918309059709F45A
:1088A0005EC00E9437859B01AC01609119087091F0
:1088B0001A0880911B0890911C08AA24AA94BA2C2B
:1088C000650118EEE12E13E0F12E00E010E00E94A9
:1088D000DD22082F882309F442C010E060912508AA
:1088E0007091260861157105D1F1111138C0FB0195
:1088F00080858F708530D9F4CE0101960E94E832D0
:1089000061E070E0CE0101960E943442892B59F05B
:108910000E9437856093190870931A0880931B088A
:1089200090931C08102FCE0101960E94810FE091B8
:108930002508F0912608309791F0828193819093D9
:10894000260880932508892B49F6E0918409F09147
:1089500085098681978190932608809325086796DC
:108960000FB6F894DEBF0FBECDBFDF91CF911F9140
:108970000F91FF90EF90DF90CF90BF90AF90089550
:108980006F927F929F92AF92BF92CF92DF92EF92BF
:10899000FF920F931F93CF93DF93CDB7DEB7E2978C
:1089A0000FB6F894DEBF0FBECDBF78AB6FA75AAB42
:1089B00049AB672B09F48FC2FA01309719F0208177
:1089C000211109C0FC012385222329F09C01255F88
:1089D0003F4F3AAB29AB5C01E9A9FAA93097E1F422
:1089E000F501E588F688E114F10401F510E000E0F6
:1089F000CFA4D8A83601600E711EF30180818823B0
:108A000009F458C0082E000C990B0E94C1BDF30157
:108A100080830F5F1F4FECCF8081882309F3CE0145
:108A2000C1960E942D1E7C01892BD1F2FEE0EF162B
:108A3000F104E1F62FA538A919821A821B821C8243
:108A40001D821E821F8218868B818F70806C8B83A3
:108A50003E832D836EE0CE0101960E94500D29A326
:108A60003AA34BA35CA36DA37EA38FA398A7E9A809
:108A7000FAA8CC24C39409811A812B813C814D81B1
:108A80005E816F817885C5010E94E736E2960FB658
:108A9000F894DEBF0FBECDBFDF91CF911F910F9134
:108AA000FF90EF90DF90CF90BF90AF909F907F901E
:108AB0006F900895C114D10481F1F601808188235B
:108AC00061F18D3209F47CC090ED980F9A3008F472
:108AD00077C008E010E0853211F10EEF1FEF8B3701
:108AE000F1F007E110E08332D1F092E3692E99E0D2
:108AF000792E01E010E0C3010E94B6B0AC01B301D1
:108B0000C6010E94CFB0892B51F00F5F1F4FF9E0D3
:108B10006F0E711C0931110571F70FEF1FEF69E737
:108B200076E08FE19DE00E94B069B8018FE19DE0A1
:108B30000E94EF7D8FE19DE00E94A76819A21AA212
:108B40001BA21CA21DA21EA21FA218A68BA18F7081
:108B50008BA309A385E0E816F104A9F1E6E0EE167F
:108B6000F10411F407E110E09E2C6E2DCE018196E8
:108B70000E94500D298F3A8F4B8F5C8F6D8F7E8FA7
:108B80008F8F98A301151105A9F104F50E3F1F4F12
:108B90000CF0A1C1CE018F960E948F13092E000CFC
:108BA000AA0BBB0B0097A105B10509F4D2C02BA1FC
:108BB0002F70206A2BA38DA39EA3AFA3B8A7C9C013
:108BC00010E000E0ACCF08E110E0CECF0731110596
:108BD00009F43DC108311105E9F660E0CE01819646
:108BE0000E94770D298B3A8B4B8B5C8B6D8B7E8B28
:108BF0008F8B988F19821A821B821C828B818F70B7
:108C000080668B83EFA5F8A9309709F48AC080812C
:108C1000882309F486C06FA478A8F3018081882393
:108C200059F08D3249F080538A3030F0FFEF6F1ADF
:108C30007F0A78AA6FA6EFCFC3010E9458B06C01DB
:108C40006EE270E0C3010E9429BE009771F0FC0142
:108C50000181002E000C110B005311090A3011057F
:108C600014F009E010E017FF02C010E000E06CE231
:108C700070E0C3010E9429BE009709F045C018AA00
:108C80001FA60115110509F443C02AE02C9DC0015F
:108C90002D9D900D11241C141D041CF0119501959F
:108CA0001109080F191F012E000C220B330B0D8325
:108CB0001E832F833887692DCE0101960E94500DA7
:108CC00029873A874B875C876D877E878F87988B4C
:108CD000DB80D2948FE0D8223E01F9E26F0E711C46
:108CE00010E000E08FA598A9892BF9F00330110559
:108CF000E1F00F5F1F4FCE018F960E948F13F3019B
:108D0000819391933F01EECF019698AB8FA7B9CF96
:108D10008601DD0C220B330B8B818F70806A8B8375
:108D2000C6CF00E010E09801C2CFFAE0EF16F104E0
:108D3000E9F08BE0E816F10469F1E9E0EE16F104E0
:108D400091F5CE0101960E94C70ECE0181960E9438
:108D5000620FE9A8FAA8CC24C39409A11AA12BA1F7
:108D60003CA14DA15EA16FA178A58DCECE0101964B
:108D70000E94C70E8BA1982F92959F7039F0923068
:108D800041F7653608F064E66EA3E3CF8F7080622A
:108D90008BA3F7CFCE0101960E94C70ECE0181961C
:108DA0000E942E0FD6CF81E090E0D11002C090E05B
:108DB00080E0800F911F8230910539F164F40197B2
:108DC00041F688E0FE013196DE01919601900D9208
:108DD0008A95E1F7BECF8330910539F1049709F008
:108DE000B8CF1BA509A5CE0101960E94C70E8BA185
:108DF0008F7080628BA36FA388A570FB80F988A712
:108E00000EA31DA36DA57EA5C9CF19A5CE01019600
:108E10000E94C70E8BA18F7080638BA36FA388A560
:108E200070FB80F988A71EA394CF1BA509A5CE01CE
:108E300001960E94C70E8BA18F7080628BA36FA3D7
:108E400088A570FB80F988A70EA31DA382CF60E0E0
:108E5000CE0181960E94770D29833A834B835C83F0
:108E60006D837E838F8398877E01F9E0EF0EF11C7E
:108E700010E000E08FA598A9892B71F0043011054E
:108E800091F00F5F1F4FCE018F960E948F13F70155
:108E9000819391937F01EECF0330110589F0043067
:108EA000110509F056CF9F852D853B8549858BA1FE
:108EB0008F7080658BA34FA33EA32DA398A749CFA6
:108EC0009D852B8539858BA18F7080648BA33FA3F3
:108ED0002EA39DA33ECF90E080E0D8CD8F929F92AD
:108EE000AF92BF92CF92DF92EF92FF920F931F93B8
:108EF000CF93DF93CDB7DEB7C855D1090FB6F8943D
:108F0000DEBF0FBECDBF6296EFAE62976396FFAE37
:108F1000639764960FAF649765961FAF65976696E3
:108F20002FAF669767963FAF679768964FAF689782
:108F300069965FAF6997009771F0D62E8C01FC019E
:108F400080858295807F85958595859585958530E9
:108F500021F0863091F180E052C0809180098F5FCE
:108F600080938009A680B780A114B10401F16296B4
:108F7000EFAC62976396FFAC639764960FAD64970E
:108F800065961FAD659766962FAD669767963FAD60
:108F9000679768964FAD689769965FAD69976D2D35
:108FA000C5010E946E47F501A280B380DDCF80919C
:108FB0008009815080938009CECF61E674E0C801BA
:108FC0000E94667D009779F16296EFAC6297639696
:108FD000FFAC639764960FAD649765961FAD659778
:108FE00066962FAD669767963FAD679768964FADCB
:108FF000689769965FAD69976D2D0E946E47C85A54
:10900000DF4F0FB6F894DEBF0FBECDBFDF91CF911B
:109010001F910F91FF90EF90DF90CF90BF90AF9096
:109020009F908F90089565E674E0C8010E94667D68
:109030004C016AE674E0C8010E94667D5C01DD2097
:10904000A9F0F1E0DF1609F47BC0F12CE12C00E07F
:1090500020E033E040E150E0BE016F5B7F4FCE0186
:109060008F5A9F4F0E943C198C0122C06FE674E01A
:10907000C8010E94667D7C0164E774E0C8010E941B
:10908000667D6C01E114F10409F47AC0F701808572
:109090008F70843009F074C0E184F284C114D1046B
:1090A000B1F2F60180858F70843089F601851285D2
:1090B0008114910409F491C0F401618572858FE1F6
:1090C0009DE0E114F10409F45EC00E944A6961EC7C
:1090D00072E18FE19DE00E94B069B7018FE19DE0F0
:1090E0000E944A698FE19DE00E94A768CE018F5AD5
:1090F0009F4F0E942827A114B10409F072C0F40107
:1091000080858F70843009F0B5C061857285CE018D
:1091100001960E945C32CE0101960E94BA2F8823EC
:1091200051F0E114F104C1F150E040E0B701CE018B
:1091300001960E94C044CE0101960E94810F9AC000
:1091400069E774E0C8010E94667D7C016EE774E007
:10915000C8010E94667D6C01E114F10409F08CC025
:109160006FE674E0C8010E94667D7C01C114D104E1
:1091700009F482CF892B09F089CFF12CE12C91CF12
:10918000F12CE12C8BCF0E944A696CEB72E18FE1EC
:109190009DE00E94B069AACFCC24C394F12CE12CAD
:1091A00062960FAD629763961FAD639764962FAD7D
:1091B000649765963FAD659766964FAD66976796DF
:1091C0005FAD679768966FAD689769967FAD699751
:1091D000CE0101960E94E736AECFA114B10409F486
:1091E00049C0F501618572858FE19DE00E944A6961
:1091F00067EB72E18FE19DE00E94B069B8018FE1F9
:109200009DE00E944A698FE19DE00E94A7680115D8
:10921000110561F1F50180858F70843039F5618524
:10922000728540E450E0CE0101960E9462BE0E9429
:10923000817D8823D9F080910E09811117C06FE2DA
:1092400070E0CE0101960E9429BE892B51F4F501F0
:109250002185328543E050E060E4CE0101960E9412
:109260003823B801CE0101960E940586811491042D
:1092700009F045CF81E0C3CE892B09F007CFFCCEA2
:109280002F923F924F925F926F927F928F929F9216
:10929000AF92BF92CF92DF92EF92FF920F931F9304
:1092A000CF93DF93CDB7DEB7E2970FB6F894DEBF6A
:1092B0000FBECDBF9AA389A3098F1A8F2B8F3C8F26
:1092C0004D8F5E8F6F8F78A3FAAAE9AADC011496FE
:1092D000ED91FC91309709F4DAC08680978018AA46
:1092E0001FA6312C212C512C412CB12CA12C712CDE
:1092F000612C8114910409F4D2C062EC73E0C401C2
:109300000E94667D9EA38DA365E774E0C4010E9460
:10931000667D9AA789A7EDA1FEA1309709F4AFC099
:10932000892B09F4ACC080858F70823009F0A7C00A
:10933000A9A5BAA518968C918F70823009F09FC0AC
:1093400063E874E0C4010E94667DDC0119962D91EA
:109350003D914D915C911C972BA73CA74DA75EA713
:10936000E9A9FAA9309709F45AC0D401CD90DC904C
:10937000BF01C6010E9434BE892B09F050C0098D7F
:10938000002309F1802F90E0B0E0A0E0E9A5FAA564
:1093900081879287A387B4878091820990918309FE
:1093A000059789F0E12CFF24F3941A8D2B8D3C8DC9
:1093B0004D8D5E8D6F8D78A1A9A1BAA112968D9168
:1093C0009C910E945E2D8B8D807F49F160E0CE01E3
:1093D00049960E94CE0D092E000CAA0BBB0BEDA1E5
:1093E000FEA181879287A387B4878091820990919B
:1093F00083090597A1F0D401CD90DC90E12C32E0F7
:10940000F32E098D1A8D2B8D3C8D4D8D5E8D6F8DBC
:1094100078A1E9A1FAA1828193810E945E2DADA17C
:10942000BEA119964D915D916D917C911C97E9A516
:10943000FAA581859285A385B4850297A105B1051A
:1094400019F12BA53CA5429FC001439F900D529F4F
:10945000900D1124680E791EABA5BCA5AA0EBB1EEB
:10946000EFA5F8A98F01FF0F220B330B0417150787
:109470002607370724F458AB4FA71C012D01D40150
:1094800012968D909C9035CF90E080E0E5CF312C06
:10949000212C512C412CB12CA12C712C612CA1140C
:1094A000B10409F482C0C301B5010E94C7B98B01A0
:1094B00069E472E18FE19DE00E94B069B5018FE13E
:1094C0009DE00E94EF7D6EE372E18FE19DE00E94DE
:1094D000B069EE24EA94F12CC301B7010E94C7B928
:1094E0008FE19DE00E94EF7D67E372E18FE19DE0F7
:1094F0000E94B069B8018FE19DE00E94EF7D69E2B2
:1095000072E18FE19DE00E94B069C101B7010E9444
:10951000C7B98FE19DE00E94EF7D62E272E18FE1C9
:109520009DE00E94B069B2018FE19DE00E94EF7D55
:109530006EE172E18FE19DE00E94B0698FE19DE0F4
:109540000E94A76819821A821B821C821D821E82B9
:109550001F8218868B818F708B83B801CE01019694
:109560000E94990D79018A015B016C01298BFA8AAD
:109570004B8B1C8B6D8BBE8A8F8BD88E68E575E00C
:10958000E9A1FAA1848195810E94667D9501A601D9
:109590006FEF0E946E47A9A1BAA11496ED91FC91BC
:1095A0003097E9F4AA24A394B12CC501E2960FB632
:1095B000F894DEBF0FBECDBFDF91CF911F910F9109
:1095C000FF90EF90DF90CF90BF90AF909F908F90E3
:1095D0007F906F905F904F903F902F900895C6803E
:1095E000D78088248A94912C9201550C440B550BFA
:1095F00029A33AA34BA35CA3C101032C000CAA0B23
:10960000BB0B8DA39EA3AFA3B8A7C114D10451F285
:1096100063E874E0C6010E94667D7C0166EC73E03D
:10962000C6010E94667D5C0162EC73E0C6010E9487
:10963000667D8C0165E774E0C6010E94667DA11419
:10964000B10409F4B0C00115110509F4ACC00097CC
:1096500009F4A9C0D50118962C912F70223009F079
:10966000A2C0F80120852F70223009F09CC0DC01D7
:1096700018962C9118972F70223009F094C0F7019A
:1096800041845284638474844114510409F48BC06E
:1096900019968D919D910D90BC91A02D0297A105D9
:1096A000B10509F484C02114310409F480C0D80143
:1096B00019968D919C91849D8001859D100D949D9E
:1096C000100D11242FEF30E0D8010E94F2B9920161
:1096D000550C440B550B0E9472B969A17AA18BA15C
:1096E0009CA10E9440B92DA13EA14FA158A50E9466
:1096F00072B929013A01F601608171818FE19DE023
:109700000E944A6965E874E08FE19DE00E944A6921
:10971000C801B4010E94C7B98FE19DE00E94EF7DAE
:1097200068E172E18FE19DE00E94B0692AE030E0DB
:10973000B301A2018FE19DE00E94C4688FE19DE02A
:109740000E94A768F50181859285A385B48584155B
:109750009505A605B70539F119861A861B861C865C
:109760001D861E861F86188A8B858F708B87B20197
:10977000CE0109960E94990D29833A834B835C831D
:109780006D837E838F83988779018A019B01AC0169
:109790006FEFC6010E946E47D50119964D925D92FA
:1097A0006D927C921C97F601C280D3802ECF412C03
:1097B000512C3201C7CFBF92CF92DF92EF92FF922E
:1097C0000F931F93CF93DF9300D000D01F921F926F
:1097D000CDB7DEB76C01B62EDC018D919C9111974F
:1097E000892B09F475C01496ED91FC91309709F41A
:1097F0006FC080818071BFEF6B1367C009F421C116
:10980000E181BE2EB2948FE0B8226CED75E08FE15D
:109810009DE00E94B0696B2D8FE19DE00E94DB7D91
:10982000D6011496ED91FC9181818F708B1559F1C1
:109830006AED75E08FE19DE00E94B069F6016381F9
:109840008FE19DE00E94DB7D68ED75E08FE19DE09A
:109850000E94B069D6011496ED91FC9161816F7000
:109860008FE19DE00E94DB7D65ED75E08FE19DE07D
:109870000E94B0696B2D8FE19DE00E94DB7D8FE13E
:109880009DE00E94A768F60104811581FB2DFF7001
:10989000EF2ED8011196FC90BCE0BB1508F4CCC0AB
:1098A000EB2DF0E08827E85AF34B8F4F0C94DBB98F
:1098B0006A4CC64C774CF94C034D774CD74C774CDF
:1098C000064D0C4DE84C0F4D194D882309F4A8CFD7
:1098D00080E0B8C0F80191819F70953009F4ACC068
:1098E000D6012D913C91963078F59230E1F169E9FD
:1098F00074E0D6018D919C910E94667D60E0009796
:1099000009F49AC0FF2DF07FEF2AD8011196EC924E
:1099100019821A821B821C821D821E821F82188657
:109920000B810F700B83E980FA801C8120E03E815F
:109930004F8158850E946E47D6011496ED91FC9197
:1099400080818F7E80837DC09730B1F09A3079F628
:1099500062E974E0C9010E94667DF801608162FBE2
:10996000662760F9CCCF6CE874E0C9010E94667D7F
:10997000F80160816170C3CF6BE874E0C9010E9497
:10998000667DD8016C9166956170B9CF6EE974E01F
:10999000F601808191810E94667DD8012C91622F11
:1099A0006170322F3E7F20FF31603C93A8CF63EA85
:1099B00074E0F601808191810E94667DD8012C912E
:1099C00021FB662760F9322F3D7F21FF3260EDCF0A
:1099D00069EA74E0F601808191810E94667DD80178
:1099E0002C9122FB662760F9322F3B7F22FF3460E7
:1099F000DCCF6FEA74E0F601808191810E94667D80
:109A0000D8016C91B7CF64EB74E0F5CF6AEB74E0EA
:109A1000F60180819181B3CF60EC74E0F9CF67ECFF
:109A200074E0F601808191810E94667DD8016C917D
:109A300096CF6DEC74E0F5CFBF2DB07FEB2AF80127
:109A4000E18281E028960FB6F894DEBF0FBECDBF4D
:109A5000DF91CF911F910F91FF90EF90DF90CF900A
:109A6000BF900895AF92BF92CF92DF92EF92FF9294
:109A70000F931F93CF93DF93CDB7DEB7C154D109B6
:109A80000FB6F894DEBF0FBECDBF5C016B018A013B
:109A900061E37AE08FE19DE00E94B069B5018FE15A
:109AA0009DE00E944A696EE27AE08FE19DE00E94AB
:109AB000B069C114D104A1F00C0D1D1DF801108274
:109AC0000E94BF0C76016A3F7105E4F461E27AE01E
:109AD00087E79CE00E94B06987E79CE00E94A76846
:109AE000CF5BDF4F0FB6F894DEBF0FBECDBFDF9167
:109AF000CF911F910F91FF90EF90DF90CF90BF908B
:109B0000AF9008950E151F0541F0F70161917F0197
:109B10008FE19DE00E94BD68F5CF8FE19DE00E943E
:109B2000A76880918209909183099E012F5F3F4F22
:109B3000790130E020E043E050E00597C9F042E0D1
:109B400050E061E4C7010E943823F7010190002032
:109B5000E9F731978F010E191F09A801B701C50157
:109B60000E9454BE892BF1F030E020E041E050E04B
:109B700061E4C7010E943823F70101900020E9F752
:109B800031978F010E191F09A801B701C5010E9465
:109B900054BE892B39F066E17AE08FE19DE00E94A6
:109BA000B0699ECF0A0D1B1D64ED74E0C8010E94D0
:109BB00034BE892B69F4F60101900020E9F7319752
:109BC000EC19FD09329720F0C6010E94536E88CF30
:109BD0006FE270E0C8010E9429BE5C01009749F065
:109BE000FC0110828181843209F47ACFFFEFAF1A31
:109BF000BF0AF8018081843209F472CFB801C7012D
:109C00000E945C32C7010E94BA2F882329F0A50167
:109C1000B601C7010E94C044C7010E94810F60CFF6
:109C20006F927F928F929F92AF92BF92CF92DF926C
:109C3000EF92FF920F931F93CF93DF93CDB7DEB7D1
:109C4000C854D1090FB6F894DEBF0FBECDBF3C019A
:109C50004B01FC010081118165E674E0C8010E949E
:109C6000667D5C016AE674E0C8010E94667D6C0155
:109C7000A114B10419F4892B09F4C5C06EE974E08C
:109C8000C8010E94667D7C0169E974E0C8010E94F8
:109C9000667D8C0166EF75E08FE19DE00E94B06902
:109CA000F30163818FE19DE00E94DB7D64EF75E04D
:109CB0008FE19DE00E94B069B4018FE19DE00E94B8
:109CC000EF7D8FE19DE00E94A768C114D10409F4E3
:109CD0004BC0F60180858F70843009F045C06185E6
:109CE000728540E450E0CE0101960E9462BE0E945F
:109CF000817D8823C9F180910E09811135C06FE201
:109D000070E0CE0101960E9429BE892B51F4F60124
:109D10002185328543E050E060E4CE0101960E9447
:109D200038238114910479F0E114F10429F0F7014A
:109D300080858F70843091F06DED74E0CE010196D6
:109D40000E94058611C00115110529F0F8018085D2
:109D50008F70843019F060EE74E0F0CF6185728509
:109D6000FB0180818111EACFA114B10409F44BC039
:109D7000F50180858F70843009F045C0618572855A
:109D8000CE0101960E945C32CE0101960E94BA2F4C
:109D90008823A9F1892809F44CC0E114F10431F0B9
:109DA000F70180858F70843009F461C025961CAE60
:109DB0001DAE1EAE1FAE259729961CAE1DAE1EAE63
:109DC0001FAE299724962FAD24972F70CC24C394CF
:109DD000F12CE12C01E023961FAD239725963FAD92
:109DE000259740E027965FAD279728966FAD289777
:109DF00029967FAD2997CE0101960E94E736CE01C4
:109E000001960E94810FC85BDF4F0FB6F894DEBF4A
:109E10000FBECDBFDF91CF911F910F91FF90EF90BB
:109E2000DF90CF90BF90AF909F908F907F906F907A
:109E300008950115110529F0F80180858F7084308F
:109E4000B1F025961CAE1DAE1EAE1FAE259729960D
:109E50001CAE1DAE1EAE1FAE299724962FAD2497C3
:109E60002F70CC24C394F12CE12C02E0B4CF618597
:109E70007285FB018081882311F250E040E0CE0121
:109E800001960E94C044BBCF2F923F924F925F92A7
:109E90006F927F928F929F92AF92BF92CF92DF92FA
:109EA000EF92FF920F931F93CF93DF93CDB7DEB75F
:109EB000CB56D1090FB6F894DEBF0FBECDBF4C0113
:109EC0003B01DC0112968C91803409F4D8C208F071
:109ED0004BC0843008F063C2F40184819581892BE2
:109EE00009F45DC2A3016FEFC4010E94DB4BD401F2
:109EF00012960C9112970695017013961C91139768
:109F00008AEC810F803108F043C064EE74E08D91DB
:109F10009C910E94667D5C010097D1F1FC018085D7
:109F20008F708530A9F580913A0C181324C0809168
:109F30003B0C803401F580913C0C90913D0C6C0100
:109F4000990FEE08FF0860E0C5010E94E27DFC0168
:109F500081859285A385B485C816D906EA06FB06D5
:109F60000CF060C0512C3EC0823409F488C208F461
:109F700016C28058AECF10933A0C80E480933B0C0D
:109F8000812F0E94858490933D0C80933C0CD7CF09
:109F9000212F30E0F901EA5CF94E8491F901E05299
:109FA000FA4E1491F901E657FA4EF490FF2009F4A5
:109FB00036C081110E94DD82EF2DF0E0EE0FFF1F11
:109FC000E95FF94FA591B491EC911E2331E020E0B7
:109FD00009F430E0832F922F552453940817190663
:109FE00009F0C0CFD4011496ED91FC91E181EF709E
:109FF000E150EC3008F07BC0F0E08827ED5FFF4ACD
:10A000008F4F0C94DBB92350975158508D50975176
:10A01000A6509751D95005511E515D517E5190E087
:10A0200080E0DACF61E0C5010E94E27D55245394BF
:10A03000FC0181859285A385B4858C159D05AE05AF
:10A04000BF0584F68FCF0E9437859B01AC01442762
:10A050005527D4011496ED91FC916281738190E0B3
:10A0600080E0AA24AA94BA2CC12CD12C18EEE12E9F
:10A0700013E0F12E00E010E00E94DD228823B9F108
:10A08000F401008111816FEA74E0C8010E94667DCD
:10A09000892B41F464EB74E0C8010E94667D892B32
:10A0A00009F408C1A30163E0C4010E94DB4B1FC097
:10A0B0000E9437859B01AC0144275527D401149693
:10A0C000ED91FC916281738190E080E0AA24AA94D2
:10A0D000BA2CC12CD12C1CE2E12EFF24F39400E019
:10A0E00010E00E94DD22A30164E0811182C0D4014E
:10A0F0001496ED91FC91808183FB992790F9951539
:10A1000009F4BAC1982F907E09F432C1982F907E3D
:10A1100090528F71892B808342C10E9437859B01A9
:10A12000AC0144275527D4011496ED91FC9162812E
:10A13000738190E080E0AA24AA94BA2CC12CD12C7F
:10A1400016E9E12EF12C00E010E0CBCF0E9437851C
:10A150009B01AC0144275527D4011496ED91FC9145
:10A160006281738190E080E0AA24AA94BA2CC12C69
:10A17000D12C18EEE12E13E0F12E00E010E00E9449
:10A18000DD22882309F4B3CFF401008111816AEB49
:10A1900074E0C8010E94667D892B41F460EC74E094
:10A1A000C8010E94667D892B09F484C0A30168E080
:10A1B0007BCF0E9437859B01AC0144275527D401F2
:10A1C0001496ED91FC916281738190E080E0AA2465
:10A1D000AA94BA2CC12CD12C1CE2E12EFF24F394BA
:10A1E00000E010E00E94DD22A30169E0882309F469
:10A1F0007ECFC4010E94DB4B0E943785D4011496A8
:10A20000ED91FC917383628372CF0E9437859B012D
:10A21000AC0144275527D4011496ED91FC9162813D
:10A22000738190E080E0AA24AA94BA2CC12CD12C8E
:10A2300016E9E12EF12C00E010E0D4CF0E94378522
:10A240009B01AC0144275527D4011496ED91FC9154
:10A250006281738190E080E0AA24AA94BA2CC12C78
:10A26000D12C18EEE12E13E0F12E00E010E00E9458
:10A27000DD22882309F43BCFF4010081118167ECD2
:10A2800074E0C8010E94667D892B39F46DEC74E09E
:10A29000C8010E94667D892B19F0A3016BE004CFF1
:10A2A00069EA74E0C8010E94667DA30166E0892B1B
:10A2B00009F4FACEA3016DE0F7CE0E9437859B0129
:10A2C000AC0144275527D4011496ED91FC9162818D
:10A2D000738190E080E0AA24AA94BA2CC12CD12CDE
:10A2E0001CE2E12EFF24F39400E010E00E94DD2246
:10A2F000882309F4FCCEA3016CE07BCF0E94378554
:10A300009B01AC0144275527D4011496ED91FC9193
:10A310006281738190E080E0AA24AA94BA2CC12CB7
:10A32000D12C16E9E12EF12C00E010E0DFCF0E94E5
:10A3300037859B01AC0144275527D4011496ED9134
:10A34000FC916281738190E080E0AA24AA94BA2CE7
:10A35000C12CD12C18E5E12E12E0F12E00E010E026
:10A360000E94DD22882309F4C2CEA30160E09CCEC6
:10A370000E943785D4011496ED91FC911597738353
:10A38000628312968C9180FF26C0552041F0608137
:10A3900068606083617070E0C4010E94104E90E0BC
:10A3A00080E0C559DF4F0FB6F894DEBF0FBECDBFBA
:10A3B000DF91CF911F910F91FF90EF90DF90CF90A1
:10A3C000BF90AF909F908F907F906F905F904F90D5
:10A3D0003F902F900895652D70E0C4010E94104EAB
:10A3E000D4011496ED91FC91552009F181818F7073
:10A3F0008230D1F060F4A30161E0882371F0D401D0
:10A400001496ED91FC91808150FA83F984CE8530C9
:10A4100059F0A3016AE0873091F7C4010E94DB4B39
:10A42000882309F4BCCFEBCFA30166E0F6CFE1812E
:10A43000EF70E150ED3018F7F0E08827ED5DFD4A50
:10A440008F4F0C94DBB93052FF5133523352FF51CE
:10A450003652FF51395239523952395239523352E8
:10A46000A30162E0DACFA30165E0D7CFA30167E0E3
:10A47000D4CFA30160E0D1CF8F7180664CCE64EE63
:10A4800074E0F401808191810E94667D8C01D40189
:10A4900013968C9190913A0C8913E3C090913B0CE8
:10A4A000903409F0DEC080913C0C90913D0C5C0131
:10A4B0000115110509F4FCC0F80120852F70253025
:10A4C00009F0F6C0C8010E94427EA2968FAFA29703
:10A4D000843008F4D2C063E0C8010E94E27DDC0150
:10A4E00019968D919C914AE0742E789E1001799E68
:10A4F000300C112462E0C8010E94E27DFC018185DC
:10A500009285789E6001799ED00C1124AC96DFAEC6
:10A51000CEAEAC972601DD0C6608770861E0C80175
:10A520000E94E27D7C0160E0C8010E94E27DDC01C6
:10A5300019962D913D914D915C911C97A6962CAF4B
:10A540003DAF4EAF5FAFA69795010B2C000C440BAF
:10A55000550BA6968CAD9DADAEADBFADA697281B95
:10A56000390B4A0B5B0BB101032C000C880B990BC8
:10A5700064197509860997090E9440B9D70119968F
:10A580002D913D914D915C911C97A696CCACDDAC84
:10A59000EEACFFACA6972C193D094E095F09A696B3
:10A5A0002CAF3DAF4EAF5FAFA6970E9472B9420E7F
:10A5B000531E641E751EA2962FADA297253009F476
:10A5C0006EC081E090E0A101032C000C660B770BBC
:10A5D000441555056605770534F42A013B01AA2484
:10A5E000AA9423E0B22EAC96CEACDFACAC97A60119
:10A5F000DD0C660B770B441655066606770624F4C9
:10A600002A013B01B12CA12CA2962FADA29722309A
:10A6100009F061C02501BB0C6608770860E0C8013D
:10A620000E94E27DFC0181859285A385B485481650
:10A6300059066A067B060CF474C161E0C8010E94E9
:10A64000E27DFC0181859285A385B48584159505FD
:10A65000A605B7050CF0A3CE412C512C3201439432
:10A6600063C180933A0C90E490933B0C0E948584E4
:10A6700090933D0C80933C0C1ACF8AE08A9D200178
:10A680008B9D500C1124052C000C66087708AC96A5
:10A690001FAE1EAEAC97212C38E2332E92CF64E071
:10A6A000C8010E94E27DDC0119968D919C918BCFAF
:10A6B0002AE0289F2001299F500C1124052C000C12
:10A6C00066087708AC961FAE1EAEAC97212C98E2B8
:10A6D000392E81E090E0D4011496ED91FC914281F5
:10A6E00053819501241B350B37FF03C0319521950C
:10A6F00031098217930774F08081982F929596956F
:10A700009770963050F49F5F9295990F907E8F715D
:10A71000892B02C080818F7180838081803AB8F05C
:10A72000AC96EEADFFADAC976F01FF0FEE08FF08E2
:10A73000C414D504E604F70451F0C101330CAA0B8C
:10A74000BB0B84159505A605B70509F028CE4A155B
:10A750005B0509F424CE6D961CAE1DAE1EAE1FAE79
:10A760006D976C968FAD6C978F7080666C968FAF7F
:10A770006C976D968CAD9DADAEADBFAD6D9765968A
:10A780008CAF9DAFAEAFBFAF659769964CAE5DAE77
:10A790006EAE7FAE699763E076E08FE19DE00E9448
:10A7A000B069D40113966C918FE19DE00E94DB7D2E
:10A7B00061E076E08FE19DE00E94B069CE018F5AA2
:10A7C0009F4F0E94282761E674E0F4018081918107
:10A7D0000E94667D6296EFAC62976396FFAC6397CA
:10A7E00064960FAD649765961FAD659766962FAD1D
:10A7F000669767963FAD679768964FAD689769967D
:10A800005FAD69976FEF0E946E47D4010D911C9167
:10A8100065E674E0C8010E94667D6C016AE674E03A
:10A82000C8010E94667D8C010097E1F1FC018085E2
:10A830008F708430B9F56185728540E450E0CE01B7
:10A8400001960E9462BE6FE270E0CE0101960E9406
:10A8500029BE892B59F4D80119962D913C9143E0DA
:10A8600050E060E4CE0101960E94382300E020E031
:10A8700032E040E150E0BE016F5B7F4FCE018F5A66
:10A880009F4F0E943C190E94817D882359F080913E
:10A890000E09811107C0BE016F5B7F4FCE0101968B
:10A8A0000E940586C114D104A9F1F60180858F703C
:10A8B000843081F561857285CE0101960E945C32FB
:10A8C000CE0101960E94BA2F882301F1CC24C394B3
:10A8D000F12CE12C62960FAD629763961FAD6397E2
:10A8E00064962FAD649765963FAD659766964FADBC
:10A8F000669767965FAD679768966FAD689769963C
:10A900007FAD6997CE0101960E94E736CE01019690
:10A910000E94810FD4011496ED91FC91B382A28222
:10A920003ECD412C512C3201D4011496ED91FC9175
:10A9300082819381092E000CAA0BBB0B841595050F
:10A94000A605B70509F42BCDB201C4010E94104E33
:10A95000D4011496ED91FC915382428220CDAF92A6
:10A96000BF92CF92DF92EF92FF920F931F93CF93FC
:10A97000DF9300D000D0CDB7DEB780912108909151
:10A980002208892B09F4BBC0809180098F5F8093D6
:10A9900080090E9437859B01AC0160911508709178
:10A9A00016088091170890911808AA24AA94BA2C26
:10A9B00065011FE0E12EF12C00E010E00E94DD2295
:10A9C000882309F459C0E0912108F09122080681FA
:10A9D00017810115110509F441C0F80180858F70B8
:10A9E0008630C1F561E674E0C8010E94667D00977B
:10A9F000F9F0FC0120852F702530D1F4E680F78036
:10AA0000E114F10439F1FA82E982B801CE0101962C
:10AA10000E9478158D819E81892B31F062E070E073
:10AA2000CE0101960E94444FF701E280F380E8CF07
:10AA30001A83098370E060E0CE0101960E947815C8
:10AA40008D819E81892B31F062E070E0CE0101960C
:10AA50000E94444FF80102811381BBCF0E943785C9
:10AA60006093150870931608809317089093180840
:10AA700010923A0C10923B0C0E9437859B01AC015E
:10AA80006091110870911208809113089091140838
:10AA9000AA24AA94BA2C650118E8E12E13E1F12E3C
:10AAA00000E010E00E94DD22882321F1E0912108DE
:10AAB000F0912208068117810115110589F0F8012E
:10AAC00080858F70863041F41A83098370E060E0DE
:10AAD000CE0101960E947815F80102811381ECCF16
:10AAE0000E943785609311087093120880931308B1
:10AAF0009093140880918009815080938009269654
:10AB00000FB6F894DEBF0FBECDBFDF91CF911F917E
:10AB10000F91FF90EF90DF90CF90BF90AF9008958E
:10AB20004F925F926F927F92AF92BF92CF92DF92DD
:10AB3000EF92FF920F931F93CF93DF93CDB7DEB7C2
:10AB400067970FB6F894DEBF0FBECDBF64EB70E120
:10AB50008FE19DE00E94B0698FE19DE00E94A768AF
:10AB60000E9437852B013C0180918009882319F1CF
:10AB70000E9437859B01AC01AA24AA94BA2C6501D6
:10AB800010E1E12E17E2F12E00E010E0C301B20166
:10AB90000E94DD2281110FC00E94CA6E809182093D
:10ABA00090918309059711F00E94F8430E948E341A
:10ABB0000E94AF54D9CF80918009882351F061E978
:10ABC00070E187E79CE00E94B06987E79CE00E9403
:10ABD000A7686BE770E18FE19DE00E94B0698FE1AB
:10ABE0009DE00E94A768E0918409F09185090681A3
:10ABF00017818091840990918509892B71F1011544
:10AC0000110559F1D80118968C918F70853009F58E
:10AC1000C8010E94427E8823E1F0F80160817181C1
:10AC2000CE0101960E945C32CE0101960E94BA2F9D
:10AC3000882359F08A859B85009739F0DC01ED91D6
:10AC4000FC910284F385E02D1995CE0101960E94B6
:10AC5000810FF80102811381CCCF10922608109247
:10AC6000250863E770E18FE19DE00E94B0698FE104
:10AC70009DE00E94A76810920B096BE570E18FE1DF
:10AC80009DE00E94B0690E94BF0CAB01BC012AE0AC
:10AC90008FE19DE00E945B688091230890912408D9
:10ACA0000E94AE7F1092240810922308109222086E
:10ACB00010922108109285091092840910920D09B2
:10ACC00010920C0910927E0910927D0966E570E1E0
:10ACD0008FE19DE00E94B0690E94BF0CAB01BC01F6
:10ACE0002AE08FE19DE00E945B688FE19DE00E9479
:10ACF000A7681092810910927F0967960FB6F894A1
:10AD0000DEBF0FBECDBFDF91CF911F910F91FF909E
:10AD1000EF90DF90CF90BF90AF907F906F905F905B
:10AD20004F90089580910E098F5F80930E09A8952A
:10AD30000E94AF5480910E09815080930E090895AE
:10AD4000CF92DF92EF92FF92CF93DF93EC018C854D
:10AD5000883068F40E94C6760E9437856B017C01BA
:10AD60008C850E94E276811109C088E08C87DF9192
:10AD7000CF91FF90EF90DF90CF9008950E94925670
:10AD800061E070E080E090E00E94CA840E94378514
:10AD9000AB01BC014C195D096E097F098D859E854B
:10ADA000B0E0A0E0481759076A077B07C8F28C8516
:10ADB0000E94D476DACFCF92DF92EF92FF921F9368
:10ADC000CF93DF93EC017B016A018C85883048F4D6
:10ADD0000E94E276882319F08C850E94C67688E06E
:10ADE0008C87F70182819381A481B5810097A105A9
:10ADF000B10551F490E080E0DF91CF911F91FF9079
:10AE0000EF90DF90CF9008958F3F9F4FAF4FBF4F90
:10AE100089F370E060E081E20E941D77182F8C8733
:10AE2000883040F780E591E00E940380A7014E5FE3
:10AE30005F4F24E030E06CE070E0812F0E94FC1E48
:10AE4000B601812F0E94F17664E070E0812F0E94AC
:10AE5000FE710E9437856B017C018C850E94E27631
:10AE6000873121F18C3111F1882321F20E9437853D
:10AE7000AB01BC014C195D096E097F098D859E856A
:10AE8000B0E0A0E084179507A607B70748F00E9436
:10AE9000925661E070E080E090E00E94CA84DDCFCD
:10AEA0008C850E94D47688E08C87A4CF81E090E0E6
:10AEB000A3CF8F929F92BF92CF92DF92EF92FF9299
:10AEC0000F931F93CF93DF93CDB7DEB76D970FB678
:10AED000F894DEBF0FBECDBF009123081091240867
:10AEE0000115110509F4ECC1809180098F5F8093F1
:10AEF000800968EE74E0C8010E94667D9093850920
:10AF0000809384096EEE74E0C8010E94667D909380
:10AF10000D0980930C0965EF74E0C8010E94667DFD
:10AF2000909322088093210868EF74E0C8010E9482
:10AF3000667D90937E0980937D090E94B1251092D1
:10AF4000260810922508E0918409F0918509309730
:10AF500009F4C8C0E680F780009184091091850942
:10AF60000115110509F4B7C0E114F10409F4B3C0E7
:10AF7000D70118968C918F70853091F7C7010E9488
:10AF8000427E823068F3B701CE0101960E94E8321A
:10AF9000CE0101960E94BA2F882309F44AC08A85FF
:10AFA0009B85009759F570E060E0CE0101960E9404
:10AFB00098168C01912C812C97FF06C01195019554
:10AFC000110988248394912CCE0101960E9499182E
:10AFD000C82ED12C89858530A9F1863051F5B02E47
:10AFE00061E0802F0E94728361E0892809F451C0DA
:10AFF000CA94CD2809F051C060E04FC0DC01ED914A
:10B00000FC910484F585E02D1995892B49F08A85FA
:10B010009B85DC01ED91FC910284F385E02D19956F
:10B020008A859B85DC01ED91FC910680F781E02DFE
:10B030001995D7011296ED90FC90CE0101960E94D1
:10B04000810F8ACFCD2829F462E0CE0101960E94BB
:10B050009D1761E0802F0E94728360E0802F0E9424
:10B06000448366E57CE08FE19DE00E94B069B80111
:10B070008FE19DE00E94EF7D61E57CE08FE19DE046
:10B080000E94B0696FE47CE08FE19DE00E94B069AE
:10B09000D0CFCA94CD2809F0AFCFC62ED12C8B2D9E
:10B0A0000E9444836AE47CE08FE19DE00E94B069E5
:10B0B000B8018FE19DE00E94EF7D68E47CE08FE1C4
:10B0C0009DE00E94B069B6018FE19DE00E94EF7D96
:10B0D00066E47CE0D9CFF8018681978190932608B9
:10B0E000809325088FE19DE00E94A768E0912108E8
:10B0F000F0912208309709F48EC0809180098F5F0B
:10B1000080938009068117810115110509F47EC01D
:10B11000D80118968C918F70863009F06DC0198F08
:10B12000088F70E060E0CE0148960E9478158C8D03
:10B130009D8D892B09F460C080912308909124088B
:10B14000892B09F459C0E88CF98CF70180858F7040
:10B150008630B9F561E674E0C7010E94667D00970C
:10B16000F1F0DC0118962C9118972F702530B9F466
:10B170001696CD90DC90C114D10419F1DA82C982FF
:10B18000B701CE0101960E947815ED81FE811082F3
:10B19000118212821382F601C280D380ECCFFA8230
:10B1A000E98270E060E0CE0101960E9478158D8101
:10B1B0009E81892B31F062E070E0CE0101960E9401
:10B1C000444FEC8DFD8D10821182128213828A8D84
:10B1D000843068F462E0823008F060E08B8D0E9479
:10B1E0007283EC8DFD8D8181807F818305C08034E9
:10B1F00041F060E0823431F0D80112960D911C913B
:10B2000083CF62E08B8D0E947283F6CF809180099C
:10B2100081508093800969E37CE08CE69CE00E9489
:10B22000B06961E37CE08CE69CE00E94B06981E05B
:10B230002091840930918509232B09F480E00E9434
:10B240000F1368E27CE08CE69CE00E94B06981E02C
:10B250002091210830912208232B09F480E00E94DC
:10B260000F1361E27CE08CE69CE00E94B06981E013
:10B2700020917D0930917E09232B09F480E00E9402
:10B280000F138CE69CE00E94A7686CE17CE08CE6E2
:10B290009CE00E94B0690E94BF0CAB01BC012AE097
:10B2A0008CE69CE00E945B688CE69CE00E94A768AC
:10B2B00081E0809381098091800981508093800989
:10B2C0006D960FB6F894DEBF0FBECDBFDF91CF9164
:10B2D0001F910F91FF90EF90DF90CF90BF909F90C4
:10B2E0008F900895CF93DF9300D000D01F921F92CC
:10B2F000CDB7DEB762E87CE08CE69CE00E94B069E6
:10B300008CE69CE00E94A76870E060E086ED9DE01E
:10B310000E94E41486ED9DE00E9435198B3791055B
:10B3200009F048C01C821B828EEA92E09A838983CE
:10B3300086ED9DE09E838D838FEF9FEF98878F83AF
:10B340008091230890912408892B11F00E94905538
:10B35000CE0101960E94E07F9093240880932308F9
:10B36000892B69F465E67CE087E79CE00E94B06980
:10B3700087E79CE00E94A76890E080E012C06EE53D
:10B380007CE08CE69CE00E94B0698CE69CE00E9428
:10B39000A7680E9459578FEB9DE00E94A05681E05C
:10B3A00090E028960FB6F894DEBF0FBECDBFDF91B8
:10B3B000CF91089561E77CE08CE69CE00E94B06943
:10B3C0008CE69CE0D7CF0C947259CF93DF9300D0DA
:10B3D00000D0CDB7DEB7CE0101960E942E68BE0127
:10B3E0006F5F7F4F8FE19DE00E94A2698FE19DE03A
:10B3F0000E94A768CE0101960E9429688FEF9FEFF7
:10B4000026960FB6F894DEBF0FBECDBFDF91CF9169
:10B410000895EF92FF920F931F93CF93DF9300D085
:10B420001F92CDB7DEB78C017B01FB01848588308C
:10B43000A8F08BE993E0F801918380831282138254
:10B4400014821582C8010F900F900F900F90DF911A
:10B45000CF911F910F91FF90EF90089580E591E0BB
:10B460000E94038024E030E0AE014F5F5F4F6CE04C
:10B4700070E0F70184850E942B20BE016F5F7F4F33
:10B48000C8010E94D469DECFAF92BF92CF92DF9203
:10B49000EF92FF920F931F93CF93DF93CDB7DEB759
:10B4A000C258D1090FB6F894DEBF0FBECDBF8E01D2
:10B4B0000F5B1F4FD8011D921C92FE01ED5BFF4FE9
:10B4C0002EE1DF011D922A95E9F702970CF451C194
:10B4D000FB01628173814FE150E0C8010E9462BEAE
:10B4E000B8018CE69CE00E944A6962E27EE08CE64C
:10B4F0009CE00E94B0698CE69CE00E94A768809165
:10B50000D50D1F928F938091D40D1F928F938091B0
:10B51000D30D1F928F938091D20D1F928F938091A4
:10B52000D10D1F928F938091D00D1F928F938DEF2D
:10B5300094E09F938F931F9280E48F93CE010196A6
:10B540006C019F938F930E947CBE64EE7DE08CE63D
:10B550009CE00E94B069B8018CE69CE00E944A69B8
:10B56000B6018CE69CE00E944A698CE69CE00E9451
:10B57000A7687E0191E6E90EF11CD70113961C9293
:10B580001E92129788EE93E0A0E0B0E0F70184836A
:10B590009583A683B78388E0848788EE93E09687B7
:10B5A00085878DE693E091838083108B0787128ACD
:10B5B000118A80E590E0948B838B178A6EED7DE095
:10B5C0008FE19DE00E94B0690E94BF0CAB01BC01FD
:10B5D0002AE08FE19DE00E945B688FE19DE00E9480
:10B5E000A76864E670E080E090E00E94CA846EEF95
:10B5F00074E688E491E70E948EB18C010FB6F8944E
:10B60000DEBF0FBECDBF892BB1F183E090E00E9479
:10B610008CADD8011D969C938E931C97FC01F182F2
:10B62000E0821282C7010E943312882319F0C701F9
:10B630000E94A056D70151966D917C9152975396D6
:10B64000AD90BC906115710509F4A6C0CE01875874
:10B650009F4F0E94D469A501BE0167587F4FC70163
:10B660000E94DB56181619060CF40DC1C8010E9481
:10B67000217110E000E066ED7DE08FE19DE00E9429
:10B68000B0698FE19DE00E94A76864E670E080E009
:10B6900090E00E94CA84D7015596ED90FC906DEC25
:10B6A0007DE08FE19DE00E94B069B7018FE19DE0F0
:10B6B0000E94EF7D8FE19DE00E94A76864E670E044
:10B6C00080E090E00E94CA840115110509F4D6C0FB
:10B6D000B8ECEB16F10409F0BFC061EC7DE08CE63C
:10B6E0009CE00E94B06964EF71E080E090E00E940D
:10B6F000CA84ED961FAE1EAEED97EF961FAE1EAE3E
:10B70000EF978FEF9FEFC158DF4F99838883CF5713
:10B71000D04084EC92E0EB969FAF8EAFEB97CF5783
:10B72000DF4F19830883C158D040F89480912308D3
:10B7300090912408892B11F00E949055CE018758D2
:10B740009F4F0E94E07F9093240880932308789471
:10B75000C8010E9421718091230890912408892BAF
:10B7600009F058C06AEA7DE087E79CE00E94B06972
:10B7700082C040E250E066E17EE0C8010E94DDB098
:10B7800068EF7DE08CE69CE00E94B069B8018CE631
:10B790009CE00E944A69AFCEF70167857089A501D8
:10B7A000C7010E9455125ECF6E01E9E7CE0ED11C93
:10B7B000DF92CF928FE19DE09F938F931F930F9322
:10B7C0000E9432B20F900F900F900F900F900F9039
:10B7D000019709F050CFD6018D919C91F701968B7E
:10B7E000858B90E0D12CFAE0DF120FC09A3009F47B
:10B7F00042CFC8010E94D9B18F3F21F4C8010E94F5
:10B80000217139CF9D2DD82EEECF8DE0D812F1CFFA
:10B81000D92EEFCF6FE97DE08CE69CE00E94B06905
:10B820000E94595768E97DE08CE69CE00E94B0696F
:10B8300084E090E0CE57DF4F0FB6F894DEBF0FBE26
:10B84000CDBFDF91CF911F910F91FF90EF90DF90CF
:10B85000CF90BF90AF90089560E87DE087E79CE0CF
:10B860000E94B069B70187E79CE00E94EF7D87E7FF
:10B870009CE00E94A7688EE090E0DCCF6DE67DE062
:10B880008FE19DE073CFF701B784A088DF92CF925C
:10B8900089E69DE09F938F931F930F930E9415B2AB
:10B8A000DF92CF9284E69DE09F938F931F930F9337
:10B8B0000E9415B2D8011C96ED91FC9181E0828323
:10B8C000DF92CF9281E69DE09F938F931F930F931A
:10B8D0000E9415B2D8011C96ED91FC911282AF9294
:10B8E000BF928BE29DE09F938F931F930F930E94D3
:10B8F00015B286E69DE09F938F931F930F930E944E
:10B9000015B2F701168A158AD8011C96ED91FC91A3
:10B91000A080B1800FB6F894DEBF0FBECDBF83E329
:10B92000C82ED12CD501ED91FC910084F185E02D3C
:10B93000C501199541970CF037CFB1E0CB1AD1086A
:10B9400009F432CF64E170E080E090E00E94CA84A4
:10B95000E9CF0E94445A90938309809382098FEB28
:10B960009DE00C94A056EF92FF920F931F93CF93FC
:10B97000DF93CDB7DEB764970FB6F894DEBF0FBE86
:10B98000CDBF0D871E872F87388B498B5A8B6B8BCA
:10B990007C8B6CE275E08FE19DE00E944A69CE01EC
:10B9A0000D960E9428279F85892F8F70082F10E001
:10B9B0002D85222309F4A1C00115110509F470C0D9
:10B9C000813009F46DC0813090F18230B1F18E3058
:10B9D00009F07BC092959F7069897A899C3011F03B
:10B9E00070E060E0CE0101960E9437686BE375E07D
:10B9F000C7010E9434BE892BE9F5BE016F5F7F4FFE
:10BA0000CE0107960E942E68CE0107960E94EA8119
:10BA1000BC0182E79BE00E94A269CE0107960E94CA
:10BA20002968CE0101960E94296880E061C06EEC11
:10BA300071E18FE19DE00E94B0696AEB71E18FE1F5
:10BA40009DE00E94B0698FE19DE00E94A7682F856C
:10BA5000207F81E090E009F480E064960FB6F894CE
:10BA6000DEBF0FBECDBFDF91CF911F910F91FF9031
:10BA7000EF90089569E475E0C7010E9434BE892BF8
:10BA800081F6BE016F5F7F4FCE0107960E942E6840
:10BA9000CE0107960E94EA81BC0185ED9AE0BBCFFA
:10BAA000213019F1223031F16DEA71E18FE19DE031
:10BAB0000E94B0696D858FE19DE00E94DB7D8FE182
:10BAC0009DE00E94A76801E010E06DE971E18FE15F
:10BAD0009DE00E94B069B8018FE19DE00E94EF7D7A
:10BAE0008FE19DE00E94A768A0CF2093000281E033
:10BAF00090E0B3CF10920002FACF813009F063CF0B
:10BB0000D3CF6F927F928F929F92AF92BF92CF923C
:10BB1000DF92EF92FF920F931F93CF93DF93CDB7F6
:10BB2000DEB72C970FB6F894DEBF0FBECDBF4C0129
:10BB300082E79BE00E942261892B79F10E94378580
:10BB4000611571058105910521F461E070E080E0E7
:10BB500090E06093B1087093B2088093B30890931B
:10BB6000B40882E79BE00E940061682E8DE290E0BD
:10BB70009A83898369824FE350E0BE016F5F7F4FF4
:10BB800087E298E00E9444BE8091AF089091B0088F
:10BB900001969093B0088093AF0885ED9AE00E94DB
:10BBA0002261892B79F10E94378561157105810524
:10BBB000910521F461E070E080E090E06093AB08D3
:10BBC0007093AC088093AD089093AE0885ED9AE031
:10BBD0000E940061782E8DE290E09A8389837982B9
:10BBE0004FE350E0BE016F5F7F4F89E698E00E940F
:10BBF00044BE8091A9089091AA0801969093AA0842
:10BC00008093A9088091B1089091B208A091B308DF
:10BC1000B091B408892B8A2B8B2B29F58AE2681204
:10BC20003CC01092B1081092B2081092B308109262
:10BC3000B4081092B0081092AF0867E278E0CE0125
:10BC400007960E94376810922708CE0107960E9437
:10BC5000FC668B859C85892B09F05CC0CE0107961C
:10BC60000E94296825C00E9437859B01AC01609124
:10BC7000B1087091B2088091B3089091B408AA24D9
:10BC8000AA94BA2C65011AE0E12EF12C00E010E034
:10BC90000E94DD22882311F2C4CFADE06A1609F2BA
:10BCA0008091AF089091B0088034910508F0B9CF29
:10BCB0008091AB089091AC08A091AD08B091AE080E
:10BCC000892B8A2B8B2B09F00DC1BAE27B1225C17F
:10BCD0001092AB081092AC081092AD081092AE080A
:10BCE0001092AA081092A90869E678E0CE0107969A
:10BCF0000E94376810926908CE0107960E94FC6680
:10BD00008B859C85892B09F02BC1CE0107960E945B
:10BD100029680FC1809100028823A1F0BE01695FEC
:10BD20007F4FCE0101960E942E68CE0101960E949F
:10BD3000EA81BC0185ED9AE00E94A269CE010196DC
:10BD40000E94296863E375E0CE0101960E9437687E
:10BD5000BE016F5F7F4FCE0107960E946B67182F61
:10BD6000CE0101960E942968112309F44DC0BE013D
:10BD7000695F7F4F8EEF9DE00E949B6781116ECFC0
:10BD8000BE01695F7F4F8EEF9DE00E9412684F8178
:10BD90005885D401ED91FC910288F389E02D30E0C3
:10BDA00020E069E375E0C4011995809167089091DE
:10BDB0006808892B09F452CF69E971E18FE19DE0B0
:10BDC0000E94B06910E000E0A0E1EA2EF12CB80179
:10BDD000CE0107960E945967FC018081882309F4EF
:10BDE00045C08B859C850817190708F03FC08091D6
:10BDF00067089091680881309105E9F1029709F48C
:10BE000065C00F5F1F4FE3CF6DE375E0CE01019674
:10BE10000E943768BE016F5F7F4FCE0107960E9478
:10BE20006B67182FCE0101960E942968112309F42F
:10BE3000BCCFBE01695F7F4F84E09EE00E949B679C
:10BE400081110CCFBE01695F7F4F84E09EE00E94AC
:10BE500012684F815885D401ED91FC910288F389D5
:10BE6000E02D30E020E063E475E09DCF8FE19DE0C0
:10BE70000E94A768F3CEB801CE0107960E945967C9
:10BE8000DC018C9168E575E0803114F463E274E0C4
:10BE90008FE19DE00E944A69B801CE0107960E9499
:10BEA0005967FC018081082E000C990BAA0BBB0B73
:10BEB00089839A83AB83BC83FE82ED82BE016F5F70
:10BEC0007F4F8FE19DE00E9468159BCFB801CE01A6
:10BED00007960E945967DC016C918FE19DE00E94FA
:10BEE000BD688FCF0E9437859B01AC016091AB0884
:10BEF0007091AC088091AD089091AE08AA24AA94E4
:10BF0000BA2C65011AE0E12EF12C00E010E00E944D
:10BF1000DD22882309F4D9CEDBCEEDE07E1609F4CC
:10BF2000D7CE8091A9089091AA088034910508F095
:10BF3000CFCE81E090E02C960FB6F894DEBF0FBE16
:10BF4000CDBFDF91CF911F910F91FF90EF90DF90C8
:10BF5000CF90BF90AF909F908F907F906F900895FB
:10BF6000809100028823A1F0BE01695F7F4FCE015E
:10BF700001960E942E68CE0101960E94EA81BC01C2
:10BF800082E79BE00E94A269CE0101960E94296887
:10BF900063E375E0CE0101960E943768BE016F5FD2
:10BFA0007F4FCE0107960E946B67182FCE01019636
:10BFB0000E942968112309F44EC0BE01695F7F4FBA
:10BFC0008AE09EE00E949B6781119FCEBE01695F5F
:10BFD0007F4F8AE09EE00E9412684F815885D4010D
:10BFE000ED91FC910288F389E02D30E020E067E4D8
:10BFF00075E0C40119958091670890916808892BB4
:10C0000009F483CE6BE971E18FE19DE00E94B06994
:10C01000912C812C00E110E0B401CE0107960E9422
:10C020005967FC018081882309F447C08B859C8572
:10C030008816990608F041C08091670890916808B9
:10C040008130910509F43EC0029709F466C0BFEF44
:10C050008B1A9B0AE1CF6DE375E0CE0101960E9439
:10C060003768BE016F5F7F4FCE0107960E946B67F6
:10C07000182FCE0101960E942968112309F4BBCF25
:10C08000BE01695F7F4F80E19EE00E949B67811146
:10C090003CCEBE01695F7F4F80E19EE00E94126846
:10C0A0004F815885D401ED91FC910288F389E02DF0
:10C0B00030E020E06BE475E09CCF8FE19DE00E94D2
:10C0C000A76823CEB401CE0107960E945967DC0110
:10C0D0008C9168E575E0803114F463E274E08FE1DF
:10C0E0009DE00E944A69B401CE0107960E945967FB
:10C0F000FC018081082E000C990BAA0BBB0B8983D5
:10C100009A83AB83BC831E830D83BE016F5F7F4F19
:10C110008FE19DE00E9468159ACFB401CE01079689
:10C120000E945967DC016C918FE19DE00E94BD681F
:10C130008ECFFC01248135816217730748F480811A
:10C140009181009729F0860F971FFC018081089547
:10C1500080E008950895AF92BF92CF92DF92EF9260
:10C16000FF920F931F93CF93DF936C017B018B01A1
:10C17000040F151FEB015E01AE18BF08C017D107F1
:10C1800059F06991D601ED91FC910190F081E02D7B
:10C19000C6011995892B79F7C501DF91CF911F91C0
:10C1A0000F91FF90EF90DF90CF90BF90AF900895E8
:10C1B000FC01A089B1898C91A689B78982FD0FC045
:10C1C0009C91818D8F5F8F73228D821749F0A18D95
:10C1D000AE0FBF2FB11D5D969C93818F08958C91FA
:10C1E0000895FC01538D448D252F30E0842F90E07D
:10C1F000821B930B541710F0CF9608950197089562
:10C20000FC01918D828D981761F0A28DAE0FBF2F2A
:10C21000B11D5D968C91928D9F5F9F73928F90E080
:10C2200008958FEF9FEF0895FC01918D828D9817EF
:10C2300031F0828DE80FF11D858D90E008958FEF2C
:10C240009FEF0895FC01918D228D892F90E0805CF5
:10C250009F4F821B91098F739927089585ED9AE06E
:10C260000E94226121E0892B09F420E0822F0895A9
:10C2700082E79BE00E94226121E0892B09F420E003
:10C28000822F089582E89CE00E94226121E0892BA0
:10C2900009F420E0822F0895FC01A48DA80FB92F86
:10C2A000B11DA35ABF4F2C91848D90E001968F73DE
:10C2B0009927848FA689B7892C93A089B1898C91FD
:10C2C00080648C93938D848D981306C00288F389C3
:10C2D000E02D80818F7D80830895EF92FF920F93F0
:10C2E0001F93CF93DF93EC0181E0888F9B8D8C8D22
:10C2F000981316C0E889F989808185FF11C0EE89FD
:10C30000FF896083E889F98980818064808381E086
:10C3100090E0DF91CF911F910F91FF90EF900895E2
:10C32000F62E0B8D10E00F5F1F4F0F731127E02EBD
:10C330008C8D8E110CC00FB607FCFACFE889F989F5
:10C34000808185FFF5CFCE010E944C61F1CFEB8D4E
:10C35000EC0FFD2FF11DE35AFF4FF0820B8FEA899E
:10C36000FB8980818062D2CFCF93DF93EC01888DEF
:10C370008823B9F0AA89BB89E889F9898C9185FD60
:10C3800003C0808186FD0DC00FB607FCF7CF8C91EE
:10C3900085FFF2CF808185FFEDCFCE010E944C61F9
:10C3A000E9CFDF91CF91089580E090E0892B29F0CB
:10C3B0000E94426181110E94000080E090E0892B80
:10C3C00029F00E94386181110E94000080E090E015
:10C3D000892B29F00E942E6181110E94000080E0CB
:10C3E00090E0892B49F080E090E0892B29F00E94B1
:10C3F000000081110C94000008950F931F93FC011D
:10C4000062857385848595850281138124813581B8
:10C41000601B710B820B930B068517852089318970
:10C42000601B710B820B930B1F910F910895DC0120
:10C43000ED91FC910190F081E02D19948FEF9FEF29
:10C440000895FC0162897389848995890895EF9222
:10C450000F931F93CF93DF93FC01248D222341F090
:10C46000213051F1DF91CF911F910F91EF900895FD
:10C47000228933894489558986899789A08DB18D10
:10C48000821B930BA40BB50B892F9A2FAB2FBB27C5
:10C490008C010F5F1F4F6281738184819581CFB7BB
:10C4A000F894DCB7E1E0ECBFEE24E394E2E0FEEFC9
:10C4B0001995DCBFCFBFD6CFF0E0E0E0DF91CF91A0
:10C4C0001F910F91EF901994FC01138E128E411160
:10C4D0000CC082899389A489B589868B978BA08F9C
:10C4E000B18F148E81E090E0089590E080E008958F
:10C4F000CF92DF92EF92FF92CF93DF93DC01CB01DB
:10C50000642FCFB7F8946D01EE24FF24CBBEDCB7C7
:10C5100041E04CBFA901E1E0FEEF1995DCBFCFBFC0
:10C52000DF91CF91FF90EF90DF90CF900895CF9360
:10C53000DF93FC01248D211110C0EC01828D938DBD
:10C54000892B49F066897789808D918D30E020E0D4
:10C5500045E00E9478621B8E1A8EDF91CF9108957C
:10C560001F93CF93DF93FC01248D211145C0162F1B
:10C57000EC01828D938D892B49F466897789808DB2
:10C58000918D30E020E043E00E9478624A8D5B8D1F
:10C59000CA0181709927FE01E80FF91F158F892BB9
:10C5A00069F02D8D3E8D6E897F89888D998D640F00
:10C5B000751F811D911D41E00E9478628A8D9B8DBF
:10C5C00001969B8F8A8F81159140B1F46E897F8986
:10C5D000888D998D30E020E045E00E9478621B8EC6
:10C5E0001A8E8E899F89A88DB98D9F5FAF4FBF4FDF
:10C5F0008E8B9F8BA88FB98F81E090E0DF91CF91D8
:10C600001F910895DC01ED91FC910280F381E02DF2
:10C6100040E01994FB012481358142815381241724
:10C62000350750F4A081B181A20FB31F8C93848190
:10C63000958101969583848380E00895CF93DF935D
:10C64000EC01E881F9810284F385E02DCE01199592
:10C650000196B9F7DF91CF910895CF92DF92EF92D3
:10C66000FF920F931F93CF93DF937C016A018B019D
:10C67000D0E0C0E0CC15DD0581F0D701ED91FC9153
:10C680000284F385E02DC70119958F3F980729F0A3
:10C69000F80181938F012196EDCFCE01DF91CF91EB
:10C6A0001F910F91FF90EF90DF90CF900895CF935F
:10C6B000C62FDC01ED91FC910088F189E02D1995E0
:10C6C000DC01ED91FC910190F081E02D6C2FCF9178
:10C6D0001994062E000C770BFC017783668308956E
:10C6E000CF93DF93EC018E819F81019611F5E88154
:10C6F000F9810088F189E02DCE011995DC01ED91D9
:10C70000FC910084F185E02D1995892BB1F0E88129
:10C71000F9810284F385E02DCE01199581329105CE
:10C7200034F3E881F9810684F785E02D682FCE0186
:10C73000199581E0DF91CF91089580E0FBCFFC0156
:10C7400020812EBD9B012150310941F051810DB452
:10C7500007FEFDCF4EB55EBD4193F5CF6150710927
:10C76000860F971F0DB407FEFDCF2EB5FC01208369
:10C770000895E0918709F091880980819091860958
:10C78000892B80830895E0918709F0918809908131
:10C790008091860980958923808308958EBD00004D
:10C7A0000DB407FEFDCF8EB5089590E02091C20A2A
:10C7B000233339F40C96982F990F990F990F80E035
:10C7C00008954896F8CFEF92FF920F931F93CF935F
:10C7D000DF93EC018B017A010E943785688B798B9E
:10C7E0008A8B9B8B8C819D81DC01ED91FC91028079
:10C7F000F381E02DA701B801DF91CF911F910F9137
:10C80000FF90EF9019941F93CF93DF93EC01162FB5
:10C810000E943785688B798B8A8B9B8B8C819D815D
:10C82000DC01ED91FC910190F081E02D612FDF9111
:10C83000CF911F911994CF92DF92EF92FF92CF93F5
:10C84000DF93EC018E819F818F3F980759F02FEF86
:10C850003FEF3F832E83DF91CF91FF90EF90DF90EA
:10C86000CF9008950E9437856B017C01A4EFCA0E1A
:10C87000A1E0DA1EE11CF11CE881F9810088F18950
:10C88000E02DCE011995DC01ED91FC910084F1853C
:10C89000E02D1995892B39F40E9437856C157D059B
:10C8A0008E059F0548F3E881F9810088F189E02D24
:10C8B000CE011995DC01ED91FC910284F385E02D08
:10C8C000DF91CF91FF90EF90DF90CF9019940E946D
:10C8D000BCBDCF92DF92EF92FF920F931F93CF9345
:10C8E000DF936C018B0186E090E00E948CADEC013F
:10C8F0009093080A8093070AF60101900020E9F757
:10C90000CF018C199D090E948CAD7C01B6010E945B
:10C910003DBEF60101900020E9F73197EC19FD09C1
:10C92000EE0DFF1D1082F982E8821B830A8380913D
:10C930000A0A90910B0A9D838C83D0930B0AC093B3
:10C940000A0ADF91CF911F910F91FF90EF90DF9036
:10C95000CF9008950F931F93CF93DF93EC018881BD
:10C960009981009759F02A813B812617370730F0CB
:10C9700081E0DF91CF911F910F9108958B016F5F3F
:10C980007F4F0E94DBBC009759F0998388831B83FB
:10C990000A832C813D81232B59F7FC011082E8CFBB
:10C9A00080E0E7CFEF92FF920F931F93CF93DF9337
:10C9B0006115710541F480E0DF91CF911F910F91D6
:10C9C000FF90EF90089541155105B1F07B01EC0106
:10C9D0000C811D81040F151FB8010E94AA648823D1
:10C9E00051F3288139818C819D81B701820F931F7A
:10C9F0000E943DBE1D830C8381E0DECFEF92FF924B
:10CA00000F931F93CF93DF93009751F4CFEFDFEF96
:10CA1000CE01DF91CF911F910F91FF90EF9008957C
:10CA2000DC011C96ED90FC90F70100811181D8018A
:10CA3000ED91FC910688F789E02DC80119958823AE
:10CA400029F3D801ED91FC910084F185E02DC80116
:10CA50001995D801ED91FC91892B61F30284F3853E
:10CA6000E02DC8011995EC01019681F2F801878942
:10CA7000882329F06C2F82E89CE00E94DB7DD7019F
:10CA800012968C91882321F2C532D10509F6D8017E
:10CA9000ED91FC910084F185E02DC8011995029774
:10CAA0005CF0D801ED91FC910688F789E02DC80172
:10CAB00019958111ECCFAACFD1E0C0E0D801ED915A
:10CAC000FC910284F385E02DC80119958F3F9807EA
:10CAD00009F49CCF9C01215431092A31310570F4AD
:10CAE0008D2F8295807F829FC00D1124D11104C0AB
:10CAF0000C2E000CDD0B8CCFD0E0E0CF9C0121563A
:10CB000031092A31310560F3C0978A30910570F7F9
:10CB10009D2F9295907F989FC00D1124E7CFFC0127
:10CB2000868197818F3F980729F02FEF3FEF37835A
:10CB300026830895808591850C94D9B17F928F9238
:10CB40009F92AF92BF92CF92DF92EF92FF920F939C
:10CB50001F93CF93DF93CDB7DEB7A6970FB6F894A8
:10CB6000DEBF0FBECDBF8C01762E942E852E20E227
:10CB7000A22ECE0101967C01DC01EA2D1D92EA95E0
:10CB8000E9F76801F3E4CF0ED11C8BE993E09AA397
:10CB900089A38FEF8BA38CA38DA38EA343E450E0D6
:10CBA000BE016F5D7F4FC6010E94BD20019609F452
:10CBB000BFC081E089838A8386E0B82EBB821C8255
:10CBC000D80114966D917D918D919C9117970E943B
:10CBD000E3B96D837E838F83988789869A8680E800
:10CBE00090E09C878B874CE150E0B701C6010E9422
:10CBF0005220FE0137968AE1DF011D928A95E9F7FE
:10CC00004801B8E08B0E911CF401D70101900D9200
:10CC1000BA94E1F740E150E0B701C6010E9452200A
:10CC2000F7011192AA94E9F796E0A92EB12C40E2FF
:10CC300050E0B701C6010E945220F1E0AF1AB108DE
:10CC4000B1F783E6898392E89A8393E59B838C838B
:10CC500085E38D8381E08E837F829DE3988797E0D3
:10CC600099878A8786E0F401DE011B9601900D9278
:10CC70008A95E1F78CE0898B8A8B6FE475E0CE01B1
:10CC800043960E943DBED8011B966C91CE014996F9
:10CC90000E948A80F8016485CE014B960E948A80AA
:10CCA000D8011D966C91CE014D960E948A804EE16E
:10CCB00050E0B701C6010E945220B3E07B121EC0B3
:10CCC00082E3898384E08A83F80196859B83978534
:10CCD0009C8390899D8391899E8396E39F83888717
:10CCE000828D8987838D8A87848D8B87858D8C87BC
:10CCF0004CE050E0B701C6010E94522087E38983CF
:10CD000086E08A8391E09B8393E09C838D838FE010
:10CD10008E838AE38F838BE388878FEF898749E04F
:10CD200050E0B701C6010E945220C6010E948C202B
:10CD3000A6960FB6F894DEBF0FBECDBFDF91CF91A0
:10CD40001F910F91FF90EF90DF90CF90BF90AF9029
:10CD50009F908F907F90089590E080E00C942A1F20
:10CD6000CF93DF93C4E1D0E00E94AC66882361F0EA
:10CD700061E070E080E090E00E94CA842197A1F712
:10CD800080E0DF91CF91089581E0FBCFFF920F9378
:10CD90001F93CF93DF931F921F92CDB7DEB7F82E6C
:10CDA00022E030E0AE014F5F5F4F66E270E00E942C
:10CDB0002B2009811A8110270127102722E030E05B
:10CDC000AE014F5F5F4F66E270E08F2D0E942B2017
:10CDD00089819A819827892798270817190749F484
:10CDE000C8010F900F90DF91CF911F910F91FF908D
:10CDF00008958C01E3CF0895AF92BF92CF92DF9256
:10CE0000EF92FF920F931F93CF93DF93DC01CD90AE
:10CE1000DC901197C114D10439F01496CD91DC91B6
:10CE20008C017601209761F4DF91CF911F910F91D2
:10CE3000FF90EF90DF90CF90BF90AF900895750175
:10CE40005701BFEFAB1ABB0AF7018081082E000C17
:10CE5000990B0E949DB0892B91F72197CC0DDD1D78
:10CE60008881082E000C990B0E949DB0892B29F017
:10CE7000CE15DF0510F02197F3CFAE014F5F5F4F66
:10CE80004E195F09D80115965C934E931497CE14F2
:10CE9000DF0420F4B701C6010E94F0BDD801ED9176
:10CEA000FC91119714968D919C91E80FF91F1082B7
:10CEB000BBCFFC01248135816217730720F4808188
:10CEC0009181009729F41092090A89E09AE0089567
:10CED000860F971F0895FB0144815581FC01248131
:10CEE00035812417350778F080819181009759F0BA
:10CEF000FB01608171816115710529F00E9454BEAA
:10CF000021E0892B09F020E0822F0895FC01248183
:10CF10003581232B39F421E0FB018081882349F0FE
:10CF200020E007C0808191810E9434BE21E0892BDE
:10CF3000B9F7822F0895FC0124813581FB014481DA
:10CF4000558124173507E1F4FC0180819181FB01B3
:10CF5000608171810097D1F061157105A1F4232BD7
:10CF6000C1F0FC01808190E008C0232B91F0FB010F
:10CF7000808190E091958195910921E0892B09F0BC
:10CF800020E0822F08950E9434BEF7CF611571050D
:10CF900061F721E0F6CFCF93DF931F921F92CDB7B9
:10CFA000DEB769831A8241E050E0BE016F5F7F4FB8
:10CFB0000E94D2640F900F90DF91CF910895CF938C
:10CFC000DF93EC0188819981009711F00E9428AECF
:10CFD000198218821D821C821B821A82DF91CF91D6
:10CFE0000895EF92FF920F931F93CF93DF93EC017D
:10CFF0007B018A01BA010E94AA6481110BC0CE0193
:10D000000E94DF67CE01DF91CF911F910F91FF90BA
:10D01000EF9008951D830C83B701888199810E9448
:10D020003DBEF0CFCF93DF93EC01FB01861797074E
:10D0300049F0608171816115710541F0448155812C
:10D040000E94F167CE01DF91CF9108950E94DF67C2
:10D05000F9CFFC01808191810C9428AEFC011182F2
:10D06000108213821282158214820C941268FC01C1
:10D070001182108213821282158214826115710549
:10D0800051F0FB0101900020E9F73197AF01461BF9
:10D09000570B0C94F1670895FB0101900020E9F70C
:10D0A0003197AF01461B570BDC01ED91FC910280DB
:10D0B000F381E02D19948F929F92AF92BF92EF92DD
:10D0C000FF920F931F93CF93DF93CDB7DEB7A19756
:10D0D0000FB6F894DEBF0FBECDBF7C01FA01CB01C5
:10D0E00019A2223008F42AE08E010F5D1F4F822E14
:10D0F000912CB12CA12CBF01A50194010E9450B923
:10D10000F901CA016A300CF5605DD8016E938D019A
:10D11000232B242B252B79F790E080E0109721F02A
:10D12000BD01C7010E944C68A1960FB6F894DEBFFE
:10D130000FBECDBFDF91CF911F910F91FF90EF9068
:10D14000BF90AF909F908F900895695CDECF66E5A9
:10D1500075E00C944C680F931F93CF93DF93EC0111
:10D160000E944C688C01CE010E94A768800F911F1D
:10D17000DF91CF911F910F910895DC01ED91FC910A
:10D180000190F081E02D1994CF92DF92EF92FF92FF
:10D190000F931F93CF93DF932115310581F4DC01A9
:10D1A000ED91FC910190F081E02D642FDF91CF9102
:10D1B0001F910F91FF90EF90DF90CF9019942A303C
:10D1C000310501F52AE077FF1DC06A017B01EC0102
:10D1D0006DE20E94BD688C0144275527BA014C19A5
:10D1E0005D096E097F092AE0CE010E945B68800F0D
:10D1F000911FDF91CF911F910F91FF90EF90DF90E2
:10D20000CF900895DF91CF911F910F91FF90EF90F4
:10D21000DF90CF900C945B688F929F92AF92BF92F9
:10D22000CF92DF92EF92FF920F931F93CF93DF93F2
:10D230007C018B014C0182E0880E911C5701E5E0D6
:10D24000AE0EB11CD0E0C0E0F40161914F01C80105
:10D250000E94DB7D6C016EE2C8010E94BD688C0DEE
:10D260009D1DC80FD91F8A149B0471F7F7016581B2
:10D27000C8010E94DB7D8C0F9D1FDF91CF911F9114
:10D280000F91FF90EF90DF90CF90BF90AF909F9065
:10D290008F9008956115710511F00C944C6890E021
:10D2A00080E008950F931F93CF93DF93EC018B01E0
:10D2B00069E575E00E944A6901151105C1F1F8019F
:10D2C00061918F01662399F1603240F0623231F052
:10D2D0006C3521F0CE010E94BD68F1CF6CE5CE0126
:10D2E0000E94BD68F801319780818C30D1F044F400
:10D2F0008930D9F08A30B9F0883009F762E6EACF90
:10D30000823259F024F462E78D3021F3D8CF8F3286
:10D3100031F06CE58C35F1F2D2CF62E2DBCF6FE217
:10D32000D9CF66E6D7CF6EE6D5CF64E7D3CF62E23A
:10D33000CE010E94BD6890E080E0DF91CF911F9107
:10D340000F910895DB0114964D915C9115976D91A5
:10D350007C91DC01ED91FC910280F381E02D199428
:10D36000EF92FF920F931F93CF93DF938C017B017A
:10D37000D0E0C0E0F701EC0FFD1F6491662361F07F
:10D38000D801ED91FC910190F081E02DC801199533
:10D39000892B11F02196EECFCE01DF91CF911F9115
:10D3A0000F91FF90EF900895DC018BE993E08D934E
:10D3B0009D9384E0FB0101900D928A95E1F7089519
:10D3C0003F924F925F926F927F928F929F92AF9215
:10D3D000BF92CF92DF92EF92FF920F931F93CF9362
:10D3E000DF93CDB7DEB7EA970FB6F894DEBF0FBE76
:10D3F000CDBF7C012A013B0169010E9437854B01A9
:10D400005C0187010D5B1F4FC8010E94FF101816B9
:10D410001906ACF00E943785681979098A099B09B9
:10D42000461657066806790608F468C10E949256A7
:10D4300061E070E080E090E00E94CA84E5CF42E2C3
:10D4400050E0BE016F5F7F4FC8010E948A10898142
:10D450008230D1F0312C832DEA960FB6F894DEBFDE
:10D460000FBECDBFDF91CF911F910F91FF90EF9035
:10D47000DF90CF90BF90AF909F908F907F906F90F4
:10D480005F904F903F900895F80184899589833487
:10D49000910501F76D817E818F8198850E94E3B9A6
:10D4A0004B015C01F60180829182A282B38246E048
:10D4B00050E0B701685F7F4FCE014D960E94E3BDFB
:10D4C000892B41F6F70180819181A281B381881671
:10D4D0009906AA06BB0608F4BDCF84819581A68172
:10D4E000B78188159905AA05BB0508F4B3CF8989CA
:10D4F0009A89AB89BC8986879787A08BB18B4EECC4
:10D5000050E070E060E0C8010E948A10312CC70131
:10D51000829698AB8FA7F701B696FAABE9AB08965F
:10D520009CAB8BAB67019AE1C90ED11CBD96FEABDB
:10D53000EDABC701429698AF8FABFD97FAAFE9AF5D
:10D540004701FEE18F0E911CF801818D928D181616
:10D5500019060CF080CFC8010E94A91083339105F1
:10D5600009F4B2C014F58130910509F464C044F4A3
:10D57000892B51F3C8010E94A910AC01552775C031
:10D580008330910509F462C00697A1F7C8010E9493
:10D59000A910B82E44E050E0B401C8010E948A10DE
:10D5A000EB2DE450FF0BAF0160C08A33910509F405
:10D5B0005FC084F585339105B1F1C697D9F6C801EE
:10D5C0000E94A9105C01B601CE0189960E94D4691F
:10D5D0008BA59CA5ADA5BEA5892B8A2B8B2BB1F065
:10D5E000EDA9FEA94080518062807380B601CE0112
:10D5F00083960E94D4698DA19EA1AFA1B8A5A50173
:10D60000481659066A067B0609F0B8CF44E050E098
:10D61000B60118C08B33910509F440C08F3F9105C6
:10D6200009F492CFA7CFC8010E94A910C8010E9497
:10D63000A910382E89CFC8010E94A91044E050E0FB
:10D640006FA978ADC8010E948A107ECFC8010E94E0
:10D65000A910B82E44E050E069AD7AADC8010E942F
:10D660008A108B2D8450990BAC0170E060E0EACFFA
:10D67000C8010E94A91044E050E069A97AA9C80134
:10D680000E948A10F70166A177A180A591A50E944A
:10D69000E3B966A377A380A791A756CFC8010E94DC
:10D6A000A91044E050E06BA97CA9C8010E948A102F
:10D6B000F70162A573A584A595A50E94E3B962A7A9
:10D6C00073A784A795A740CFC8010E94A91044E082
:10D6D00050E06FA578A9C8010E948A10F70162A1E5
:10D6E00073A184A195A10E94E3B962A373A384A34B
:10D6F00095A366A777A780AB91AB26CF33243A9446
:10D70000AACE2F923F924F925F926F927F928F920A
:10D710009F92AF92BF92CF92DF92EF92FF920F93C0
:10D720001F93CF93DF9300D000D0CDB7DEB78C012D
:10D730000E94FDAE2FEC37E040E050E00E9472B94D
:10D74000DC01CB010196A11DB11DF80184839583F5
:10D75000A683B78380839183A283B3835801F3E4C4
:10D76000AF0EB11CC5010E94541064E470E0C50105
:10D770000E94CE11882309F445C10E9437852B01F0
:10D780003C01480182E4880E911C48EEC42E43E01F
:10D79000D42EE12CF12C52E0252E1E821D82D401C4
:10D7A0008C918330B1F1811166C0F801848195813B
:10D7B000A681B7810196A11DB11D84839583A6839F
:10D7C000B7830E9437856419750986099709A701EF
:10D7D00096010E9450B9A90161E0C8010E949E65AE
:10D7E00081E0D4018C938D819E810197C1F20E94CA
:10D7F00037856419750986099709D801D6962D9140
:10D800003D914D915C91D9972617370748075907E5
:10D8100020F6C5010E945410F80184819581A681EB
:10D82000B7810196A11DB11D84839583A683B7831B
:10D830000E943785F801FE9660837183828393830B
:10D840008D819E8126960FB6F894DEBF0FBECDBFA8
:10D85000DF91CF911F910F91FF90EF90DF90CF90CC
:10D86000BF90AF909F908F907F906F905F904F9000
:10D870003F902F9008958430F1F4F80184819581D0
:10D88000A681B7810196A11DB11D84839583A683CE
:10D89000B7830E9437856419750986099709A7011E
:10D8A00096010E9450B9A90163E0C8010E949E65DB
:10D8B000D4012C9298CF813051F5F80142AD53AD8F
:10D8C00064AD75AD9E012F5F3F4FC8010E94E069B6
:10D8D000382EF2E08F1390C089819A81AB81BC8190
:10D8E000F80184839583A683B7830E9437856419E2
:10D8F000750986099709A70196010E9450B9A901E7
:10D9000063E0C8010E949E65D4013C926CCF8230D6
:10D9100009F069CFF80142AD53AD64AD75AD9E011C
:10D920002F5F3F4FC8010E94E069382EF5E08F134A
:10D930005DC0E3E0D401EC93F80182A193A1A4A11E
:10D94000B5A1892B8A2B8B2B41F484E893E0A0E0CE
:10D95000B0E082A393A3A4A3B5A3F80186A197A1E5
:10D96000A0A5B1A5892B8A2B8B2B61F482A193A151
:10D97000A4A1B5A1B695A7959795879586A397A3DA
:10D98000A0A7B1A7F80182A593A5A4A5B5A5892B49
:10D990008A2B8B2BA9F482A193A1A4A1B5A1AC01E0
:10D9A000BD0123E076956795579547952A95D1F760
:10D9B000841B950BA60BB70B82A793A7A4A7B5A7AB
:10D9C000F80186A197A1A0A5B1A586A797A7A0ABAE
:10D9D000B1AB82A593A5A4A5B5A582AB93ABA4AB2F
:10D9E000B5AB81E090E09E838D83FDCE96E08913F8
:10D9F00003C0D4011C92F7CEBFEF3B12F4CEF4016A
:10DA00001082F1CE1E821D821BCF1F920F920FB685
:10DA10000F9211240BB60F922F933F934F935F9366
:10DA20006F937F938F939F93AF93BF93EF93FF93E6
:10DA300085ED9AE00E944C61FF91EF91BF91AF910B
:10DA40009F918F917F916F915F914F913F912F9116
:10DA50000F900BBE0F900FBE0F901F9018951F9246
:10DA60000F920FB60F9211240BB60F922F933F9384
:10DA70004F935F936F937F938F939F93AF93BF93D6
:10DA8000EF93FF9385ED9AE00E94D860FF91EF91AC
:10DA9000BF91AF919F918F917F916F915F914F91C6
:10DAA0003F912F910F900BBE0F900FBE0F901F90C4
:10DAB00018951F920F920FB60F9211240BB60F926A
:10DAC0002F933F934F935F936F937F938F939F9386
:10DAD000AF93BF93EF93FF9382E79BE00E944C616B
:10DAE000FF91EF91BF91AF919F918F917F916F9136
:10DAF0005F914F913F912F910F900BBE0F900FBEF2
:10DB00000F901F9018951F920F920FB60F9211242D
:10DB10000BB60F922F933F934F935F936F937F9327
:10DB20008F939F93AF93BF93EF93FF9382E79BE015
:10DB30000E94D860FF91EF91BF91AF919F918F911B
:10DB40007F916F915F914F913F912F910F900BBEFD
:10DB50000F900FBE0F901F9018951F920F920FB647
:10DB60000F9211240BB60F922F933F934F935F9315
:10DB70006F937F938F939F93AF93BF93EF93FF9395
:10DB800082E89CE00E944C61FF91EF91BF91AF91C0
:10DB90009F918F917F916F915F914F913F912F91C5
:10DBA0000F900BBE0F900FBE0F901F9018951F92F5
:10DBB0000F920FB60F9211240BB60F922F933F9333
:10DBC0004F935F936F937F938F939F93AF93BF9385
:10DBD000EF93FF9382E89CE00E94D860FF91EF9161
:10DBE000BF91AF919F918F917F916F915F914F9175
:10DBF0003F912F910F900BBE0F900FBE0F901F9073
:10DC00001895CF92DF92EF92FF921F93CF93DF93FD
:10DC1000EC016A017B01122F60E079E08DE390E076
:10DC2000A70196010E9450B92150310941095109BB
:10DC30005695479537952795E889F98982E080833D
:10DC4000211580E1380798F0E889F989108260E8A9
:10DC500074E88EE190E0A70196010E9450B921502E
:10DC60003109410951095695479537952795EC8516
:10DC7000FD853083EE85FF852083188EEC89FD8934
:10DC80001083EA89FB89808188698083EA89FB891E
:10DC900080818F7D8083DF91CF911F91FF90EF90E6
:10DCA000DF90CF900895CF92DF92EF92FF920F9383
:10DCB0001F93CF93DF93CDB7DEB7EC970FB6F894F1
:10DCC000DEBF0FBECDBFDC012C91222309F444C07E
:10DCD0006FEC76E00E94ECB09A8389837E01B3E01A
:10DCE000EB0EF11C01E010E0D02EC12E6FEC76E0BF
:10DCF00090E080E00E94ECB0F701819391937F0166
:10DD00000E31110521F00F5F1F4F892B69F700912C
:10DD1000070A1091080AE980FA800115110579F1C6
:10DD2000D8016D917C91C7010E9434BE892B19F5F1
:10DD3000D8011296ED91FC91BE016F5F7F4F8D2D42
:10DD40009C2D199582E89CE00E94A76866EC72E120
:10DD500082E89CE00E94B069EC960FB6F894DEBFB2
:10DD60000FBECDBFDF91CF911F910F91FF90EF902C
:10DD7000DF90CF900895F80104811581CECF6AEC31
:10DD800072E182E89CE00E94B06982E89CE00E9417
:10DD9000A768D8CFCF9382E89CE00E942261892BAC
:10DDA000E9F182E89CE00E940061C82F8A3089F086
:10DDB0008D3079F0883001F568E082E89CE00E94BF
:10DDC000BD6880910C0A882331F3815080930C0A3E
:10DDD000E2CFE0910C0AF0E0E553F64F108266E5E1
:10DDE00075E082E89CE00E944A698BEC99E00E9411
:10DDF000536E10920C0ACFCF682F82E89CE00E94ED
:10DE0000BD68E0910C0AEB3330F681E08E0F809311
:10DE10000C0AF0E0E553F64FC083BDCFCF910895D3
:10DE20008F929F92AF92BF92CF92DF92EF92FF922A
:10DE30000F931F93CF93DF936115710509F497C07A
:10DE4000DB011896EC911897E295E07FE595E59552
:10DE5000E595E595E73008F08AC0EC010E2E000C40
:10DE6000FF0B8827E95CF0498F4F0C94DBB93E6FBC
:10DE70004F6F586F6F6FBA6FCC6F05706BE575E0C1
:10DE8000CE01DF91CF911F910F91FF90EF90DF9026
:10DE9000CF90BF90AF909F908F900C944C68199644
:10DEA0008C9165E675E0882359F360E675E0E8CF6C
:10DEB00019964D915D916D917C911C972AE030E00F
:10DEC000CE01DF91CF911F910F91FF90EF90DF90E6
:10DED000CF90BF90AF909F908F900C94C46819968C
:10DEE000CD90DD90ED90FC901C9720E030E0A901F2
:10DEF000C701B6010E9406B887FF09C06AE174E055
:10DF0000CE010E944A69F7FAF094F7F8F094C7013D
:10DF1000B6010E94DFBA4B015C012AE0BC01A401FA
:10DF2000CE010E945B686BE675E0CE010E944A69F3
:10DF3000C501B4010E940BB89B01AC01C701B60139
:10DF40000E94F9B92DEC3CEC4CE45DE30E94FAB977
:10DF500020E030E040E251E40E946CB80E94DFBA59
:10DF6000AB0170E060E02AE0CE010E945B6890E0C7
:10DF700080E01DC019966D917C91CE01DF91CF910B
:10DF80001F910F91FF90EF90DF90CF90BF90AF90D7
:10DF90009F908F900C94526916960D911C916BE591
:10DFA000CE010E94BD68019679F48FEF9FEFDF915B
:10DFB000CF911F910F91FF90EF90DF90CF90BF9086
:10DFC000AF909F908F9008950115110579F0B801D9
:10DFD000CE010E94106F019641F3D80112960D9167
:10DFE0001C910115110511F06CE2DACF6DE5CE013F
:10DFF0000E94BD6821E030E0019611F030E020E0A1
:10E0000088279927821B930BD2CF16960D911C91CE
:10E010006BE7CE010E94BD68019639F2011511052A
:10E0200029F1D8016D917C91CE010E94526901962F
:10E0300009F4BBCF6AE3CE010E94BD68019609F4E2
:10E04000B4CFB801CE010E94106F019609F4ADCF94
:10E05000D80112960D911C910115110539F06CE251
:10E06000CE010E94BD680196C9F69FCF6DE7BFCF74
:10E07000CF93DF93EC01E881F9810284F385E02DF1
:10E08000CE0119958F3F980769F0E881F9818132B7
:10E0900091059CF30684F785E02D682FCE01199534
:10E0A00090E080E0DF91CF910895CF92DF92EF92E0
:10E0B000FF920F931F93CF93DF937C016B01DC01E1
:10E0C000ED91FC910284F385E02D1995829761F022
:10E0D000CFEFDFEFCE01DF91CF911F910F91FF9036
:10E0E000EF90DF90CF900895F6018085807F846067
:10E0F000808786E090E00E948CAD8C01009741F310
:10E10000EBE8F9E0DC01ED93FC9380E4DF011D9284
:10E110008A95E9F780E490E0F80193838283158281
:10E120001482D701ED91FC910284F385E02DC701A3
:10E130001995EC010196C9F0C232D10509F44DC020
:10E14000C032D1050CF449C0B8018C2FCC35D105B3
:10E1500049F5D701ED91FC910284F385E02DC701CB
:10E160001995EC018F3F980721F4C8010E9428AE51
:10E17000B1CF8236910541F15CF48F32910509F1FE
:10E180008C359105D9F0829761F6B80182E20AC018
:10E190008E369105E1F04CF4B8018CE0C636D1051D
:10E1A00009F0BFCF0E940A63BCCF8237910591F07E
:10E1B000B80189E0C437D105A9F3B3CFB8018CE524
:10E1C000F1CFB8018FE2EECFB80188E0EBCFB80114
:10E1D0008AE0E8CFB8018DE0E5CFF8018481958130
:10E1E000009749F00190F081E02DE80FF91F319779
:10E1F0008081882321F0B80180E00E940A63D80161
:10E2000014968D919C910E948CADEC01009739F091
:10E210006BE879E00E943DBEC8010E9428AEF6017D
:10E22000D287C187D0E0C0E055CF8DE090E00E945A
:10E230008CAD009729F02DE0FC0111922A95E9F7A9
:10E2400008950F931F93CF93DF930097E1F0EC01B4
:10E250000C851D850115110579F0D8018D919C91D2
:10E26000009739F0DC01ED91FC910488F589E02DEF
:10E270001995C8010E9428AECE01DF91CF911F9160
:10E280000F910C9464B1DF91CF911F910F9108957C
:10E29000AF92BF92CF92DF92EF92FF920F931F93B4
:10E2A000CF93DF9300D01F92CDB7DEB76115710514
:10E2B000B1F06B01182FDB011C96AD90BC90F501FD
:10E2C000E080F180D701ED91FC910688F789E02D7F
:10E2D000C7011995811106C0C6010E9421718FEFF7
:10E2E0009FEF13C0F5019281911124C0D701ED91E8
:10E2F000FC910190F081E02D612FC7011995F70184
:10E300008789811111C090E080E00F900F900F90ED
:10E310000F90DF91CF911F910F91FF90EF90DF90C1
:10E32000CF90BF90AF900895612F82E89CE00E944B
:10E33000BD68E9CF812F8F7D81548A31B8F280ED9D
:10E34000810F8A3098F283ED810F823078F21F3589
:10E3500069F21E3759F21132B1F086EC810F82302A
:10E3600090F08AED810F873070F01D3361F0812FBE
:10E370008F7E8F3241F08DED810F823020F01B3582
:10E3800011F01D3511F491FFB1CF19821A821B8251
:10E390001C82812F012E000C990B9F931F938DE6F9
:10E3A00095E09F938F938E010F5F1F4F1F930F93E5
:10E3B0000E94B9BE6E01F4E0CF0ED11C0F900F90F9
:10E3C0000F900F900F900F90D8016D918D01D70194
:10E3D000ED91FC910190F081E02DC7011995F701B5
:10E3E0008789882339F0F8013197608182E89CE0C1
:10E3F0000E94BD680C151D0539F785CFCF93C82F36
:10E40000462F61E070E00E940D1F61E070E08C2FEC
:10E410000E943B1F8111F9CFCF910895AF92BF9217
:10E42000CF92DF92EF92FF920F931F93CF93DF93E0
:10E4300000D01F92CDB7DEB78C016B017A018091BD
:10E44000C20A8333E9F45B016801C40ED51EC0160D
:10E45000D106A9F10E94C3638FE00E94CE63812F91
:10E460000E94CE63802F0E94CE630F5F1F4F80E01B
:10E470000E94CE63F50181935F010E94B963E7CFEB
:10E48000843369F50E94C36319830A838F2D8F77C4
:10E490008B83EC8264E070E0CE0101960E949F6362
:10E4A000A70170E060E0C6010E9449B7E114F104E1
:10E4B00021F0B701C6010E949F630E94B963C701A2
:10E4C0000F900F900F900F90DF91CF911F910F91B0
:10E4D000FF90EF90DF90CF90BF90AF9008950E9493
:10E4E000C3630F3F110509F030F419820A831B82C0
:10E4F00063E070E0D1CF17FD0BC019820A8333E0CF
:10E50000169507953A95E1F7007E08600B83F0CFEA
:10E51000C80126E0969587952A95E1F7807E1983B4
:10E520000A830115104C18F480618B83E1CF886158
:10E53000FCCFAF92BF92CF92DF92EF92FF920F93F8
:10E540001F93CF93DF9300D000D01F921F92CDB7BF
:10E55000DEB78C017B016A018091C20A8333E1F44A
:10E560005801A40EB51EA016B10609F46FC00E9492
:10E57000C36380EF0E94CE63812F0E94CE63802F01
:10E580000E94CE630F5F1F4FF70181917F010E94B0
:10E59000CE630E94B963E7CF5B01A40EB51E84333E
:10E5A000C1F40E94C36319830A838D2D80688B8315
:10E5B000CC8264E070E0CE0101960E949F63AE14AD
:10E5C000BF0409F441C0F70181917F010E94CE632D
:10E5D000F6CF0E94C3630F3F110509F028F419829A
:10E5E0000A8384E08B830CC017FD17C019820A834D
:10E5F00033E0169507953A95E1F7007E0C600B83A2
:10E6000086E0C816D104A0F5F701DE011496EA15DC
:10E61000FB0599F081918D93FACFC80126E096957C
:10E6200087952A95E1F7807E19830A830115104C9E
:10E6300010F48461D7CF8C61D5CFB6016D5F7F4F69
:10E64000CE0101960E949F630E94B963C60128967D
:10E650000FB6F894DEBF0FBECDBFDF91CF911F91F3
:10E660000F91FF90EF90DF90CF90BF90AF90089503
:10E6700063E070E0CE0101960E949F63F7018191F3
:10E680007F010E94CE63AE14BF04C1F7DDCFCF93EC
:10E69000DF931F92CDB7DEB7898341E050E0BE0122
:10E6A0006F5F7F4F90E080E00E9499720F90DF9142
:10E6B000CF9108951F93CF93DF931F921F92CDB7F1
:10E6C000DEB780918A09811100C160E372E080E0C9
:10E6D00090E00E94CA841FB7F89480918909811143
:10E6E00027C0EFEBF5E18491E5E1F6E19491E82FA5
:10E6F000F0E0EE0FFF1FEA5AFA4EA591B491EC91AB
:10E70000E92321F461E085E30E94448361E085E32D
:10E710000E9472838CB580618CBD8CB580648CBD89
:10E7200061E084E30E94728361E083E30E9472836C
:10E73000809189098F5F809389091FBFE4E9F5E122
:10E74000E491F0E0EE0FFF1FE059FA4E85919491AD
:10E750009093880980938709EAEEF5E1E491E093CC
:10E76000860961E08AE00E9472830E94B96380E5B5
:10E7700091E00E94038084E38093C20A80E80E94B3
:10E7800047730E94B0668823A1F188E00E94477316
:10E790000E94AC66883069F580E10E9447730E9450
:10E7A000AC66803131F580E00E9447730E94AC6610
:10E7B000182F81111EC08FE190E00E942A1F833024
:10E7C000C1F480E480937A0942E06EE170E0812F29
:10E7D0000E940D1F42E06FE170E0812F0E940D1F2B
:10E7E0001F5F183089F70E94512081E080938A09C9
:10E7F00066C087E38093C20A80E80E9447730E9444
:10E80000B0668823F9F088E00E9447730E94AC66E6
:10E810008830C1F480E10E9447730E94AC66182FD3
:10E82000803181F480E00E9447730E94AC668111C0
:10E8300009C089E390E00E942A1F843019F41093E4
:10E840007A09D1CF83E38093C20A80E80E9447739C
:10E850000E94B066882371F180E10E9447730E9494
:10E86000AC66803139F582E10E9447730E94AC6644
:10E87000823101F580E00E9447730E94AC668111ED
:10E8800019C084E080937A0915E51A8341E050E0CD
:10E89000BE016E5F7F4F8BE190E00E9499721983F9
:10E8A00041E050E0BE016F5F7F4F8AE190E00E943F
:10E8B000997299CF1092C20A0E94512080E00F9065
:10E8C0000F90DF91CF911F91089581E0F8CF6F9263
:10E8D0007F929F92AF92BF92CF92DF92EF92FF9280
:10E8E0000F931F93CF93DF931F921F92CDB7DEB785
:10E8F000982E8B013A01690122E030E0AE014F5FB2
:10E900005F4F64E270E00E942B20E980FA80FE24D1
:10E91000EF24FE24E00EF11E970137704091C20AE9
:10E92000092D10E0C801433309F04CC00896982F18
:10E930008827990F990F990F820F931F473309F476
:10E9400046C0A9014C0D5D1D4130584008F43FC040
:10E9500060E078E05B01A21AB30AA501B3010E944E
:10E960009972A6014A195B09B3016A0D7B1D80915A
:10E97000C20A833349F5085F1F4F000F000F000FD5
:10E9800080E0902F0E949972EC0CFD1CF982EA82C3
:10E9900022E030E0AE014F5F5F4F64E270E0892D0E
:10E9A0000E94FC1E0F900F90DF91CF911F910F914D
:10E9B000FF90EF90DF90CF90BF90AF909F907F90AF
:10E9C0006F9008954096B3CF005F1F4FD6CFA6013A
:10E9D000B301D8CFEF92FF921F93CF93DF931F9293
:10E9E0001F92CDB7DEB7182F22E030E0AE014F5FA7
:10E9F0005F4F60E270E00E942B20E980FA80FE24E5
:10EA0000EF24FE2422E030E0AE014F5F5F4F60E272
:10EA100070E0812F0E942B2089819A819827892775
:10EA20009827E816F90689F487E0189FF001112469
:10EA3000E658F54FF582E482C7010F900F90DF9101
:10EA4000CF911F91FF90EF9008957C01DBCF1F9332
:10EA5000CF93DF93182F80E591E00E940380812FF0
:10EA60000E94EA74EC01812F0E94491F182F0E9416
:10EA70005120173121F01C3111F0D0E0C0E0CE015F
:10EA8000DF91CF911F910895CF92DF92EF92FF9285
:10EA90000F931F93CF93DF93182F7B01EA0141302F
:10EAA000584010F0C0E0D8E080E591E00E9403807B
:10EAB000812F0E94EA746C01812F0E94491F082F48
:10EAC0000E945120073111F00C3169F5CC16DD069A
:10EAD00058F380E591E00E9403809E01A70170E059
:10EAE00060E0812F0E94677460E270E0812F0E94D5
:10EAF000FE7162E070E0812F0E943B1F84FD1DC00B
:10EB0000812F0E94491F811111C00E945120D0E025
:10EB1000C0E0CE01DF91CF911F910F91FF90EF9058
:10EB2000DF90CF900895D0E0C0E0D3CF0E94512075
:10EB300080E591E00E940380DCCF40E162E070E07C
:10EB4000812F0E940D1F0E945120E3CF1F93CF936E
:10EB5000DF931F92CDB7DEB7182F80E591E00E94BA
:10EB60000380812F0E94D56327E0129FF0011124BA
:10EB7000E658F54F22813381377041E050E0BE0105
:10EB80006F5F7F4F820F931F0E940E720E94512071
:10EB900089810F90DF91CF911F9108950F931F935B
:10EBA000CF93DF93C82F27E0829F8001112406585E
:10EBB000154FF80180819181009791F480E591E0F3
:10EBC0000E9403808C2F0E94C666EC010E94512097
:10EBD000F80186819E01281B3109C90131832083F8
:10EBE000DF91CF911F910F9108954F925F927F9285
:10EBF0008F929F92AF92BF92CF92DF92EF92FF924D
:10EC00000F931F93CF93DF931F921F92CDB7DEB761
:10EC1000782E6B014A01A82EB12C27E0829FC001FB
:10EC20001124FC01E658F54F7F010081118180E538
:10EC300091E00E9403800815190554F4872D0E9465
:10EC4000C666F70126818C01021B1109118300831E
:10EC50000115110529F5872D0E94491F843159F0AE
:10EC6000882349F001E010E08C3111F410E000E05D
:10EC70001195019511090E945120C8010F900F9024
:10EC8000DF91CF911F910F91FF90EF90DF90CF9088
:10EC9000BF90AF909F908F907F905F904F9008951E
:10ECA000801691060CF4840187E08A9DF0018B9D0B
:10ECB000F00D1124E658F54FE280F380C114D10421
:10ECC00051F12701F7E05F22872D0E94D563840D63
:10ECD000951D2091C20A273309F453C09801240DD1
:10ECE000351D2130384008F44CC020E038E049019F
:10ECF00084189508A401B6010E940E722601480CE2
:10ED0000591C6801C818D908872D0E94D563A6012F
:10ED1000B2010E940E72E00EF11E87E08A9DF001A2
:10ED20008B9DF00D1124E658F54FF382E28220818D
:10ED30003181201B310B318320838681800F912FFD
:10ED4000911D8A3F910510F4232BF1F487E08A9DF1
:10ED5000F0018B9DF00D1124E658F54F1682F982D3
:10ED6000EA8222E030E0AE014F5F5F4F68E270E080
:10ED7000872D0E94FC1E60E470E0872D0E94FE71CA
:10ED80007ACFA801B601C5CF868375CFCF93C82FA0
:10ED900080E591E00E94038068E070E08C2F0E9483
:10EDA000FE71CF910C945120CF93C82F80E591E054
:10EDB0000E94038060E170E08C2F0E94FE71CF9171
:10EDC0000C945120CF93C82F80E591E00E940380DE
:10EDD0008C2F0E94491FC82F0E9451208C2FCF9149
:10EDE0000895CF93DF931F921F92CDB7DEB779833B
:10EDF0006A8322E030E0AE014F5F5F4F60E170E078
:10EE00000E94FC1E0F900F90DF91CF910895CF9339
:10EE1000DF931F921F92CDB7DEB779836A8322E01A
:10EE200030E0AE014F5F5F4F64E070E00E94FC1E77
:10EE30000F900F90DF91CF9108958F929F92AF9294
:10EE4000BF92CF92DF92EF92FF920F931F93CF93D7
:10EE5000DF9300D000D000D01F92CDB7DEB79091E5
:10EE6000C20A992369F128E0F22E933311F494E059
:10EE7000F92E6B01082F80E591E00E9403809E012E
:10EE80002F5F3F4F5901490110E0812F0E94491F18
:10EE9000F40181934F018823D9F01F5FF112F5CF60
:10EEA000F12CF50191915F019D3161F0983151F0A4
:10EEB0009A51923038F0F3941F11F3CF0E945120F1
:10EEC00018E05EC060E170E08F2D0E94FE711F2D82
:10EED000E12EF12CF701EE0FFF1FEE54F54F1182DA
:10EEE00010820E94FE7F402F70E060E0812F0E9420
:10EEF0000D1F4FEF62E070E0812F0E940D1FB601E1
:10EF0000CD2891F480910102909102020196811521
:10EF1000F0EC9F0708F448C090930202809301022E
:10EF20006091010270910202812F0E94077761E0D7
:10EF300070E0812F0E94FE7127E02E9DC0012F9D61
:10EF4000900D11249C012658354F7901F901118249
:10EF5000108222E030E0AE01475F5F4F68E270E070
:10EF6000812F0E942B2089859A85982789279827A9
:10EF7000F701938382831682158214820E945120A6
:10EF8000812F2A960FB6F894DEBF0FBECDBFDF915A
:10EF9000CF911F910F91FF90EF90DF90CF90BF9096
:10EFA000AF909F908F90089580E090ECB5CF4F92F6
:10EFB0005F926F927F928F929F92AF92BF92CF9209
:10EFC000DF92EF92FF920F931F93CF93DF93EC01A9
:10EFD0004B017A012901DB010D911C918881882365
:10EFE00009F45AC05E01FE0181E090E021912223E4
:10EFF00021F02E3211F00196F9CF6C01B1E0CB1A5D
:10F00000D108F7013196D701CC923E01680E791EE6
:10F010002BE030E0D5018D915D01A615B70509F50E
:10F02000CC0EDD1EE601BFEFCB1ADB0A88818E32E3
:10F03000C9F32C30310591F28091590D90915A0D00
:10F040004CE050E06A01C21AD30ADC01ED91FC9158
:10F050000280F381E02DA601B70119950C0D1D1D4D
:10F06000BDCF80832150310931961216130694F2D8
:10F070008091590D90915A0DDC01ED91FC91028027
:10F08000F381E02D4CE050E0B7011995045F1F4F6C
:10F09000F7012CE030E0BECF452891F0F701108257
:10F0A0008091590D90915A0DDC01ED91FC910280F7
:10F0B000F381E02D41E050E0B70119950F5F1F4F3C
:10F0C000F40111830083DF91CF911F910F91FF9085
:10F0D000EF90DF90CF90BF90AF909F908F907F90F8
:10F0E0006F905F904F900895CF92DF92EF92FF92D2
:10F0F0000F931F93CF93DF931F921F92CDB7DEB76D
:10F100006C018B01DC018D919C919A83898389E547
:10F11000E82E8DE0F82E21E030E0AB01BE016F5FFC
:10F120007F4FF701828993890E94D777D8011C927B
:10F1300081E011968C93119790E812969C93129708
:10F1400013968C93F70180819181DC01ED91FC9104
:10F150000280F381E02D44E050E0B80119958981E7
:10F160009A8104969A83898380E090E0A0E0B8E7D2
:10F17000F80180839183A283B38380E094E0958338
:10F180008483D70115962C91159716969C91169706
:10F1900017968C91179714963C9114973683278372
:10F1A000908781878D919C91DC01ED91FC9102808B
:10F1B000F381E02D4AE050E0B801199589819A81E8
:10F1C0000A96F601918380830F900F90DF91CF9183
:10F1D0001F910F91FF90EF90DF90CF900895AF9225
:10F1E000BF92CF92DF92EF92FF920F931F93CF9334
:10F1F000DF931F921F92CDB7DEB77B016A015901E1
:10F20000FB01208131813A8329838C01065F1F4FE6
:10F21000F801EE0FFF1FE75AF24F0190F081E02D49
:10F22000A114B10459F1868197819501A601BE010F
:10F230006F5F7F4F0E94D777AB2871F4000F111FCB
:10F24000F801E75AF24F0190F081E02D828193811D
:10F250000097B9F0019709F189819A81F7019183AB
:10F2600080830F900F90DF91CF911F910F91FF90AE
:10F27000EF90DF90CF90BF90AF90089584819581FB
:10F28000D4CF8EE796E021E030E0A601BE016F5FAB
:10F290007F4F01960E94D777DFCF82E796E0F3CFCA
:10F2A0008F929F92AF92BF92CF92DF92EF92FF9296
:10F2B000CF93DF93EC014A015B01C12CD12C760185
:10F2C000CE010E943312882399F0C814D904EA04AD
:10F2D000FB0474F4CE010E94F610892B89F38FEFA2
:10F2E000C81AD80AE80AF80ACE010E94D310E8CF5B
:10F2F000DF91CF91FF90EF90DF90CF90BF90AF90D4
:10F300009F908F9008952F923F924F925F926F92AD
:10F310007F928F929F92AF92BF92CF92DF92EF92A5
:10F32000FF920F931F93CF93DF9300D000D01F92D3
:10F330001F92CDB7DEB78C016B010E943870019629
:10F3400019F48FEF9FEF1DC0D801ED91FC9102845D
:10F35000F385E02DC80119957C018F3F980789F34B
:10F36000D801ED91FC910684F785E02D682FC80146
:10F370001995B2E2EB16F104E9F4B601C8010E9456
:10F38000557028960FB6F894DEBF0FBECDBFDF9143
:10F39000CF911F910F91FF90EF90DF90CF90BF9092
:10F3A000AF909F908F907F906F905F904F903F9025
:10F3B0002F900895EDE2EE16F10429F0C701C097F1
:10F3C0000A9708F043C1D801ED91FC910284F385BE
:10F3D000E02DC80119957C018F3F980709F4B1CF42
:10F3E0008D9799F5D801ED91FC910284F385E02D7C
:10F3F000C80119957C01019609F4A3CFEFEFFFEF47
:10F40000F887EF83C701C097812C912C54010A978C
:10F4100008F5AAE0B0E0A50194010E9491B930E39B
:10F42000E31AF1084701FF0CAA08BB08860E971ED5
:10F43000A81EB91ED801ED91FC910284F385E02D40
:10F44000C80119957C01C097E2CF21E030E03887F0
:10F450002F83D8CFBEE2EB16F10401F1C7018F7DF7
:10F4600085349105D9F0AF81B885A50194010E943A
:10F470009CB9F60161877287838794878085807F36
:10F4800082608087D801ED91FC910684F785E02D9C
:10F490006E2DC801199590E080E073CFC501B401CD
:10F4A0000E940DB82B013C01312C212CFEE2EF16FD
:10F4B000F10499F5D801ED91FC910284F385E02DDA
:10F4C000C80119957C01312C212C20E030E040E26C
:10F4D00051E4C301B2010E946CB84B015C01B70159
:10F4E00060537109072E000C880B990B0E940DB810
:10F4F000A50194010E94FAB92B013C01B1E02B1A3D
:10F500003108D801ED91FC910284F385E02DC8010A
:10F5100019957C01C0970A97C0F2C7018F7D853489
:10F52000910509F040C0D801ED91FC910284F3856A
:10F53000E02DC80119957C01D801ED91FC918B3229
:10F54000910519F50284F385E02DC80119957C0118
:10F55000E1E0EE83B12CA12C8AE0982ED801ED9148
:10F56000FC91C701C0978A30910508F59A9C9001DB
:10F570009B9C300D11245C01A20EB31E0284F38506
:10F58000E02DC80119957C01E9CF8D9749F40284DB
:10F59000F385E02DC80119957C013FEF3E83DACF5A
:10F5A00081E08E83D7CFB1E0BE83B12CA12CEF8157
:10F5B000F885BF01FF0F880B990B0E940DB8A301BE
:10F5C00092010E946CB82B013C01B501BB0C880B69
:10F5D000990B0E940DB84B015C01FE816F2FFF0F4C
:10F5E000770B880B990B0E940DB89B01AC01C501EC
:10F5F000B4010E946CB84B015C01B101330C880B63
:10F60000990B0E940DB89B01AC01C501B4010E9489
:10F61000FAB99B01AC0160E070E080E291E40E94E5
:10F6200013BB9B01AC01C301B2010E946CB8D601AF
:10F6300019966D937D938D939C931C9718968C913E
:10F640001897807F836018968C931CCFBBE5EB16D0
:10F65000F10409F062C0D801ED91FC910284F385B8
:10F66000E02DC80119958B35910509F06ACEF60198
:10F670008085807F85608087C8010E943870D801AE
:10F68000ED91FC910284F385E02DC80119958D352B
:10F69000910509F400CFD801ED91FC910684F7851E
:10F6A000E02D682FC8011995BB24BA940E941571EA
:10F6B0007C01009709F445CEBB2031F1F601978318
:10F6C0008683C8010E943870B701C8010E948379FF
:10F6D000892B09F036CEC8010E943870D801ED910F
:10F6E000FC910284F385E02DC8011995B12C4701E6
:10F6F0008C329105D9F221E030E08D35910509F089
:10F700008DC030E020E08AC0D40113969C938E9384
:10F710001297FC0195828482D4CFBBE7EB16F104EB
:10F7200009F08AC0D801ED91FC910284F385E02DA7
:10F73000C80119958B37910509F003CEF601808534
:10F74000807F86608087C8010E943870D801ED9163
:10F75000FC910284F385E02DC80119958D37910540
:10F7600009F499CED801ED91FC910684F785E02D3E
:10F77000682FC801199599249A940E9415717C01EB
:10F78000009709F4DECD992009F44DC0F601978366
:10F790008683C8010E943870B701C8010E94557065
:10F7A000019609F4CECDC8010E943870D701199690
:10F7B0008D919C911A9711969C938E931A961C92F8
:10F7C0001E921997D801ED91FC910284F385E02DEA
:10F7D000C8011995CA9709F0B4CDC8010E943870C4
:10F7E000B701C8010E948379019609F4AACDC80126
:10F7F0000E943870D801ED91FC910284F385E02DD0
:10F80000C8011995912C57018C32910509F4B5CF97
:10F8100021E030E08D37910509F473CF88279927CF
:10F82000821B930BAECDD50113969C938E931297AA
:10F83000FC01B582A482ADCFBEE6EB16F10421F542
:10F8400019821A821B821C82D801ED91FC910484DA
:10F85000F585E02D44E050E0BE016F5F7F4FC801A9
:10F860001995049709F06DCD44E050E06BE575E023
:10F87000CE0101960E9454BE009709F062CDF601B8
:10F880002085207F20877DCDF6E6EF16F10441F537
:10F890009E012F5F3F4F790185E0D9011D928A9526
:10F8A000E9F7D801ED91FC910484F585E02D45E060
:10F8B00050E0B901C8011995059709F042CD45E01E
:10F8C00050E065E675E0C7010E9454BE009709F05C
:10F8D00038CDF6012085207F21602087118651CD0B
:10F8E000F4E7EF16F10409F02CCD19821A821B827D
:10F8F0001C82D801ED91FC910484F585E02D44E053
:10F9000050E0BE016F5F7F4FC8011995049709F061
:10F9100018CD44E050E060E675E0CE0101960E940B
:10F9200054BE009709F00DCDF6012085207F21609F
:10F93000208721E0218725CD4F925F926F927F92A1
:10F94000AF92BF92CF92DF92EF92FF920F931F93ED
:10F95000CF93DF931F921F92CDB7DEB76C015B018F
:10F960007A0128013901DB018D919C919A83898369
:10F9700021E030E0BE016F5F7F4FC6010E94EF784B
:10F98000F70110828CE08183128281E08383742CE2
:10F990006624552444244482558266827782F60187
:10F9A000EE0FFF1FE359F24F0190F081E02D04802C
:10F9B000F581E02DDF010D900020E9F7CD018E1BD0
:10F9C0009F0B0C96982789279827F70191878087A6
:10F9D0008091590D90915A0DDC01ED91FC910280BE
:10F9E000F381E02D4AE050E0B701199589819A81B1
:10F9F0000A969A83898330E020E0A701BE016F5FF9
:10FA00007F4FC6010E94EF7889819A81F501918329
:10FA100080830F900F90DF91CF911F910F91FF90F6
:10FA2000EF90DF90CF90BF90AF907F906F905F90FE
:10FA30004F900895CF93DF93FC0144815581411588
:10FA40005105C1F09A016417750708F49B01EC0198
:10FA500088819981421B530B5D834C83BC01620FEB
:10FA6000731F0E9462BEE881F9818C819D81E80F3D
:10FA7000F91F1082DF91CF9108950F931F93CF93B9
:10FA8000DF93EC018B01CE010E94F610892B21F04F
:10FA9000CE010E94D310F7CF6AE876E0CE010E9433
:10FAA000AB686AE976E0CE010E94AB686CEA76E06A
:10FAB000CE010E944A69B801CE010E94AB68CE0116
:10FAC000DF91CF911F910F910C94A7680F931F9313
:10FAD000CF93DF938B01FC01C681D781209759F02A
:10FAE000B801888199810E940BBE892B21F00A8080
:10FAF000DB81C02DF3CFCE01DF91CF911F910F910C
:10FB000008958091420C9091430C009711F480E08D
:10FB10002FC0DC01ED91FC910688F789E02D199545
:10FB20002091650C3091660C81111FC0232B79F751
:10FB30008DEF9FEF9093660C8093650C8091420C43
:10FB40009091430CDC01ED91FC910680F781E02D52
:10FB500019958091420C9091430CDC01ED91FC9140
:10FB60000488F589E02D1995D2CF81E0232B79F611
:10FB70000895CF93DF93EC01FA013296E60FF71F59
:10FB8000DC019D012C1B3D0BCF01861B970B4D917A
:10FB9000442311F04193F5CFAC01421B530B640F8A
:10FBA000751FFB013297308361507109FB0120837F
:10FBB000DF91CF910895462F50E070E060E02AE099
:10FBC0000C945B68FC0186819781009739F066236D
:10FBD00029F06150FC0182819381F7CF0895AB0138
:10FBE000770F660B770B2AE030E00C94C468FF9225
:10FBF0000F931F93CF93DF93F12C61157105D9F10A
:10FC0000EB018C01CB010E94BA2FF82E882399F1C9
:10FC1000EC81FD813097B1F080858F708250823009
:10FC200088F4D80114964D915D916D917C91179750
:10FC30004187528763877487EC81FD818085807F4F
:10FC400082608087EC81FD81309761F090859F70A4
:10FC50008EEF890F823030F4D80112968C91807F1C
:10FC6000982B90876CE876E18FE19DE00E94B06967
:10FC7000C8010E9428278F2DDF91CF911F910F91EE
:10FC8000FF900895DC011696ED91FC9180E030978D
:10FC900029F08F5F0280F381E02DF9CF0895CF9393
:10FCA000DF938091CE0D9091CF0D009719F1DC017B
:10FCB000ED91FC910684F785E02D70E060E01995E8
:10FCC000C4EED2E08091CE0D9091CF0DDC01ED918C
:10FCD000FC910284F385E02D19952991022E000CE8
:10FCE000330B8217930731F4B2E0C83EDB0751F7BC
:10FCF00081E001C080E0DF91CF9108956115710529
:10FD0000C1F0DC011696ED91FC911797309731F414
:10FD100017967C936E9316970895FC0182819381C8
:10FD20000097D9F773836283DB011596FC93EE93FA
:10FD3000149708958F929F92AF92BF92EF92FF9285
:10FD40000F931F93CF93DF938C017B0149015A01DD
:10FD50000E941571EC01892B09F18885807F8260F2
:10FD6000888789869A86AB86BC8688819981009728
:10FD700011F00E9428AEC7010E94C9BD99838883F3
:10FD8000BE01C801DF91CF911F910F91FF90EF90BD
:10FD9000BF90AF909F908F900C947E7EDF91CF911B
:10FDA0001F910F91FF90EF90BF90AF909F908F9019
:10FDB00008954F925F926F927F928F929F92AF922F
:10FDC000BF92CF92DF92EF92FF926B017C01AC0168
:10FDD0009B010E946EBB6BEB76E0811126C0460151
:10FDE0005701E894B7F82FEF3FEF4FE75FE7C50102
:10FDF000B4010E946EBB81110CC02FEF3FEF4FE7A3
:10FE00005FE7C501B4010E9406B86FEB76E01816F3
:10FE100064F02FEF3FEF4FE75FE4C701B6010E94A8
:10FE20000EBB181694F463EC76E08FE19DE0FF9032
:10FE3000EF90DF90CF90BF90AF909F908F907F908A
:10FE40006F905F904F900C944C682FEF3FEF4FE70F
:10FE50005FECC701B6010E9406B887FDE4CF20E041
:10FE600030E0A901C701B6010E9406B8B12CA12C4F
:10FE700087FF0AC06DE28FE19DE00E94BD685C01D2
:10FE8000F7FAF094F7F8F0942AE037ED43EA5BE3F1
:10FE9000C701B6010E94FAB92B013C010E94DFBAEA
:10FEA0006B017C010E940BB89B01AC01C301B20144
:10FEB0000E94F9B92B013C012AE0B701A6018FE1AC
:10FEC0009DE00E945B687C01EA0CFB1C6EE28FE106
:10FED0009DE00E94BD68E80EF91E20E030E040E29F
:10FEE00051E4C301B2010E946CB82B013C010E9495
:10FEF000DFBA4B01B12CA12C2AE0B501A4018FE19E
:10FF00009DE00E945B68E80EF91EC501B4010E94E5
:10FF10000BB89B01AC01C301B2010E94F9B920E00A
:10FF200030E040E251E40E946CB80E94DFBAAB01BD
:10FF300070E060E02AE08FE19DE00E945B688E0D3A
:10FF40009F1DFF90EF90DF90CF90BF90AF909F905C
:10FF50008F907F906F905F904F9008950F931F93B5
:10FF6000CF93DF93EC01209731F10A811B818885C3
:10FF70008295807F859585958595859583FD06C0BD
:10FF80008E819F81009711F00E94AE7F88858F70CF
:10FF9000843031F489859A85009711F00E9428AE4B
:10FFA00088819981009711F00E9428AECE010E94AD
:10FFB00028AEE801D8CFDF91CF911F910F9108951E
:10FFC0000F931F93CF93DF938C010E941571EC0167
:10FFD000892B71F0C8010E943870BE01C8010E94CF
:10FFE0008379019629F4CE010E94AE7FD0E0C0E073
:10FFF000CE01DF91CF911F910F91089583EE93E091
:020000021000EC
:100000000197F1F708958CBD9DBD0895EF92FF9281
:100010000F931F93CF93DF9300D01F92CDB7DEB71E
:100020001092C30A02967C0110E000E0F701819172
:100030007F014AE0BE016F5F7F4F90E00E9422B1D6
:1000400040E150E0BE016F5F7F4F83EC9AE00E9479
:1000500044BE0330110531F06BE675E083EC9AE0A5
:100060000E941EBE0F5F1F4F04301105F9F683EC8E
:100070009AE00F900F900F900F90DF91CF911F910A
:100080000F91FF90EF900895AF92BF92CF92DF92C1
:10009000EF92FF920F931F93CF93DF936C017B013D
:1000A000BA015901D7010D911C91FC01C081D18188
:1000B00080E090E0021713075CF0A901CE010E94D6
:1000C000E3BD31E020E0892B09F030E0832F922F4F
:1000D000FE01EA0DFB1DD601ED93FC930A191B09E5
:1000E000D7010D931C9320812E3249F43196D6010D
:1000F000ED93FC9301501109F70111830083DF9107
:10010000CF911F910F91FF90EF90DF90CF90BF9014
:10011000AF90089520E3FC0120833296862F8295CC
:100120008F706F706A3030F4605D6293682F811158
:10013000F5CF0895695CF9CF0F931F93CF93DF93A9
:10014000009739F490E080E0DF91CF911F910F91FB
:100150000895EC0180916B0D90916C0D009711F05A
:100160000E9428AEFE0101900020E9F7CF018C1B10
:100170009D0B06960E948CAD8C0190936C0D809324
:100180006B0D0097F9F2BE010E943DBEFE01019089
:100190000020E9F73197CF018C1B9D0B63E876E0D7
:1001A000800F911F0E943DBE81E090E0CDCFCF92A5
:1001B000DF92EF92FF920F931F93CF93DF936C0127
:1001C000EB017A0189010E945A73882331F180E59D
:1001D00091E00E94038046E050E060ED7DE089E020
:1001E00090E00E949972C60102960E943C20C701CD
:1001F00002960E944A20C80102960E9443200E9453
:1002000051208A819B81AC81BD818093360C909373
:10021000370CA093380CB093390CDF91CF911F911C
:100220000F91FF90EF90DF90CF900895CF92DF92E3
:10023000EF92FF92CF93DF93CDB7DEB768970FB6FB
:10024000F894DEBF0FBECDBFFA012BE933E03A834D
:1002500029835FEF5B835C835D831E8238872F83F6
:10026000C280D380E480F580C986DA86EB86FC867E
:100270003E872D87FB0142815381648175814F87C1
:10028000588B698B7A8B3C8B2B8BFC018281938101
:10029000A481B5818D8B9E8BAF8BB88F9E012F5F14
:1002A0003F4FAE01495F5F4FBE01635F7F4FCE019D
:1002B00043960E94D78068960FB6F894DEBF0FBEB3
:1002C000CDBFDF91CF91FF90EF90DF90CF90089559
:1002D0000F931F93CF93DF93CDB7DEB768970FB619
:1002E000F894DEBF0FBECDBFFB01DC0112964D912D
:1002F0005D916D917C9115974D8B5E8B6F8B788F97
:100300008BE993E09A83898321E0288F0D891E89E8
:100310002F89388D0B831C832D833E8398878F8391
:10032000028113812481358109871A872B873C87B5
:100330009E878D874F87588B698B7A8BAE014F5F75
:100340005F4FBE01695F7F4FCE010D960E941681FF
:1003500068960FB6F894DEBF0FBECDBFDF91CF9188
:100360001F910F910895CF93DF93CDB7DEB76297BA
:100370000FB6F894DEBF0FBECDBFFC018281938122
:10038000A481B5818F87988BA98BBA8B2BE933E039
:100390003A83298341E04A8B4F85588969897A8954
:1003A0004B835C836D837E8338872F8389879A870D
:1003B000AB87BC87BE016F5F7F4FCE0107960E945F
:1003C000688162960FB6F894DEBF0FBECDBFDF9195
:1003D000CF910895CF93DF93EC016DE00E94CB673E
:1003E000811103C0CE010E94DF67CE01DF91CF9162
:1003F00008958F929F92AF92BF92CF92DF92EF9229
:10040000FF920F931F93CF93DF93CDB7DEB7609723
:100410000FB6F894DEBF0FBECDBF7C019091C20A2B
:10042000992351F108E0933309F404E06B0180E56E
:1004300091E00E9403809E012F5F3F4F59014901C7
:1004400010E0812F0E94491FF40181934F018823FE
:10045000D9F01F5F0113F5CF00E0F50181915F0135
:100460008D3161F0883151F08A51823038F00F5F60
:100470001013F3CF0E94512018E088C060E170E0B3
:10048000802F0E94FE71102FA12EB12CF501EE0FCE
:10049000FF1FEE54F54F118210820E94FE7F42E84A
:1004A00070E060E0812F0E940D1F4FEF62E070E06E
:1004B000812F0E940D1FB601C114D10491F48091C7
:1004C00001029091020201968115F0EC9F0708F459
:1004D00071C09093020280930102609101027091B9
:1004E0000202812F0E94077786E0EDEDF2E0DE0147
:1004F000199601900D928A95E1F7F70183818F7724
:100500008C8784818D8785818E87A7014E5F5F4FA1
:1005100024E030E06CE070E0812F0E94FC1EB60108
:10052000812F0E94F17626E030E0AE01475F5F4FF9
:1005300066E070E0812F0E94FC1E61E070E0812F78
:100540000E94FE7127E02A9DC0012B9D900D112471
:100550009C012658354F7901F9011182108222E061
:1005600030E0AE01415F5F4F68E270E0812F0E9492
:100570002B208F859889982789279827F7019383BF
:1005800082831682158214820E945120812F6096E8
:100590000FB6F894DEBF0FBECDBFDF91CF911F9194
:1005A0000F91FF90EF90DF90CF90BF90AF909F9012
:1005B0008F90089580E090EC8CCF8250823108F0CB
:1005C0005FC0E82FF0E08827E751FD478F4F0C947C
:1005D000DBB93D834183FB8201830583408309832B
:1005E0000F83138319831D83218327832B834083E8
:1005F0002F8335833983809180008F7780938000AB
:100600000895809180008F7DF9CF80918000877F51
:10061000F5CF8091B0008F778093B00008958091DE
:10062000B0008F7DF9CF809190008F7780939000FC
:100630000895809190008F7DF9CF80919000877F01
:10064000F5CF8091A0008F778093A00008958091CE
:10065000A0008F7DF9CF8091A000877FF5CF80919A
:1006600020018F77809320010895809120018F7D54
:10067000F9CF80912001877FF5CF84B58F7784BD36
:10068000089584B58F7DFBCF1F93CF93DF93282FE1
:1006900030E0F901EA5CF94E8491F901E052FA4E3A
:1006A000D491F901E657FA4EC491CC23A9F0162F44
:1006B00081110E94DD82EC2FF0E0EE0FFF1FE05968
:1006C000FA4EA591B4918FB7F894EC91111108C02E
:1006D000D095DE23DC938FBFDF91CF911F910895DA
:1006E000DE2BF8CFCF93DF9390E0FC01E052FA4E7F
:1006F000249186579A4EFC0184918823C9F090E09A
:10070000880F991FFC01EA5AFA4EA591B491FC0199
:10071000E059FA4EC591D49161110DC09FB7F8947C
:100720008C91209582238C938881282328839FBFD6
:10073000DF91CF910895623051F49FB7F8943C91C6
:10074000822F809583238C93E8812E2BEFCF8FB758
:10075000F894EC912E2B2C938FBFEACF1F93CF935D
:10076000DF93182FEB0161E00E947283209739F428
:1007700060E0812FDF91CF911F910C944483CF3F94
:10078000D10511F461E0F5CFE12FF0E0EA5CF94E1C
:10079000E491E250E23108F0B3C0F0E08827EC5277
:1007A000FC478F4F0C94DBB9E683EE83F383FD8324
:1007B000078480841184198421842B8435843F84A8
:1007C0004E845884808462846C84768484B5806886
:1007D00084BDC7BDDF91CF911F91089584B580621C
:1007E00084BDC8BDF7CF8091800080688093800071
:1007F000D0938900C0938800EDCF80918000806203
:1008000080938000D0938B00C0938A00E3CF8091C7
:100810008000886080938000D0938D00C0938C000E
:10082000D9CF8091B00080688093B000C093B300AE
:10083000D1CF8091B00080628093B000C093B400AB
:10084000C9CF80919000806880939000D0939900E8
:10085000C0939800BFCF80919000806280939000F9
:10086000D0939B00C0939A00B5CF80919000886090
:1008700080939000D0939D00C0939C00ABCF80915B
:10088000A00080688093A0008091A0008F7B80935F
:10089000A000D093A900C093A8009CCF8091A00095
:1008A00080628093A000D093AB00C093AA0092CF47
:1008B0008091A00088608093A000D093AD00C09389
:1008C000AC0088CF80912001806880932001D09374
:1008D0002901C09328017ECF8091200180628093FE
:1008E0002001D0932B01C0932A0174CF8091200165
:1008F000886080932001D0932D01C0932C016ACF92
:10090000C038D1050CF03ECF33CF803120F0853395
:1009100008F485E3865320917B00982F9870277FF9
:10092000922B90937B008770806480937C008091F1
:100930007A00806480937A0080917A0086FDFCCFF3
:10094000809178009091790008953FB7F894809154
:100950001B0E90911C0EA0911D0EB0911E0E26B57F
:10096000A89B05C02F3F19F00196A11DB11D3FBFE7
:10097000BA2FA92F982F8827BC01CD01620F711DB6
:10098000811D911D42E0660F771F881F991F4A95B0
:10099000D1F708958F929F92AF92BF92CF92DF923C
:1009A000EF92FF924B015C010E94A5846B017C01D8
:1009B0000E94A5846C197D098E099F09683E7340C9
:1009C00081059105A8F321E0821A9108A108B108D8
:1009D00088EEC80E83E0D81EE11CF11C811491043E
:1009E000A104B10429F7FF90EF90DF90CF90BF9062
:1009F000AF909F908F900895EF92FF920F931F9367
:100A0000CF93DF93EC017B018A01CE010E94F610A7
:100A1000892B21F0CE010E94D310F7CF67EC76E04E
:100A2000CE010E944A69B701CE010E94EF7D6FECB2
:100A300076E0CE010E944A69B801CE010E94AB68FF
:100A40006AE976E0CE010E94AB68CE010E94A768F9
:100A500064EF71E080E090E00E94CA84CE01DF91F3
:100A6000CF911F910F91FF90EF900C94A0562FB74C
:100A7000F8946091170E7091180E8091190E909154
:100A80001A0E2FBF0895EF92FF920F931F93CF93EB
:100A9000DF9300D01F92CDB7DEB7FA0120E08E01C0
:100AA0000F5F1F4F9E2F9F77EE0FEF2FEE1FFF0B55
:100AB000F195309709F09068D801A20FB11D9C9371
:100AC0002F5F309779F730E0FB01E21BF30B848353
:100AD000FB01E21BF30B3596D801CD01801B910B76
:100AE000821793071CF48D918193F7CF2F5F3F4FAF
:100AF0008091420C9091430C8901040F151F621BD9
:100B0000730B6B5F7F4FDC01ED91FC910280F381F1
:100B1000E02DA80119957C010E94378560934E0C49
:100B200070934F0C8093500C9093510C81E00E15F4
:100B30001F0509F080E00F900F900F900F90DF914C
:100B4000CF911F910F91FF90EF900895AF92BF92B8
:100B5000CF92DF92FF920F931F93CF93DF936C019D
:100B6000EB018A01F22E0E94817D882309F442C0A4
:100B7000A090460CB090470CB501C6010E94F0B0A1
:100B80009801295F3F4F820F931FA816B90690F175
:100B90006091440C7091450C45E050E0C6010E9404
:100BA000B97DAC019E01200F311FFE01EC01CE1B6F
:100BB000DF0BDE01AE0FBF1F6091440C7091450C3E
:100BC000E217F30729F08191A60FB71F8C93F1CF9D
:100BD0000550110980E3F11081E3400F511FDF91AF
:100BE000CF911F910F91FF90DF90CF90BF90AF906A
:100BF0000C94438580E0DF91CF911F910F91FF907E
:100C0000DF90CF90BF90AF9008950F931F93CF9335
:100C1000DF938C01EB0190E080E0209739F0609148
:100C2000460C7091470CCE010E94F0B021E0AC015F
:100C3000BE01C801DF91CF911F910F910C94A68541
:100C40000F931F93CF93DF938C01EB0190E080E033
:100C5000209739F06091460C7091470CCE010E94AC
:100C6000F0B020E0AC01BE01C801DF91CF911F912F
:100C70000F910C94A6850F931F93CF93DF93EC01F4
:100C80000091460C1091470CB8010E94F0B00996F3
:100C900008171907E8F10E94817D8823C9F1809126
:100CA0004C0C90914D0C019681F190934D0C8093DA
:100CB0004C0CE091440CF091450C80914D0C8583D7
:100CC000E091440CF091450C80914C0C868360912E
:100CD000440C7091450C47E050E0CE010E94B97D74
:100CE000E091440CF091450CE80FF91F1082AC0123
:100CF000445051096091440C7091450C82E8DF9199
:100D0000CF911F910F910C94438581E090E0CDCF5E
:100D100080E0DF91CF911F910F9108950F931F9362
:100D2000CF93DF93EC010E943785688779878A87A4
:100D30009B87CE010E94D31097FF15C00E94378574
:100D4000088519852A853B85601B710B820B930BE7
:100D50000C811D812E813F816017710782079307E7
:100D600040F38FEF9FEFDF91CF911F910F91089587
:100D70008F929F92AF92BF92CF92DF92EF92FF92AB
:100D8000CF93DF93EC010E9437854B015C0180918A
:100D9000420C9091430CDC01ED91FC910084F185B3
:100DA000E02D1995892BB9F40E9437856B017C01E0
:100DB000C818D908EA08FB0820914A0C30914B0C5E
:100DC000A8EEB3E00E94A4B9C616D706E806F90655
:100DD000F0F280E00DC08091420C9091430CDC0158
:100DE000ED91FC910284F385E02D1995888381E0D3
:100DF000DF91CF91FF90EF90DF90CF90BF90AF90B9
:100E00009F908F9008952F923F924F925F926F9292
:100E10007F928F929F92AF92BF92CF92DF92EF928A
:100E2000FF920F931F93CF93DF9300D000D000D099
:100E30001F92CDB7DEB71C018091440C9091450CF8
:100E40000E94B88681111CC060E070E0CB012A9638
:100E50000FB6F894DEBF0FBECDBFDF91CF911F91CB
:100E60000F91FF90EF90DF90CF90BF90AF909F9049
:100E70008F907F906F905F904F903F902F9008954C
:100E8000E091440CF091450CD0801982EE24E3945B
:100E9000F12C812C912C5401412C512C3201439482
:100EA000CE0101960E94B886882371F287010F5FF8
:100EB0001F4F8981E091440CF091450CEE0DFF1D10
:100EC0008083E981AE2FAF77B0E0A30192010E9449
:100ED00091B9860E971EA81EB91E37E0440C551C0A
:100EE000661C771C3A95D1F7E7FD3FC0BD2DB07F5A
:100EF000BE838FEF800FF1018083B03309F04CC0C7
:100F00008091440C9091450C800F911F0E94B886EF
:100F1000882309F499CF2091440C3091450CC701E6
:100F20000296820F931F0E94B886882309F48CCF03
:100F30000E5F1F4FE091440CF091450CD1018C9154
:100F4000DF01A80FB11D11968C91119790E0982F99
:100F5000882712962C91820F911D208121FD0296E7
:100F6000F2E0E0E030E020E01DC07801053011053E
:100F700009F096CF8FEF9FEF9093660C8093650CEE
:100F80008091420C9091430CDC01ED91FC9104881E
:100F9000F589E02D199558CFF0E0E0E030E020E051
:100FA00090E080E070E060E0CF2EDE2EE32EF22EA7
:100FB00028013B014C185D086E087F084A825B825D
:100FC0006C827D822C01712C612C4F82588669863F
:100FD0007A864A805B806C807D804C0C5D1C6E1C28
:100FE0007F1CC814D904EA04FB0408F046C0CE01F3
:100FF00001960E94B886882309F426CF8091630C5D
:101000009091640C009711F12E812033F9F4D101F5
:101010002C914EEF5FEF6FEF7FEF421B510961099B
:101020007109440E551E661E771E2F81388549852D
:101030005A85241535054605570540F4DC01ED9128
:10104000FC910190F081E02D698119958091460C09
:101050009091470C0817190750F48981E091440CCE
:10106000F091450CE00FF11F80830F5F1F4FBFEF22
:10107000CB1ADB0AEB0AFB0AACCF8091630C909190
:10108000640C892B69F48091460C9091470CB0E078
:10109000A0E084159505A605B70510F410E000E062
:1010A000B80190E080E0D3CECF93DF93CEE3DCE0D5
:1010B000EE81FF8180EE8083EE81FF8111828C8141
:1010C0009D816E817F81DC01ED91FC910280F38135
:1010D000E02D42E050E019958FEF9FEF98A78FA386
:1010E0008C819D81DC01ED91FC910680F781E02DE2
:1010F00019958C819D81DC01ED91FC910488F58925
:10110000E02D19950E943785688B798B8A8B9B8B94
:101110006C8B7D8B8E8B9F8BDF91CF9108954F923F
:101120005F926F927F928F929F92AF92BF92CF9277
:10113000DF92EF92FF920F931F93CF93DF93CDB780
:10114000DEB763970FB6F894DEBF0FBECDBF7C014C
:101150006B013A01FB0120E090E080E06AE0319110
:10116000332309F461C040ED430F4A3008F04DC00D
:10117000689FA001699F500D1124CA01C097830F79
:10118000911D37FD9A958F3F910549F340F3F70183
:1011900042815381648175818091450E9091460E04
:1011A000A091470EB091480E481759076A077B0770
:1011B00009F412C28701085F1F4F0E9437856F70C4
:1011C00077277C5FC8010E94CE11813009F009C2E7
:1011D0008BE993E09A838983F70182819381A481CB
:1011E000B5818B839C83AD83BE8345E350E0BE0114
:1011F0006F5F7F4FC8010E94BD20892BA9F5D12CBC
:10120000C12CC8010E94541017C03E3209F0BFCF54
:10121000233009F4BCCFD301A20FB11D12968C93D9
:101220002F5F90E080E09BCF233009F0B0CFF30137
:101230008583CC24C394D12CC60163960FB6F89451
:10124000DEBF0FBECDBFDF91CF911F910F91FF90F9
:10125000EF90DF90CF90BF90AF909F908F907F9056
:101260006F905F904F9008950E943785F7017783C4
:10127000668342E050E0B7016A5F7F4FC8010E9479
:10128000522081E090E09A83898342E050E0BE01E1
:101290006F5F7F4FC8010E94522080E091E09A83E7
:1012A000898342E050E0BE016F5F7F4FC8010E941A
:1012B00052201A82198242E050E0BE016F5F7F4FD8
:1012C000C8010E94522042E050E0BE016F5F7F4F94
:1012D000C8010E94522042E050E0BE016F5F7F4F84
:1012E000C8010E9452205601F6018081882301F135
:1012F0006501F60181912F01882311F08E32B1F43E
:1013000046018A189B081814190474F48D8641E06C
:1013100050E0BE01635F7F4FC8010E945220A401CC
:10132000B501C8010E9452205201DECF6201E1CF17
:101330001D8641E050E0BE01635F7F4FC8010E94FF
:101340005220C12CDD24D394DA82C98242E050E0DD
:10135000BE016F5F7F4FC8010E945220DA82C982AE
:1013600042E050E0BE016F5F7F4FC8010E945220F3
:10137000C8010E948C20892B09F441CFF3E0AF2EE5
:10138000B12C230122E0420E511CDDC0F701428145
:10139000538164817581808D918DA28DB38D4817A5
:1013A00059076A077B0709F00DC1848D958DC59794
:1013B00009F008C181A192A15DEFC52EDD24DA9468
:1013C0000C970CF4AEC04CE050E0BE016F5F7F4F55
:1013D000C8010E948A108B819C81982789279827B1
:1013E0009A8B898BF7014681578129813A8142176F
:1013F000530709F0ECC097FFEAC08F7092703BEF83
:10140000C32EDD24DA94892B09F08BC06F80788499
:101410007624672476242AEFC22EDD24DA94611420
:10142000710409F47EC0D12CC12C8D819E81982736
:1014300089279827C816D906F8F441E050E0BE0184
:10144000635F7F4FC8010E948A104D85442331F0AD
:1014500050E070E060E0C8010E948A108D85811123
:10146000ECCF44E050E070E060E0C8010E948A10D8
:10147000FFEFCF1ADF0AD9CF912C812C41E050E049
:10148000BE016D5E7F4FC8010E948A104B89842F78
:10149000807C09F071C0442331F050E070E060E0DE
:1014A000C8010E948A108B898111E8CF42E050E088
:1014B000BE01615F7F4FC8010E948A1042E050E088
:1014C000BE01635F7F4FC8010E948A1044E050E074
:1014D00070E060E0C8010E948A1042E050E0BE0166
:1014E0006F5E7F4FC8010E948A108F859889498955
:1014F0005A898115914009F048C0CD84DE84DC24EE
:10150000CD24DC2481E0C816D10409F03EC0411589
:10151000544009F04EC044E050E0B201C8010E94BE
:101520008A100E94925661E070E080E090E00E9494
:10153000CA8421E0A21AB10809F463CEFFEFCF16E6
:10154000DF0609F05ECE0E9437853B014C01C801E1
:101550000E94FF10181619060CF418CF0E94378548
:1015600066197709880999096938734181059105D8
:1015700028F50E949256EBCF41E050E070E060E029
:10158000C8010E948A101B8A8ECF542745275427F2
:1015900070E060E0C8010E948A10FFEF8F1A9F0A76
:1015A0006814790409F06ACF96EFC92EDD24DA9425
:1015B000B8CFE7EFCE2EDD24DA94B3CFCC24CA9493
:1015C000DC2CAFCF6EEFC62EDD24DA94AACF4CEF21
:1015D000C42EDD24DA94A5CF8EEFC82EDD24DA9454
:1015E0002BCED12CC12C28CE1F920F920FB60F926A
:1015F00011242F933F938F939F93AF93BF93809129
:10160000170E9091180EA091190EB0911A0E3091EC
:10161000160E23E0230F2D3768F126E8230F0296DC
:10162000A11DB11D2093160E8093170E9093180ED6
:10163000A093190EB0931A0E80911B0E90911C0E60
:10164000A0911D0EB0911E0E0196A11DB11D80939B
:101650001B0E90931C0EA0931D0EB0931E0EBF91F7
:10166000AF919F918F913F912F910F900FBE0F904F
:101670001F9018950196A11DB11DD4CF4F925F9276
:101680006F927F92AF92BF92CF92DF92EF92FF92D2
:101690000F931F93CF93DF93CDB7DEB764970FB649
:1016A000F894DEBF0FBECDBF8A0179011C8A1B8A68
:1016B000FE0133962AE0DF011D922A95E9F776278D
:1016C000672776277A8369834230510509F457C02A
:1016D0006CF44130510509F45BC080E091E09887DB
:1016E0008F838B81806884608B8308C0CA010497D4
:1016F000029798F780E091E09E838D83C090590D0A
:10170000D0905A0DD601ED91FC91A488B58863E084
:1017100072E0CE010D960E94D46949EE54E1BE01FB
:10172000635F7F4FC601F50119958091590D909126
:101730005A0DDC01ED91FC910280F381E02D4CE02B
:1017400050E0BE016F5F7F4F19958B899C890C9685
:101750009C8B8B8B0330110509F4D1C13CF5013012
:10176000110509F4FAC10230110509F46CC0BE017B
:101770006F5F7F4FCE0143960E947478CCC180E0AA
:1017800094E098878F8380E091E09C878B87A9CF36
:1017900080E091E09E838D839C878B878C81807F06
:1017A00083608C838B81846080689ECF06301105B6
:1017B000F4F68091830D9091840D0530110521F090
:1017C0008091810D9091820D21E030E0AE014F5F5C
:1017D0005F4FBE016D5E7F4F0E94D7771B821982DB
:1017E00081E00530110509F48CE08A8381E08C8367
:1017F0008091590D90915A0DDC01ED91FC91028080
:10180000F381E02D4CE050E0BE016F5F7F4F1995F2
:101810008B899C890C969C8B8B8B0E94378521E051
:1018200030E00530110511F030E020E0F9013B9681
:10183000EE0FFF1FEE0FFF1FE75AF24F6083718319
:101840008283938368C130E020E0AE014F5F5F4F39
:10185000BE016D5E7F4FC7010E94EF78198281E261
:101860008A8300E80B8311E01C83412C512C612CEE
:1018700048E7742E4D825E826F827886E0916B0D10
:10188000F0916C0DDF010D900020E9F7CD018E1B6A
:101890009F0B07969827892798279A878987809191
:1018A000590D90915A0DDC01ED91FC910280F3816C
:1018B000E02D4AE050E0BE016F5F7F4F19958B89A4
:1018C0009C890A969C8B8B8B1C821B821A821982A4
:1018D0006701BAE0CB0ED11CC601880F991FFC012D
:1018E000E75AF24F5F010190F081E02D80819181F4
:1018F0009827892798279E838D838091590D9091F1
:101900005A0DDC01ED91FC910280F381E02D46E05F
:1019100050E0BE016F5F7F4F19958B899C890696B9
:101920009C8B8B8B21E030E0AE014F5F5F4FBE019F
:101930006D5E7F4F80916B0D90916C0D0E94D777FB
:1019400030E020E0AE014F5F5F4FBE016D5E7F4F24
:10195000C7010E94EF78198280E18A830B831C8380
:101960004D825E826F8278868091590D90915A0DDA
:10197000DC01ED91FC910280F381E02D48E050E024
:10198000BE016F5F7F4F19958B899C8908969C8B50
:101990008B8BD501ED91FC910084F185E02D809138
:1019A000590D90915A0D309709F074C019821A831D
:1019B0001B82DC01ED91FC910280F381E02D43E07C
:1019C00050E0BE016F5F7F4F19958B899C8903960C
:1019D0009C8B8B8B21E030E0AE014F5F5F4FBE01EF
:1019E0006D5E7F4F81E696E00E94D77719828CE08A
:1019F0008A831B8281E08C8380E090E0A0E0B8E7DE
:101A00008D839E83AF83B887F601EE0FFF1FE75AE1
:101A1000F24F0190F081E02D0680F781E02DDF018B
:101A20000D900020E9F7CD018E1B9F0B01969827A2
:101A3000892798279A8789878091590D90915A0D07
:101A4000DC01ED91FC910280F381E02D4AE050E051
:101A5000BE016F5F7F4F19958B899C890A969C8B7D
:101A60008B8B21E030E0AE014F5F5F4FBE016D5EBA
:101A70007F4FC7010E94EF7808E710E020E030E0D8
:101A8000AE014F5F5F4FBE016D5E7F4FC7010E9489
:101A90009C7C6DCEDF010D900020E9F711978D0140
:101AA0000E1B1F0B302F212F3A832983DC01ED9170
:101AB000FC910280F381E02D42E050E0BE016F5FB7
:101AC0007F4F19958B899C8902969C8B8B8B80917B
:101AD000590D90915A0DD501ED91FC91608571855C
:101AE000DC01ED91FC910280F381E02DA8011995B4
:101AF0008B899C89080F191F1C8B0B8B6BCF00E007
:101B000010E09801AE014F5F5F4FBE016D5E7F4FE9
:101B1000C7010E949C7C8091590D90915A0DDC0167
:101B2000ED91FC91008CF18DE02D199581E090E014
:101B300064960FB6F894DEBF0FBECDBFDF91CF9194
:101B40001F910F91FF90EF90DF90CF90BF90AF90DB
:101B50007F906F905F904F90089521E030E0AE014C
:101B60004F5F5F4FBE016D5E7F4F80916B0D909117
:101B70006C0D0E94D7771B8219828CE18A8381E0E9
:101B80008C838091590D90915A0DDC01ED91FC915F
:101B90000280F381E02D44E050E0BE016F5F7F4F93
:101BA00019958B899C8904969C8B8B8BE0CDAF9289
:101BB000BF92CF92DF92EF92FF920F931F93CF933A
:101BC000DF936C015B010DE61DE0F12CE12CF801C7
:101BD000819191918F01892B09F07FC08AE090E07B
:101BE0000E948CADEC01892B09F477C01986188608
:101BF0001D821C82F60101900020E9F7CF010197B8
:101C00008C199D090E948CAD8C019D838C83892B3E
